:1010000000000420F9120000211300002313000047
:101010002513000027130000291300000000000022
:10102000000000000000000000000000451C00005F
:101030002D130000000000002F130000C52C00003D
:1010400095230000331300004928000033130000EB
:101050003313000085200000331300003313000019
:1010600061250000752500003313000033130000D4
:1010700033130000F1290000331300003313000084
:101080003313000033130000331300003313000048
:101090003313000033130000331300003313000038
:1010A00033130000331300003313000089250000C0
:1010B00033130000331300000000000000000000A4
:1010C0003313000033130000331300003313000008
:1010D0003313000033130000331300008D2B000086
:1010E000331300003313000033130000000000002E
:1010F0000000000033130000000000003313000064
:1011000000000000000000000000000000000000DF
:1011100000000000000000000000000000000000CF
:1011200000000000000000000000000000000000BF
:1011300000000000000000000000000000000000AF
:10114000000000000000000000000000000000009F
:10115000000000000000000000000000000000008F
:10116000000000000000000000000000000000007F
:10117000000000000000000000000000000000006F
:10118000000000000000000000000000000000005F
:10119000000000000000000000000000000000004F
:1011A000000000000000000000000000000000003F
:1011B000000000000000000000000000000000002F
:1011C000000000000000000000000000000000001F
:1011D000000000000000000000000000000000000F
:1011E00000000000000000000000000000000000FF
:1011F00000000000000000000000000000000000EF
:101200000348044B834202D0034B03B11847704795
:101210005801002058010020000000000548064B3E
:101220001B1AD90F01EBA301491002D0034B03B1E4
:1012300018477047580100205801002000000000A6
:1012400010B5064C237843B9FFF7DAFF044B13B10E
:101250000448AFF300800123237010BD5801002023
:1012600000000000D07C020008B5044B1BB104490B
:101270000448AFF30080BDE80840CFE7000000005D
:101280005C010020D07C0200A3F5803A704700BFCB
:10129000154B002B08BF114B9D46FFF7F5FF0021B2
:1012A0008B460F461148124A121A14F035FC0C4BAB
:1012B000002B00D098470B4B002B00D09847002004
:1012C000002104000D000B4815F0ACFA14F082FB6D
:1012D0002000290001F082FE15F092FA00000800BB
:1012E0000000000000000000000004205801002061
:1012F000CC4B0020E96B01000649074A074B9B1ABB
:1013000003DD043BC858D050FBDC00F029F8FFF7A0
:10131000BFFF0000EC7D0200080000205801002003
:10132000FEE7FEE7FEE7FEE7FEE7FEE7FEE7FEE795
:10133000FEE7FEE74FF08053D3F83021082A03BFC1
:10134000D3F83401B0FA80F0400900207047000063
:10135000024AD2F80034002BFBD0704700E0014075
:1013600010B54FF08053D3F83021082A4ED14FF0FA
:1013700080420021C2F80C11C2F81011C2F83815D1
:1013800002F54042D3F80414C2F82015D3F808142B
:10139000C2F82415D3F80C14C2F82815D3F8101489
:1013A000C2F82C15D3F81414C2F83015D3F8181459
:1013B000C2F83415D3F81C14C2F84015D3F8201421
:1013C000C2F84415D3F82414C2F84815D3F82814E9
:1013D000C2F84C15D3F82C14C2F85015D3F83014B9
:1013E000C2F85415D3F83414C2F86015D3F8381481
:1013F000C2F86415D3F83C14C2F86815D3F8401449
:10140000C2F86C15D3F84434C2F87035FFF792FF78
:1014100018B1404B404AC3F88C26FFF78BFF18B138
:101420003E4BFB22C3F81825FFF784FF58B14FF05D
:1014300080424FF08051D2F8E43ED1F8581261F367
:101440000303C2F8E43EFFF775FF20B1344B4FF4BD
:101450000072C3F840264FF08053D3F83031082B88
:1014600009D14FF08043D3F80024D20744BF6FF076
:101470000102C3F800242B4AD2F8883043F47003E9
:10148000C2F88830BFF34F8FBFF36F8F4FF0805398
:10149000D3F83021082A0BD1D3F83431032B81BF84
:1014A0004FF01023D3F808224FF08043C3F858259B
:1014B0004FF01023D3F80022002A03DBD3F80432C4
:1014C000002B22DA184901234FF01020C1F804350F
:1014D0001224FFF73DFFC0F80042FFF739FFC0F8C4
:1014E0000442FFF735FF0023C1F80435FFF730FF52
:1014F000BFF34F8F0B490D4BCA6802F4E0621343F0
:10150000CB60BFF34F8F00BFFDE7094B094A1A605C
:1015100010BD00BF005000404881030000F00040B3
:101520000090024000ED00E000E001400400FA05F8
:10153000080000200090D00310B5034653E8000FC8
:101540000A4643E8002494F0000FF7D110BD10B50F
:10155000034653E8002F42EA010043E8000494F0F8
:10156000000FF6D110BD10B5034653E8000F00EA96
:10157000010243E8002494F0000FF6D110BD10B52D
:10158000034653E8002F02EB010043E8000494F007
:10159000000FF6D110BD10B5034653E8002FA2EBA3
:1015A000010043E8000494F0000FF6D110BD0121C2
:1015B000FFF7CDBF0021FFF7D6BF10B590B1D0E93E
:1015C000012301689B1ADBB20A60013BDBB2FF2BEF
:1015D000026802D10020107110BD11684C1C14600B
:1015E0000B70F2E70E20F7E738B50446002000F054
:1015F00089FB2268616813688B4215D9591E1160F6
:1016000013F8013C228AE56802FB03552268A368AF
:1016100011685B1A1179DBB2994200D21371002074
:1016200000F072FB284638BD0025F8E738B50546BE
:1016300000200C4600F066FB2A681368591C1160F4
:10164000EA68A41A2A8AB4FBF2F41C70BDE8384098
:10165000002000F059BB7047037813F0040215D046
:1016600003F00303012B03D0022B09D001207047A4
:101670000B6802880233C2F3831213440B60F5E750
:101680000B684288023303EB9213F7E7104670476A
:101690002DE9F04F414C884685B00546871C002057
:1016A000164600F02FFB6268C8F80020A36803F517
:1016B00080739B1A04F21C4804F5836A04F21449EF
:1016C000BB4217D30021002E63D005F00F05AD01FA
:1016D00045F0050565F30F016368DAB203323B4458
:1016E00044F822100020636000F00EFB012005B0DA
:1016F000BDE8F08F01214046FFF741FF5046FFF75C
:1017000056FF4846FFF753FFA0680090C0B2033071
:1017100004EB80006946FFF79FFF20BB009BDAB215
:1017200004EB8202D16801919A1C0133DBB204EB15
:1017300083030092D3F80CB001F00303012B20D0F7
:10174000022B13D083464846FFF734FF08B1009BB5
:10175000A36059464046FFF712FFA368626803F58D
:1017600080739B1AACE79DF80000D0E7BDF8063007
:10177000C3F3891303334FEA1B4B02EB930300932C
:10178000E1E7BDF80430C3F383134FEA1B4B134466
:10179000F5E7AD0545F006019EE700BF74010020A6
:1017A000064B074810B501221A7000F0B0F9044644
:1017B00010B9044800F00BFA204610BD7401002057
:1017C000D07D02000C5F0200034BD3E90130C31A45
:1017D00058425841704700BF740100202DE9F04382
:1017E00085B0FFF7F1FF002874D1724CC4F81804DB
:1017F000BFF34F8FA0680090C0B2033004EB8000AD
:101800006946FFF729FF009B18B1D4F81824002A75
:101810005CD0DAB29F1C013304EB8202DBB204EB32
:101820008303D268DB68029302F00303022B019268
:10183000009758D1BDF806305F48C3F38918464673
:10184000502E28BF502666F38F1306F10801ADF81D
:10185000063000F074F90546002800F0958000F08D
:101860009AF9002301A90822284600F0A6F9FB43B3
:10187000DBB20133F9B20331B6EB830F4FEA8309D0
:1018800004EB81012CD908234A46A6EB0906284619
:1018900000F093F9F6B2494909F10803324608F11C
:1018A0000308284607EB980700F087F90097D4F85B
:1018B0001834D4F81064002B55D0284600F06FF986
:1018C000FFF782FF80F00100C0B204E062689A4234
:1018D00004D8A260002005B0BDE8F083D8B28CE740
:1018E00008233246DBE7012B4ED1BDF804303248E5
:1018F000C3F38311062928BF062161F3891302313E
:1019000001F00F018900ADF8043000F018F9054628
:10191000002839D000F03FF90023082201A9284609
:1019200000F04BF90026BDF80420C2F38312B30087
:10193000B24203F10803BAD900994A1CC9B2033173
:10194000009204EB81010422284600F036F90136AA
:10195000E9E7F3685B7923B1336829461B683046B1
:101960009847F3681E68002EF3D1284600F017F957
:10197000304600F0C7F9D4F818340BB9009BA360C7
:10198000002000F0C1F99BE7D4F8104454B90C4B87
:101990000C480D49C01AC008000440F0020000F0D5
:1019A0005BF88DE7236820469B689847E3681C68CE
:1019B000ECE700BF74010020D07D02008001002010
:1019C000907D0200B87D0200744F02002DE9F347BC
:1019D00004460E46924601A9012218469946FFF791
:1019E00057FE1B4F10B3019D4FF00008AA1CC845BD
:1019F00008EB020123D117480021FFF79DFD80F37A
:101A00001000000440EA1440E4006B1C04F03804A9
:101A1000DBB2EDB244F0010407EB8303033544EA83
:101A2000881444EA8624D86047F825403B781BB1E7
:101A3000FFF7D4FE0028FBD102B0BDE8F087C9B2A1
:101A400007EB81015AF82830CB6008F10108CEE796
:101A5000740100209005002000231A46FFF7B6BF4E
:101A600038B5084B0125D3F810441D7004B938BDB2
:101A7000E3685D71236820465B689847E3681C68EB
:101A8000F4E700BF740100202DE9F84FB0F806A07C
:101A90004579D2F800B09DF828900AFB05F5043D81
:101AA00088460BEB0301A94203F1040488BFA5EBB0
:101AB000030BB4FBFAF607460AFB1644C2F800B063
:101AC0004EB9AAEB04055D4528BF5D46BBF1000F8A
:101AD00004D1BDE8F88F3F68013EF1E7043408EB1C
:101AE00006003C442A46B9F1000F0DD02146ABEB6D
:101AF000050B14F035FADA452E443F6855464FF091
:101B0000000428BF5D46E1E701462046EFE7FFF706
:101B100054BDF8B546790146721E0546002393422E
:101B20002D6803D30024A64202D8F8BD0133F6E79E
:101B30000F682846FFF77AFD01343946F3E72DE9AF
:101B4000F041CD1C078A0646FFF74EFD043F3D4499
:101B50000446B5FBF7F5D0B14FF48073EDB2C78002
:101B60008380013D066080460027AF4210D2304698
:101B7000FFF73AFD40B16379013363710137C8F86B
:101B8000000006608046F0E72046FFF7C2FF002411
:101B90002046BDE8F08101210430FFF7F0BC10B50C
:101BA000012104460430FFF7F6FCC0B220B92046FC
:101BB000BDE81040FFF7ADBF10BD1FB50392002276
:101BC000009203AAFFF760FF05B05DF804FB82688E
:101BD0000023936082681361826853618268D360D6
:101BE00082685360826813607047000070B5816935
:101BF000124B134A11F8025C0446D21A45B9006927
:101C00000C21B2FBF1F200218A4204D1012010E044
:101C10004FF0FF30F4E71E68AE420CD1461C02D0F4
:101C20005E68864207D19D68D4E90001D4E90223A9
:101C3000A847206070BD01310C33E5E7847D0200C8
:101C4000907D02001EF0040F0CBFEFF30880EFF34D
:101C50000980FFF7CBBF00BF38B572B6FFF700FFB2
:101C6000FFF7BCFD0028FBD1104B114C114D124960
:101C7000E41AE408240444F00100FFF7EDFED5F86F
:101C8000F030DB0700D500BE0C4944F00200FFF73E
:101C9000E3FEBFF34F8FEA68094B02F4E06213439F
:101CA000EB60BFF34F8F00BFFDE700BF907D0200E8
:101CB000B87D020000ED00E0894F0200954F020060
:101CC0000400FA051FB50021039001AA44F20100A7
:101CD000CDE90111FFF7C0FF05B05DF804FB00007E
:101CE00072B6024A1368013313607047FC06002085
:101CF000034A1368013B136003B962B6704700BF23
:101D0000FC060020FFF7ECBFFFF7F2BF074B1B5CA0
:101D10001F2B86BF064903F01F034FF0A04101228D
:101D200002FA03F3C1F80C35704700BF185F0200D8
:101D300000030050074B1B5C1F2B86BF064903F0B6
:101D40001F034FF0A041012202FA03F3C1F8083546
:101D5000704700BF185F02000003005008B5002064
:101D6000FFF7E8FF0120FFF7E5FF0220FFF7E2FFA2
:101D7000BDE808400320FFF7DDBF0000034BD3F8A8
:101D800010056FEA901000F001007047000300504A
:101D9000C10710B5044642D54FF08043D3F8403612
:101DA000DA072ED54FF01023D3F8043303F00703DE
:101DB000072B26D11D4A0123C2F80435D2F800347E
:101DC000002BFBD04FF01021D1F8043323F0070390
:101DD00043F00403C1F804330023C2F80435134A66
:101DE000D2F80034002BFBD0BFF34F8F1049114BBA
:101DF000CA6802F4E0621343CB60BFF34F8F00BFA9
:101E0000FDE74FF0A0420C490323C2F81837C2F88F
:101E10002037C1F82437C2F83037FFF79FFFA307F8
:101E200042BF054B0C22C3F8182710BD00E001404B
:101E300000ED00E00400FA050003005038B5074C3F
:101E4000051EA4F1080308BF1C4623682BB11A68BD
:101E500022605B6828469847F7E738BD10070020E6
:101E600020B9054B01225A70FFF7E8BF012802D1C3
:101E7000014A9070F8E770470007002038B50C4C15
:101E800023789BB90B486360A3602361E36000F093
:101E90005DF8054600F066F801232370064BD3F881
:101EA00000340BB10123A370284638BD8525F5E722
:101EB00000070020611E000000000140024AD2F825
:101EC0000034002BFBD0704700E0014010B5094CF6
:101ED0000123C4F80435BFF36F8FBFF34F8F016048
:101EE000FFF7ECFF0023C4F80435BFF36F8FBFF397
:101EF0004F8F10BD00E0014070B50E4E0123154616
:101F0000C6F80435BFF36F8FBFF34F8F0024AC4288
:101F100007D10023C6F80435BFF36F8FBFF34F8F8F
:101F200070BD51F8243040F82430FFF7C7FF01346A
:101F3000EDE700BF00E0014000F18040002382B0E7
:101F4000036003680193019B02B07047044B024693
:101F5000187918B91A6001229A8070478520704755
:101F600018070020084B1A68D20704D4C02283F84F
:101F7000002301221A604FF080420123C2F8183575
:101F8000024A1370704700BF00E100E01407002010
:101F900010B54FF08041D1F8003163B14FF480703B
:101FA000FFF7CAFF01220D4BC1F80823587910B979
:101FB0005A711B6898474FF08042D2F8043163B1E0
:101FC0004FF48270FFF7B8FF0223C2F80833034BC7
:101FD000BDE810401B680120184710BD18070020FD
:101FE000034BD3F83C0410F0030018BF01207047E6
:101FF0000050004070B5204A86B0137A8DF8070073
:1020000023BB9DF80730032B05D1FFF7E9FF013013
:10201000C0B28DF807009DF80730012BDCB217D055
:10202000022C13D1154D6B7A03F0FF0173B91248DE
:1020300091720126168100F05DFA0F4800F040FA17
:102040006B686E7202940BB102A8984706B070BD1F
:102050000A4B5A7A002AF9D0094A4FF48F619460EA
:10206000C2F8081300215972042102914FF48051E3
:10207000C2F808155B68E6E70C0000202007002086
:10208000005000401FB5794AD2F8043153B1D2F85C
:10209000043313F0020305D00023C2F80431BFF368
:1020A0004F8F0223714AD2F80811002900F0D8801E
:1020B000D2F80413490740F1D3800021C2F8081177
:1020C000BFF34F8F8B4214BF03200120FFF792FF15
:1020D000664BD3F81821A2B3D3F80423520630D5A7
:1020E0000021C3F81811BFF34F8F402201910092D5
:1020F000D3F810250392D3F82425C2F30B02103A2B
:10210000C2F3CC020292D3F828217AB1D3F8042387
:1021100050050BD5D3F80C2402F00D020192C3F840
:102120002811BFF34F8F0D22C3F80C24504B5B686E
:102130000BB1684698474D4B0022C3F80C21BFF302
:102140004F8F4A4BD3F81021AAB1D3F80423D106FC
:1021500011D50022C3F81021BFF34F8FCDE9012222
:102160000392102200921822C3F80823404B5B68A8
:102170000BB1684698473D4BD3F84C2172B3D3F866
:10218000042312032AD50022C3F84C21BFF34F8F3A
:10219000C3F81821BFF34F8FC3F82821BFF34F8F27
:1021A000C3F80C21BFF34F8FC3F81021BFF34F8F3B
:1021B0002F48C168C1F31301C3F808150D21C3F8F6
:1021C0000C140121C3F804144FF400230093436856
:1021D0000392CDE901220BB168469847234BD3F80F
:1021E0001C21F2B1D3F8042310061AD50022D3F82B
:1021F0000414C3F81C21BFF34F8FCDE901220392D1
:10220000C9074FF08002009207D50122C3F80424C9
:10221000174B5B680BB168469847144B0122C3F813
:102220000424124BD3F80C21BAB1D3F804231207BB
:1022300013D50022C3F80C21BFF34F8F0C4A52680C
:102240005AB108210091D3F810150291D3F81C352A
:10225000C3F3C80301936846904705B05DF804FBDB
:10226000002B3FF435AF022030E700BF00500040A4
:102270002007002000F1804382B01A68002A14BFB2
:102280000120002004D000221A601B680193019BEA
:1022900002B070470E4A1378C3B903784FF08041FB
:1022A000C3F34003C1F88035037803F00103C1F89C
:1022B0007835084B1968C90704D4C02183F8001386
:1022C0000121196001231370002070478520704799
:1022D0003C07002000E100E0014B02681A607047F3
:1022E000300700204FF080434FF46072C3F804239E
:1022F0007047000010B54FF08043D3F804436207E5
:1023000007D54FF48470FFF7B5FF10B11E4B1B6863
:102310009847A30608D54FF48A70FFF7ABFF18B1B2
:102320001A4B00201B689847600608D54FF48C7044
:10233000FFF7A0FF18B1154B01201B689847210635
:1023400008D54FF48E70FFF795FF18B1104B0020A1
:102350001B689847E20508D54FF49070FFF78AFF95
:1023600018B10B4B01201B689847A3050AD54FF401
:102370009270FFF77FFF28B1054BBDE810401B6846
:102380000220184710BD00BF380700203407002086
:102390003007002008B5FFF7ADFFBDE80840FFF7A4
:1023A000F7BD2DE9F347002406460F46904600F599
:1023B000A0754FF48039A2462B688BB1D6F8043350
:1023C00009FA04F21A420BD0C5F800A02B68019359
:1023D000A000019B00F5A07398B2D7E9003198479F
:1023E0000134444505F10405E6D102B0BDE8F087AB
:1023F000F7B506792F4D0C237343EF1814463A7A3C
:10240000002A54D1EC504B687B60944647790368AE
:10241000D4B2A74241D843F30733CA78002BAEBFEA
:1024200003F1604303F00F03234C4FEA4212A8BFAD
:1024300003F56143D2B2B4BFE25483F800230368CA
:1024400043F30733002B08DB01225C0903F01F0371
:1024500002FA03F3194A42F8243002684C78D2F8A1
:10246000043564F30103C2F8043502688C78D2F8AD
:10247000083564F30103C2F8083502680978D2F818
:10248000103561F30303C2F810350C2303FB065526
:1024900001232B72002003B0F0BDA40004F5A0744A
:1024A000013243F804C01B590193019BAEE7082099
:1024B000F1E700BF4007002014ED00E000E100E07C
:1024C000036801221A600279034B0C2101FB0233DD
:1024D00002221A72704700BF4007002003680122E1
:1024E0001A610179024B0C2000FB01331A7270470C
:1024F0004007002003680122DA60704773B54FF48B
:10250000803405688C408BB18B0003F5A0730026E6
:10251000EE50EB580193019B0368C3F80443036832
:1025200001F5A87143F8212002B070BDC5F8084339
:10253000F5E7F0B4076840F20116D7F800528E4074
:1025400025EA0605C7F800520468D4F800522B4368
:10255000C4F800329DF81030F0BCFFF7CFBF000088
:10256000024903480422FFF71CBF00BF40070020B8
:1025700000800040024903480422FFF712BF00BF59
:102580004C07002000900040024903480622FFF754
:1025900008BF00BF5807002000B00140002343508F
:1025A00082B043580193019B02B070471FB50123CD
:1025B0008DF80030044BCDE90110D3E900126846D4
:1025C000904705B05DF804FB64070020F8B56B4D3B
:1025D0000679242303FB0653044693F82030002B8E
:1025E00040F0CA800B685F1C19D01F2B4FF0010010
:1025F0008ABF634F4FF0A04703F01F0300FA03F3B5
:10260000C7F808350B681F2B86BF03F01F035C4813
:102610004FF0A04003F5E073032740F823704B68A8
:10262000581C0BD01F2B86BF03F01F0354484FF0DC
:10263000A04003F5E073002740F823702368886901
:10264000C3F824050F7D4B7D20683B43C0F86C35F3
:10265000D1E900702368C3F80C75C3F814050B7D2D
:10266000012B32D18B685F1C0BD01F2B86BF03F070
:102670001F0343484FF0A04003F5E073002740F8E4
:102680002370CB68581C19D01F2B4FF001008ABF54
:102690003B4F4FF0A04703F01F0300FA03F3C7F8C6
:1026A0000835CB681F2B86BF03F01F0334484FF05B
:1026B000A04003F5E073032740F82370D1E9020737
:1026C0002368C3F80875C3F8100524237343E8187A
:1026D00042600869E850002A3FD00A7F20684FF422
:1026E0008871FFF75BFF20684FF49071FFF756FF8A
:1026F00020684FF49271FFF751FF20684FF4A271E8
:10270000FFF74CFF4FF4AC712068FFF747FF2368D9
:102710001C49C3F80413236843F30733002BAEBFEF
:1027200003F1604303F00F0317494FEA4212A8BFB9
:1027300003F56143D2B2B4BFCA5483F800232368BF
:1027400043F30733002B08DB0122590903F01F0371
:1027500002FA03F30D4A42F8213023680822C3F835
:102760000025242303FB06550020C5E906000123AC
:10277000686185F82030F8BD0820FCE76407002078
:10278000000300501003420014ED00E000E100E0FF
:102790000279044B242101FB02335869003818BF29
:1027A000012070476407002001F06043B3F1005F2F
:1027B0002DE9F0470546884692463CD190F80490B2
:1027C000FFF7E6FF0446002837D11E4F242606FBFC
:1027D00009764FF49071C6F814A0C6F808802868EE
:1027E000FFF7DCFE4FF4AC712868FFF7D7FE2B68CB
:1027F0007269B168C3F84415C3F848252B680122F3
:102800009A607368DBB92B68D3F82021D3F858019C
:102810000243F9D068B90122DA602A68D2F8583147
:10282000002BFBD0242303FB097700237B61BDE849
:10283000F0870F20F6E71020F9E71120F7E7204690
:10284000F5E700BF640700207FB5434AD2F8246152
:10285000002E60D010464FF49271FFF79FFE0223C6
:102860008DF80030D2F88034C2F880340393D2F867
:102870003C350293394BDA6801920022C3E9062203
:102880006846D3E9001290473348D0F8443173B119
:102890004FF4A271FFF782FE304B9A693AB10022E1
:1028A000C3E90622D968D0F83C05FFF77FFE2A4825
:1028B000D0F82031ABB14FF49071FFF76FFE0123D8
:1028C000C360264B5A6962B1D0F84C1502910022C0
:1028D00099688DF8002001915A616846D3E9001289
:1028E00090471D48D0F858319BB14FF4AC71FFF7B9
:1028F00055FE1A4B5A6962B1D0F84C15029100226C
:1029000099688DF8002001915A616846D3E9001258
:10291000904704B070BDD2F81031002BB4D04FF402
:1029200088711046FFF73AFE0C4BD2F83C059969C6
:102930008842A9D1DC69D96864B1D2F8005225F087
:102940002005C2F800521A699C61DA60DE61FFF767
:102950002DFE99E79C61FAE7002000406407002003
:1029600010B5124C2378FBB9114B1960037813F0A2
:10297000010F104B1EBFD3F8042542F00102C3F82B
:102980000425D3F8002222F00102C3F80022437884
:10299000094A5B01DBB282F80D334FF40053136038
:1029A00001232370002010BD8520FCE78C07002048
:1029B0008807002000D0004000E100E0074B002223
:1029C000C3F8002182B0D3F800210192019A0122BC
:1029D000C3F804231A6002B0704700BF00D0004063
:1029E000024B0122C3F808235A60704700D0004010
:1029F000074B0022C3F8002182B0D3F800210192D6
:102A0000019AD3F80805034B1B68C0B202B01847FF
:102A100000D00040880700204FF08053024618691C
:102A2000B2FBF0F300FB132068B9084B0221C3F896
:102A30000415C3F80825D3F80024D207FBD50022DB
:102A4000C3F8042570471020704700BF00E0014024
:102A50004FF080531869704770B5064608480D4618
:102A600012F0EEFF064904460246286813F078FA91
:102A7000AC80B368A4B2A34238BFAB80002070BD65
:102A8000D04F020038B50C46054607492068082299
:102A900013F066FA0823237100236371AB68072BD8
:102AA00098BFA380002038BD6000001070B50646B6
:102AB0000C480D4612F0C4FF0A4904460246286835
:102AC00013F04EFA2868084902222044023413F019
:102AD00047FAAC80B368A2B29A4288BFAB800020AC
:102AE00070BD00BFE34F0200EC4F02004FF0102317
:102AF000D3F808321BB102480021FFF7E7B970474D
:102B0000081200104FF0A0430322C3F84C274FF4E3
:102B10000022C3F80C25704708B58379222B08D012
:102B2000552B0CD1C379012B09D1FFF7DFFF002012
:102B300008BDC379222B02D1FFF7E4FFFEE76FF057
:102B400079038B716A23CB71F1E703688B4204D15F
:102B50000260BFF35F8F002070474FF0FF30704777
:102B600012F056BA074A1368032B09D8064B1968A6
:102B7000090219601968084318601368013313606B
:102B8000704700BF9807002094070020002012F033
:102B900039B8000070B54FF0804301220024DA609C
:102BA00090B0C3F818459A60FFF768F90320FFF763
:102BB000EFF8364B4FF47A721B68B3FBF2F3013B2C
:102BC000B3F1807F09D24FF0E022E0215361304B16
:102BD00083F823100723946113612E4C2E4E0FCCE3
:102BE00008AD0FC594E80F0085E80F00002208A982
:102BF0002A48FFF7EBFC2A4B2A4A002506A9304653
:102C0000CDE90635FFF7F4FB33682749D3F81025E3
:102C10000123D2B2009321FA02F230462946FFF78F
:102C200088FC3046FFF74CFC06A9204A2048FFF7F5
:102C3000DFFB204B402283F8272303A88DF80C509C
:102C4000FFF728FB1C4B059305A8FFF745FBFFF793
:102C500049FB4FF08043103CD3F8386416F0010F65
:102C600002D0284612F0D4F9B30702D5022012F0A0
:102C7000CFF9238C1149ADF8103004A8FFF770FE8E
:102C80000F4B00221A6010B070BD00BF080000207A
:102C900000ED00E01C5F020028000020180000206A
:102CA00000000306692D0000007102005D2E000087
:102CB0002000002000E100E0612B0000652B0000F7
:102CC00098070020024A136801331360704700BF61
:102CD0009007002010B50A460C4601460348FFF74E
:102CE00063FD00280CBF2046002010BD1800002006
:102CF00010B5084614461146FFF7ECFF204610BDFC
:102D000001DF704710B503460C461846002101222A
:102D100001DF00B910BD002CF7D14FF0FF30F9E70B
:102D2000BFF35F8F0023036070470000014B1868FA
:102D3000704700BF9007002070B5074D2E6804460D
:102D40002B689B1BA34200D370BD00214FF0FF30C6
:102D500011F016F9F4E700BF900700200020FEF7FD
:102D6000D5BF0020FEF7E6BF70B5224B224D1C6890
:102D70002B68032B0ED8DFE803F002112A351F4B16
:102D80001B783BB10020FEF7F9FF18B101232B603F
:102D90001B4B1C60BDE870400EF048BD0020FEF7E4
:102DA000EDFF174E20B13368E31AB3F5FA7FF1D97E
:102DB0003368E31A142B1AD9B3F5FA7F94BF0120B4
:102DC00002200EF03FFC02232B603460E2E70C4B44
:102DD0001B68E41AB4F5487FDCD900200EF032FC01
:102DE000032305E00020FEF7C9FF0028D2D100230D
:102DF0002B60CFE790070020A0070020A807002045
:102E00009C07002070B5134D06460C462846FFF778
:102E100065FBF4B1104B1E602B68D3F810154FF40E
:102E20007A53C9B2A4FB0343C1F1200003FA00F0B6
:102E3000A1F12002CC40044323FA02F228462243A7
:102E400001230021FFF75AFB2846BDE87040FFF739
:102E500037BB70BD20000020A4070020024B1B6878
:102E600003B11847704700BFA407002010B5FFF753
:102E7000A5FD064C2368032BFCD9FFF7B1FD044ADE
:102E8000002310681360236010BD00BF9807002066
:102E9000940700200020704770B50E461D4614466A
:102EA000FFF7D6FD0449049A06FB00442144284656
:102EB00013F056F8002070BD00000A0010B50C4653
:102EC000FFF7C6FD054B04FB0030FFF7A5FD00280A
:102ED00014BF6FF00400002010BD00BF00000A0006
:102EE0002DE9F843089E16F003080F4614461D46C8
:102EF00005D00D4B0D4A0E482A2112F0C9FADFF811
:102F000038900123C9F80435FFF7A2FD07FB004400
:102F10000848B20820442946FEF7EEFFC9F80485A8
:102F20004046BDE8F88300BFEF4F02003E5F02005D
:102F3000FD4F020000000A0000E0014038B51C4CC3
:102F40004C21204615F0FCFF1A4B63601A4BA3601E
:102F50001A4BE3601A4B236101220423C4E90523C1
:102F6000FFF776FDE061FFF773FD164B164A174930
:102F70009B1AB3FBF0F323628023C4E909131023E7
:102F8000E362134B2363134B6363134BA363032568
:102F900020460EF073FC48B1013DF9D104480EF013
:102FA00067FC03480EF06AFC00B1FEE738BD00BFC5
:102FB000BC080020992E0000E12E0000BD2E00006C
:102FC000952E000000000E0000000A00A0860100FF
:102FD0003C080020BC070020AC0700200F4C08B5BF
:102FE00001232370FFF7D6FD4FF480410020FEF748
:102FF000D7FB08B1FEF766FEFEF72DFBFFF79EFF3D
:103000000AF00CFA0EF07CFA09F0DCF9FEF7E6FBA8
:103010000028FBD120780EF0DFFAF7E7A8070020A0
:1030200038B50C4C0C4D0422FF21204612F074FDE3
:103030000322FF21284612F06FFD01236B7063709D
:10304000022300222B70A37003232270AB70E37065
:1030500038BD00BFBA190020B71900200020704702
:10306000024B187800F00100704700BF08090020EB
:10307000024B1878C0F34000704700BF08090020D9
:10308000024B1878C0F38000704700BF0809002089
:10309000014B00229A70704730000020194B00222B
:1030A00013B59A70044678B1174B18491B780B700A
:1030B00001231748009300220EF01AFC002817DAAB
:1030C0004FF0FF3002B010BD11480EF0BFFC0128D8
:1030D0000346E9D10D490E4822460EF0D5FB0028E3
:1030E000EEDB0C480EF0B2FC002803DB0020E9E721
:1030F000002CF6D008490348032306220FF0C4F839
:10310000C017DFE730000020495F020008090020F7
:1031100025500200330000202F50020010B5014658
:1031200004460423064800220EF0AEFB042806D015
:1031300020460422BDE81040002112F0EDBC10BD75
:103140003650020070B500230B714B718B716FF01C
:103150006F03CB714379322B86B005460C4630D0D5
:1031600012D8202B00F08D80312B1BD0B14A9278E1
:10317000002A61D0212B00F20781002B40F0BB8098
:103180000023A3716D234DE0502B32D0A42BEDD141
:103190008379042B03D1C379002B00F085806FF075
:1031A000790333E08379012BF9D8C279002AF6D16B
:1031B00023B9FFF77BFC002876DA45E0FFF74CFCEB
:1031C000F9E78679012EEAD8C379002BE7D16EB9E9
:1031D0008368032B03D80023A371672322E00868C8
:1031E000FFF79CFF0423237166715DE0FFF74AFC43
:1031F000E1E78379002BD2D18289052AEBD18E4970
:10320000006814F0D0FE20B16FF07F03A3716A2331
:1032100008E088480FF0FBF8002805DD6FF07A031E
:10322000A3716923E3713FE00EF01AFA0028F5D18B
:103230000EF0CAFA002802DA6FF07D03F0E70120F1
:1032400006F0D8FA002801DA0023E9E7012008F0A7
:1032500065FB0028F8DB012005F0F4FA0028F3DB19
:10326000012002F085F8012004F0E2FF0028EBDBEA
:10327000012007F023FD0028E6DB0120FFF70EFF09
:1032800099E78379002B8AD1C679002E87D182896C
:103290006AB9684883783BB90FF0B9F80028D3DBE6
:1032A00000F5C7404030E080002006B070BD0168E6
:1032B00060480DF11703D2B20FF00AF8411CC3D0D9
:1032C000C21C01D1A67188E79DF8173013B96FF0C1
:1032D0007C03A5E70230E7D103F5C7434033E38021
:1032E000E2E7413B032B00F2CA80DFE813F0EE0077
:1032F000040129012E01013B202B3FF641AF01A221
:1033000052F823F0DD330000E7330000F133000012
:10331000F93300000134000081310000093400005D
:10332000113400002334000081310000813100009D
:1033300081310000813100008131000081310000C5
:1033400081310000413400004B3400001B34000088
:103350002B340000813100008131000081310000F8
:103360008131000081310000813100008131000095
:103370008131000081310000813100008131000085
:103380008131000055340000442B1FD83F2BA8D8B2
:10339000302B7FF4F5AEAB79002B7FF400AFEE79E4
:1033A000002E7FF4FCAEAB89042B7FF414AF2348CE
:1033B0000EF04CFB0028BFF631AF01230093AB8920
:1033C00029681E4832460EF093FAF4E6FF2B7FF48C
:1033D000D7AE21462846FFF79FFBECE6214628465C
:1033E00002F070F8E7E62146284602F09BF8E2E694
:1033F000012006F0FFF9DEE6012008F08FFADAE698
:10340000012005F01FFAD6E6012004F011FFD2E6F4
:103410002146284604F0CEFECDE6012007F04EFC02
:10342000C9E6012001F0A4FF3EE721462846FFF748
:1034300015FEC0E630000020395002003650020070
:103440002146284602F084F8B5E62146284602F0D7
:103450008FF8B0E6AB79002B7FF4A1AEEB79002BAF
:103460007FF49DAEAA8929683A48D2B20EF0A0FF37
:10347000431C3FF4E9AE03307FF416AFABE6AB7903
:10348000042B16D0052B1AD0012B7FF488AE324BBB
:10349000E9791A7861F300021A7001232E4900932A
:1034A00000222E480EF024FA03900EF0FFF8039845
:1034B00081E6294BE9791A7861F34102ECE7264B62
:1034C000E9791A7861F38202E6E7AB79002B7FF4A1
:1034D00066AEEE79002E7FF462AEAB68012B7FF60C
:1034E0007AAE0EF0E1FA236818700EF0D1FA236874
:1034F0005870022377E6AB79002B7FF450AEEE795B
:10350000002E7FF44CAEAB68042B7FF664AE124DF8
:1035100022682B78C3F30003137023685E7004F0F5
:103520003FFE236898702B782268C3F34001D17066
:103530002268C3F38003137123685E71062352E689
:103540002146284607F0DCFB35E62146284607F0F1
:10355000EBFB30E630000020080900202550020077
:1035600010B5837BA02B0C4606D00D4B0D4A0E48A0
:1035700040F2462111F08CFFC37BD9060DD413F025
:10358000020308D00FF09AFA0B462060181E18BFED
:103590000120800210BD8089F7E70220FAE700BF12
:1035A0003F500200D25F02005850020010B5837BEA
:1035B000402B06D0054B064A06484FF4F97111F02E
:1035C00067FFBDE8104000230FF066BC9250020078
:1035D000B65F02005850020010B5837B602B06D006
:1035E000054B064A06484FF4F67111F051FFBDE84D
:1035F000104000230FF050BCF45002009A5F02000C
:1036000058500200F52908B506D0064B064A07486F
:1036100040F2871111F03CFF003818BF01201070F4
:10362000002008BDB3500200675F0200585002003E
:1036300010B5837B03F0DF03402B0C4606D00D4B07
:103640000D4A0E484FF4EC7111F022FFC37BD906EE
:103650000DD413F0020308D00FF030FA0B462060AF
:10366000181E18BF0120800210BD8089F7E70220D4
:10367000FAE700BFD05002004A5F02005850020033
:1036800010B5837B802B0C4606D00D4B0D4A0E489F
:1036900040F2392111F0FCFEC37BD9060DD413F0A2
:1036A000020308D00FF00AFA0B462060181E18BF5C
:1036B0000120800210BD8089F7E70220FAE700BFF1
:1036C000155102007E5F0200585002002DE9F041C2
:1036D0008B7BA02B8AB005460C4603D011200AB084
:1036E000BDE8F08106A920460FF0B8FA08B1122013
:1036F000F5E7204601A9FFF733FF04460028F6D17D
:103700003C4FDFF8FC800C26019BA34201D800202F
:10371000E5E79DF82630602BE0D102AA03A906A8B0
:103720000296FFF759FFB0F1004F01D11520D6E7FF
:103730000028DCD106A80FF0FFFB0028D7D13946BE
:1037400003A812F0EDFEC0B99DF82630402BC5D17C
:1037500002AA294606A80293FFF728FFB0F1004FFE
:10376000E4D00028C3D1029B85F8403006A80FF0B2
:10377000E3FB0028BBD10134C6E7414603A812F0A1
:10378000CFFE90B99DF82630602BA7D1402302AA26
:1037900005F1820106A80293FFF71EFF0028A6D1BB
:1037A000029B2B4483F88200E0E7134903A812F040
:1037B000B7FE98B99DF82630602B8FD1402302AA1E
:1037C00005F1410106A80293FFF706FF00288ED1FC
:1037D000029B2B44002283F84120C7E7074903A836
:1037E00012F09EFE0028C1D19DF82630602BBDD07E
:1037F00074E700BF305102003F5102004451020003
:10380000335102002DE9F047837B802B90B00446B2
:103810000F461BD104A90FF021FAF8B9204602A9DE
:10382000FFF72EFF0446C8B9029DDFF8B490DFF819
:10383000B4A0DFF8B4802E46A54203D1AE423AD000
:1038400000200CE09DF81E30A02B01D0112006E0D6
:1038500008AA494604A80FF0B9FB18B1122010B00D
:10386000BDE8F0870CAA514604A80FF0AFFB002872
:10387000F4D19DF82E30602B1FD19DF83E30E3B976
:1038800016490DF1070208A80FF07AFB0028E5D1D0
:103890009DF807307BB103A90CA80FF053FA00285C
:1038A000DCD1039B03F10802012A08D8B54204BF0A
:1038B0003B6026460AE02620D1E71420CFE798F89F
:1038C00000201AB1D8F805209342EFD004A80FF0D9
:1038D00033FB0028C2D10134AEE700BF4E510200D5
:1038E00049510200B7520200A20A002030B5837B82
:1038F000A02B87B005460C4624D1134902AA0FF02D
:1039000065FB10B1122007B030BD9DF81630402B7A
:1039100001D01420F7E7462301935CB90B4902AAB2
:1039200028460FF053FB0028ECD19DF81630602B91
:10393000E9D0EEE701AA214602A8FFF737FE0028EA
:10394000ECD0DFE71120DEE73051020049510200E0
:1039500010B5837B802B86B004461FD101A9FFF7E9
:103960008FFE10B1122006B010BD204602A90FF044
:1039700075F904460028F5D1019B9C4201D3002033
:10398000F1E7002102A8FFF7B1FF0028EBD102A860
:103990000FF0D2FA0028E5D10134EDE71120E2E77B
:1039A0002DE9F0418B7BA02B88B005460C4640F0FA
:1039B000838004A920460FF051F918B1122008B0F5
:1039C000BDE8F081204602A9FFF7CAFD04460028A1
:1039D000F4D13A4E3A4FDFF8EC80029B9C4201D37F
:1039E0000020ECE79DF81E30602B65D103A904A8E8
:1039F0000FF0BEFA0028E1D1039B022B2CD103AAC1
:103A000001A904A8FFF7E8FD0028D7D104A80FF00A
:103A100093FA0028D2D19DF81E30F52B4CD102220A
:103A2000314601A812F004FFC8B99DF81E10BDF878
:103A30001C000DF10302FFF7E5FD0028BED19DF843
:103A400003202B7862F305132B7004A80FF074FA8F
:103A50000028B3D10134C0E7ADF80400D6E7022254
:103A6000394601A812F0E4FE78B99DF81E10BDF8A1
:103A70001C000DF10302FFF7C5FD00289ED19DF843
:103A800003202B7862F38303DEE70222414601A87C
:103A900012F0CEFE0028D8D19DF81E10BDF81C00F3
:103AA0000DF10302FFF7AEFD002887D19DF803203A
:103AB0002B7862F30103C7E7112080E75951020018
:103AC0005C5102005F510200F0B5837BA02B89B0EE
:103AD00004460E4602D0112009B0F0BD04A90FF033
:103AE000BDF808B11220F7E701A92046FFF738FD1D
:103AF00005460028F6D104462027019BAB4204D896
:103B0000042C34BF14200020E6E79DF81E30002B63
:103B1000E1D103A904A80FF015F90028E2D104A807
:103B20000FF00AFA0028DDD1039B0333062B48D897
:103B3000DFE803F03C2D2047134704009DF81E30BA
:103B4000002BC8D103A904A80FF0FCF80028C9D1A4
:103B5000039B193333D0F120BEE79DF81E30002BB4
:103B6000B9D103A904A80FF0EDF80028BAD1039B3E
:103B7000022BEFE79DF81E30002BACD103A904A85F
:103B80000FF0E0F80028ADD1039B012BE2E79DF890
:103B90001E30402B9FD1029702AA314604A8FFF79E
:103BA00005FD00289ED1029B202BD3E79DF81E30F7
:103BB000402B90D1029702AA06F12001EEE70134D2
:103BC000E4B204A80FF0B8F900288BD1013594E7CE
:103BD0002DE9F0418B7BA02B8CB004460D4603D021
:103BE00011200CB0BDE8F08108A928460FF036F886
:103BF00008B11220F5E7284601A9FFF7B1FC0546F8
:103C00000028F6D1484FDFF82C810D26019BAB42EE
:103C100001D80020E5E79DF82E30602BE0D102AA04
:103C200004A908A80296FFF7D7FCB0F1004F78D09E
:103C30000028DED108A80FF07FF90028D9D1394635
:103C400004A812F06DFCC0B99DF82E30002BC7D12E
:103C500003A908A80FF076F80028CAD1039B5A1EC2
:103C6000022A01D92C20BCE784F86F3108A80FF094
:103C700063F90028BDD10135C8E7414604A812F018
:103C80004FFC18BB9DF82E30402BA9D194F89031F1
:103C900043F0010384F89031202302AA04F5B8719F
:103CA0000DEB03000293FFF781FCB0F1004F07D149
:103CB00094F89031212262F3470384F89031D5E7DC
:103CC000002896D194F89031029AF4E7174904A895
:103CD00012F026FC80B99DF82E10F52980D1BDF890
:103CE0002C0004F5B772FFF78DFC002881D194F801
:103CF0006E31002BBAD1B5E70D4904A812F010FCC3
:103D00000028B3D19DF82E30F52B7FF469AFBDF8B4
:103D10002C0004F26D12F521FFF774FC0028A5D0E9
:103D200067E715205DE700BF62510200775102008E
:103D3000845102006E5102002DE9F04F8B7BA02BC5
:103D400093B004460D4601D0112005E00AA928468B
:103D50000EF084FF18B1122013B0BDE8F08F01A956
:103D60002846FFF7FDFB06460028F4D1DFF80C9249
:103D7000DFF80CA24FF00D08019BB34201D80020E0
:103D8000EAE79DF83630602BDED102AA06A90AA820
:103D9000CDF80880FFF720FCB0F1004F00F0E9807B
:103DA0000028D8D10AA80FF0C7F80028D3D1494677
:103DB00006A812F0B5FB002840F0AE80012384F87D
:103DC00033319DF83630A02BBED10EA90AA80EF0D3
:103DD00045FF0028BFD104A90AA8FFF7C1FB05468B
:103DE0000028B8D107464FF0200B049BAB420ED8F9
:103DF000072F40F08F8094F83331012B6ED194F867
:103E00001131402B76D0202B74D00320A4E79DF8ED
:103E10004630002B98D105A90EA80EF093FF00287C
:103E200099D10EA80FF088F8002894D1059B013B8A
:103E3000032B0CD8DFE803F002132C4204F18101BC
:103E40000EA8FFF741FE002885D147F001070EA814
:103E50000FF072F800287FF47EAF0135C5E79DF8BA
:103E60004630402B7FF470AF502302AA04F1C10109
:103E70000EA80293FFF79AFBB0F1004FC5D00028BF
:103E80007FF469AF029B84F8113147F00207DEE747
:103E90009DF84630402B7FF457AF02AA04F5897194
:103EA0000EA8CDF808B0FFF781FB00287FF453AFD0
:103EB000029B84F8323147F00407C8E79DF846308A
:103EC000002B7FF441AF03A90EA80EF03BFF0028A2
:103ED0007FF441AF039B84F83331B8E7022B0DD157
:103EE00094F81131502B01D0302B8ED194F832310F
:103EF000202B02E094F83231102B86D1236843F452
:103F0000805323600AA80FF017F800287FF423AF2E
:103F1000013631E714201FE7514606A812F000FBD6
:103F200068B99DF83610F5297FF40EAFBDF834005E
:103F300004F23512FFF766FB0028E3D00BE70E49C9
:103F400006A812F0EDFA0028DCD19DF83610F5290C
:103F50007FF4FAAEBDF8340004F59A72FFF752FB15
:103F600000287FF4F8AE94F83431002BCAD12C200D
:103F7000F2E61520F0E600BF7751020084510200FE
:103F80006E5102002DE9F043002313608B7BA02BC0
:103F900089B004460E46174603D0112009B0BDE88B
:103FA000F08304A930460EF059FE08B11220F5E75F
:103FB00001A93046FFF7D4FA05460028F6D104F1EE
:103FC000300804F17609019BAB4205D87268059B65
:103FD0009B1A3B600020E1E79DF81E30002BDCD1EE
:103FE00003A904A80EF0AEFE0028DFD104A80EF04D
:103FF000A3FF0028DAD1039B022B23D0032B2BD065
:10400000012B18D19DF81E30402BC6D102A904A85F
:10401000FFF70EFB0028C9D1029B202BC6D102AAB4
:1040200004F1100104A8FFF7C1FA0028BED12368EB
:1040300043F00203236004A80EF07EFF0028B5D1F0
:104040000135C0E7414604A8FFF750FC0028ADD178
:10405000236843F40043EDE704A94846FFF736FB25
:104060000028A3D1236843F00403E3E72DE9F04FD0
:104070000C46D7B00746164600214FF4CA722046B8
:10408000039311F049FD94F8441121F03F0141F0F0
:104090002A010AAD84F844113B4603990095002299
:1040A00030460EF08BFD002859D19DF83630A02BFC
:1040B0004ED10EA928460EF0D1FD00284FD128463A
:1040C00004A9FFF74DFA0546002848D1049BAB42EE
:1040D00007D8236803F00F030F2B14BF1420002010
:1040E0003EE09DF84630002B32D105A90EA80EF017
:1040F00029FE002833D10EA80EF01EFF78BB059BC9
:10410000013B092B00F2DF80DFE813F00A001E00FC
:10411000AF00BB00C700E500F000FC001C0132014D
:104120009DF84630402B13D1202303AA211D0EA851
:104130000393FFF73BFA90B9039B202B0FD1236821
:1041400043F001032360BEE09DF84630A02B01D070
:10415000112005E012A90EA80EF080FD18B1122062
:1041600057B0BDE8F08F08A90EA8FFF7F9F90028AD
:10417000F5D180464FF00409089B984503D3236886
:1041800043F00203DEE79DF85630602BE0D109AA28
:1041900007A912A8CDF82490FFF71EFAB0F1004F3E
:1041A00000F0EE800028DAD112A80EF0C5FE00283B
:1041B000D5D19DF85630602BCAD1724907A812F0AC
:1041C000AFF9F0B90DF1580AFE2309AA514612A819
:1041D0000993FFF701FA0028C1D1099F202F0AF89F
:1041E000070004F1240B3A4613D85146584611F003
:1041F000B7FE3E460999666404F1480216A815F018
:104200001FF812A80EF098FE0028A8D108F10108A6
:10421000B2E73A21504611F053FE20B3A0EB0A005A
:10422000461C202E28BF202632465146584611F003
:1042300097FEC6F12003022BDCD9E2230BF80630EF
:104240000BEB060380225A70A7F11D01A6229A707B
:10425000F01C314416ABC6F11D021944584411F04C
:104260007FFE2026C6E70026E7E70EA904F16800D6
:10427000FFF72CFA00287FF473AF236843F00403A0
:1042800060E704F596710EA8FFF7BCFA00287FF4EA
:1042900067AF236843F0080354E70EA8FFF758FB05
:1042A00000287FF45DAF04F598710EA80EF0D6FCDF
:1042B00000287FF454AF04F5A0710EA8FFF7E0F9D1
:1042C00000287FF44CAF0EA80EF036FE00287FF4D5
:1042D00046AF0135FAE60EA92046FFF779FC002823
:1042E0007FF43EAF236843F010032BE70EA904F5DB
:1042F000A270FFF755FB00287FF432AF236843F02C
:1043000020031FE79DF84630402B7FF421AF04F5D2
:10431000B47631460EA8FFF78BF900287FF41FAF63
:10432000D4F86831202B27D81BB9236843F0400309
:1043300008E7324604F245110EA8FFF737F90028C6
:10434000F3D00CE79DF84630002B7FF401AF06A9AF
:104350000EA80EF0F7FC00287FF401AF069B5A1E52
:10436000012A0BD884F86C31236843F08003E9E616
:10437000236843F40053E5E63320F1E60220EFE63C
:104380001520EDE630510200F0B50C46D1B00746DD
:10439000164600214FF49C722046039311F0BCFB9B
:1043A00094F8581021F03F0141F02A0108AD84F83B
:1043B00058103B4603990095002230460EF0FEFB54
:1043C00010B1122051B0F0BDAB7BA02B01D0112059
:1043D000F8E70CA928460EF041FC0028F1D1284648
:1043E00005A9FFF7BDF805460028EAD1059BAB42B9
:1043F00007D8236803F00303032B14BF1420002005
:10440000E0E79DF83E30002BE1D106A90CA80EF0A4
:1044100099FC0028D5D10CA80EF08EFD0028D0D133
:10442000069B013B062B46D8DFE803F0041D324C07
:10443000535F7E009DF83E30602BC8D1FE2303AA57
:1044400010A90CA80393FFF7C7F80028B9D18DF87D
:104450003D010399221D10A814F0F2FE236843F0D9
:104460000203236027E09DF83E30402BAFD120238C
:1044700003AA04F124010CA80393FFF797F800287E
:104480009FD1039B202B9CD1236843F00103E8E7D5
:104490000CA8FFF75DFA002894D104F144010CA8A0
:1044A0000EF0DCFB00288CD104F154010CA8FFF7BE
:1044B000E7F8002885D10CA80EF03EFD002880D139
:1044C000013593E70CA92046FFF736FC0028F2D00F
:1044D00078E70CA904F15800FFF762FA00287FF48E
:1044E00071AF236843F02003BBE79DF83E30402BBB
:1044F0007FF46DAF04F17C0631460CA8FFF798F805
:1045000000287FF45EAFE36F202B23D81BB923680C
:1045100043F04003A5E7324604F159010CA8FFF728
:1045200045F80028F3D04CE79DF83E30002B7FF48F
:104530004EAF07A90CA80EF005FC00287FF441AF90
:10454000079B5A1E012A07D884F88030236843F05D
:10455000800386E7332035E7022033E7F0B50C46C9
:10456000CFB0074616460021F822204606AD039339
:1045700011F0D2FA039900953B46002230460EF026
:104580001DFB10B112204FB0F0BDAB7BA02B01D0B2
:104590001120F8E70AA928460EF060FB0028F1D1A7
:1045A000284604A9FEF7DCFF05460028EAD1049B53
:1045B000AB420DD82368DA0540F120812279022A26
:1045C00040F0EF8013F0800F0CBF14200020DAE7DA
:1045D0009DF83630002BDBD105A90AA80EF0B2FBFE
:1045E0000028CFD10AA80EF0A7FC0028CAD1059B4D
:1045F000013B092B1AD8DFE803F00520303A567B3F
:104600001919A0B99DF83630002BC1D105A90AA807
:104610000EF098FB0028B5D1059B5A1E012A00F226
:10462000E7806371236843F0800323600AA80EF0DB
:1046300083FC0028A6D10135B9E79DF83630002B60
:10464000A6D105A90AA80EF07DFB00289AD1059BEA
:104650002371236843F48073E7E7A11D0AA8FFF7DD
:1046600033FA00288FD1236843F40073DDE79DF807
:104670003630402B8CD103A90AA8FEF7D9FF0028B9
:1046800080D1039B013B1F2B00F2B48003AA04F1ED
:1046900046010AA8FEF78AFF00287FF473AF23685B
:1046A00043F04003C1E79DF83630402B7FF470AFF4
:1046B00003A90AA8FEF7BCFF00287FF463AF637963
:1046C000012B10D1039B402B7FF45CAF03AA04F1B4
:1046D00066010AA8FEF76AFF00287FF453AF23683B
:1046E00043F48063A1E7022BF0D1039B502BEBE74F
:1046F0009DF83630402B7FF44BAF03A90AA8FEF794
:1047000097FF00287FF43EAF6379012B10D1039B04
:10471000102B7FF437AF03AA04F1B6010AA8FEF705
:1047200045FF00287FF42EAF236843F400637CE745
:10473000022BF0D1039B202BEBE79DF83630002BAA
:104740007FF426AF05A90AA80EF0FCFA00287FF432
:1047500019AF9DF8143084F8D630002B48D013F0F0
:10476000280F49D1236843F480435EE79DF8363033
:10477000602B7FF40DAF0EAEFE2303AA31460AA8CC
:104780000393FEF729FF00287FF4FCAE039904F1A0
:10479000D7027054304614F053FD236843F00203EF
:1047A00043E7032A07D103F4D863B3F5D86F14BFE6
:1047B00014200020E7E6042A04D103F46C63B3F567
:1047C0006C6FF4E7052A0CD103F42862B2F5286F68
:1047D00014D144F20202134214BF01200020400011
:1047E000D1E6092A0CD103F49543B3F5954FDEE7E2
:1047F0000220C8E63320C6E64020C4E61420C2E604
:104800000020C0E6F0B50C4691B0074616460021E0
:104810004FF4AE72204608AD039311F07DF9039971
:1048200000953B46002230460EF0C8F910B1122028
:1048300011B0F0BD9DF82E30A02B01D01120F7E76C
:104840000CA928460EF00AFA0028F0D1284605A93E
:10485000FEF786FE05460028E9D104F59D76059B06
:10486000AB4219D82368DE0540F192802279072AED
:1048700000F29080D621D140CD077AD55C0640F178
:104880008580190640F18480042A6DD113F0020F4F
:104890000CBF14200020CBE79DF83E30002BCDD17B
:1048A00006A90CA80EF04EFA0028C0D10CA80EF0F4
:1048B00043FB0028BBD1069B013B032B1ED8DFE83E
:1048C00003F0021324389DF83E30002BB6D107A91F
:1048D0000CA80EF037FA0028A9D1079B2371236892
:1048E00043F48073236009E00D9BA36004F10C0284
:1048F0000CA92046FFF746FB002898D10CA80EF023
:104900001BFB002893D10135A9E79DF83E30002B11
:1049100094D107A90CA80EF015FA002887D1079B9F
:104920005A1E012A2ED884F83931236843F08003B7
:10493000D8E79DF83E30402B80D103A90CA8FEF7A4
:1049400077FE00287FF473AF039B013B1F2B1BD81E
:1049500003AA31460CA8FEF729FE00287FF467AFB2
:10496000236843F04003BDE7062A02D113F4004F49
:104970008EE7072A0ED148F204029A4314BF14208E
:10498000002055E7022053E7332051E736204FE758
:1049900014204DE700204BE7F0B50C4691B00746D8
:1049A000164600213822204608AD039311F0B4F8D2
:1049B000039900953B46002230460EF0FFF810B1F7
:1049C000122011B0F0BD9DF82E30A02B01D0112087
:1049D000F7E70CA928460EF041F90028F0D1284647
:1049E00005A9FEF7BDFD05460028E9D1059BAB42B0
:1049F00031D82368590340F1CB8013F4403F00F0D5
:104A0000C780DA030AD5794A1A40002A40F0C080EC
:104A1000A18840F2D442914200F2E48013F40030C5
:104A2000CFD0E16840F2D442914200F2DB8003F43F
:104A30000020238A002B40F0CF80002800F0A880BF
:104A4000608AB0F5805F00F2CF8010288CBF002014
:104A500001204000B5E79DF83E30002BB7D106A9F4
:104A60000CA80EF06FF90028AAD10CA80EF064FA79
:104A70000028A5D1069B013B052B1DD8DFE803F0DC
:104A80000324405C8F789DF83E30002B9FD107A90E
:104A90000CA80EF057F9002892D1079B002B96DB4B
:104AA000B3F5803FA4BF4FF6FF730793079BA38026
:104AB000236843F4803323600CA80EF03DFA0028ED
:104AC0007FF47EAF013591E79DF83E30402B7FF4B7
:104AD0007EAF04F10C010CA8FEF7AAFD00287FF4BC
:104AE0006FAF0D9B5A1CA260E268172A04D9FF2AF7
:104AF00094BF02330333A360236843F40033DAE73F
:104B00009DF83E30002B7FF462AF07A90CA80EF091
:104B100019F900287FF454AF079B002BFFF657AF1D
:104B2000B3F5803FA4BF4FF6FF730793079B238223
:104B3000236843F48023BEE79DF83E30002B7FF4CA
:104B400046AF07A90CA80EF0FDF800287FF438AF97
:104B5000079B002BFFF63BAFB3F5803FA4BF4FF69A
:104B6000FF730793079B6382236843F40023A2E744
:104B70009DF83E30002B7FF42AAF07A90CA80EF059
:104B8000E1F800287FF41CAF079B5A1E012A01D9C7
:104B9000022016E72375236843F080038BE79DF816
:104BA0003E30402B7FF413AF03A90CA8FEF740FD65
:104BB00000287FF405AF039B013B1F2B10D803AAED
:104BC00004F115010CA8FEF7F1FC00287FF4F8AE03
:104BD000236843F040036EE7003818BF012038E730
:104BE0003320EEE60320ECE61820EAE6C0000800D9
:104BF00070B596B009AE322231460546002301A8B1
:104C00000DF0FDFC042205A90DEB02000DF039FDAD
:104C100018B11224204616B070BD0122002305A849
:104C20000DF000FD0028F4D10122002305A80DF0AD
:104C3000F9FC0028EDD10322002305A80DF0F2FCB9
:104C40000028E6D16FF007024FF0FF3305A80DF002
:104C5000E9FC0028DDD14FF0FF324FF0FF3305A80B
:104C60000DF0E0FC0028D4D10622002305A80DF0A9
:104C7000D9FC0028CDD16FF001024FF0FF3305A819
:104C80000DF0D0FC0028C4D12022294605A80DF043
:104C9000EBFC0028BDD105A901A80DF003FD0028FB
:104CA000B7D1019CA41B22463146284611F058F981
:104CB000B0E7F0B59DB008AE05460F4668463146F0
:104CC0001446002350220DF09AFC052204A96846E0
:104CD0000DF0D7FC18B1122420461DB0F0BD012202
:104CE000002304A80DF09EFC0028F4D1022200232A
:104CF00004A80DF097FC0028EDD10322002304A89E
:104D00000DF090FC0028E6D13A46FB1704A80DF000
:104D100089FC0028DFD14FF0FF324FF0FF3304A8A9
:104D20000DF080FC0028D6D12246E31704A80DF030
:104D300079FC0028CFD16FF001024FF0FF3304A8B7
:104D40000DF070FC0028C6D12022294604A80DF0E1
:104D50008BFC0028BFD16FF002024FF0FF3304A894
:104D60000DF060FC0028B6D12022A91804A80DF08F
:104D70007BFC0028AFD104A968460DF093FC002805
:104D8000A9D1009CA41B22463146284611F0E8F820
:104D9000A2E738B5054608460C4610F051FE2146FC
:104DA00002462846BDE838400DF063BC2DE9F041CD
:104DB000E6B0134605460A4602A828A9FFF7CEFB2F
:104DC0000446D0B9102108A814F0BAF89DF8A43010
:104DD000013B082B11D8DFE813F009002B0052002B
:104DE0009E0032011000100010003201012204A9BF
:104DF00028460DF046FC20B11224204666B0BDE8DE
:104E0000F0810322002304A80DF00CFC0028F3D14C
:104E100002F092FF0246C31704A80DF003FC00281D
:104E2000EAD104A928460DF03DFC0028E5D0E3E7CF
:104E3000012204A928460DF024FC0028DCD101221F
:104E4000002304A80DF0EEFB02460028D4D10CA9E3
:104E500004A80DF016FC0028CED10C9E013E304671
:104E600002F090FC01226FF018013046FFF721FF9D
:104E70000CA9064404A80C960DF014FCCFE702F030
:104E800015FF08B13324B8E79DF8A5100DF1A60071
:104E900002F082FC002801DDC4B2AEE79DF8A53027
:104EA0000193012B0DF1E60300930DF5837214BFFE
:104EB0005023402320210DF1A60002F02DFD0028F3
:104EC000E0D09DF8A5300093012B0DF5837314BF3E
:104ED0005022402219460DF1A60002F0E7FC08B16D
:104EE000F1248AE70DF5A3733F2113F8012D62B178
:104EF000CB1E3B2B0DD80131C9B20DF5837002F0EA
:104F0000E5FE0028BFF679AFEAE7013911F0FF01AD
:104F1000EBD1372471E702F0C9FE002800F092803F
:104F200002F00AFF061EDBDB01D1322465E7864D65
:104F30002B780BB9342460E79DF8A5100DF1A6007D
:104F400002F02AFC0028A7DC9DF8A530012B0DF10A
:104F5000E60742D140220DF583710CA811F000F84C
:104F600010220DF5AB711CA810F0FAFF9DF8A530CA
:104F7000CDE9007350230CAA20210DF1A60002F008
:104F8000CBFC00283FF47EAF013EF0B202F0E6FE1B
:104F90000028A5DB9DF8A5300093012B0DF5AB7320
:104FA00014BF2022102219460DF1A60002F07EFC4B
:104FB000002895D10DF5AB7002F0A8FE00288FDB1C
:104FC0001DD002F0C5FB002EAFD02B78013BDBB229
:104FD0002B70002BAED031240FE750220DF58371DA
:104FE0000CA810F0BDFF20220DF5AB7120A810F029
:104FF000B7FF9DF8A530CDE900737023BBE703230D
:105000002B709DF8A5300093012B0DF5837314BF11
:105010005022402219460DF1A60002F047FC00285C
:105020007FF45EAF0DF5A3733F2113F8012D002A25
:105030007FF45EAF013911F0FF01F6D169E702F0AC
:1050400035FE08B93524D8E602F076FE061EFFF6D6
:1050500047AF3FF46AAF3C4F3B78002B3FF46AAF59
:105060009DF8A5100DF1A60002F096FB00283FF771
:1050700013AF013EF0B202F071FE0028FFF630AF30
:105080009DF8A5300093012B0DF5AB7314BF2022C2
:10509000102219460DF1A60002F008FC00287FF44A
:1050A0001FAF0DF5AB7002F031FEB0F10008FFF656
:1050B00017AF07D0002E3FF438AF3B78013BDBB28F
:1050C0003B7086E7032308203B7002F047FE002870
:1050D000FFF606AF02F042FB404602F0BBFA9DF835
:1050E000A430052B24D1032002F052FC9DF8A5200A
:1050F0000CA90DF1A60002F0CDFB012204A928465F
:105100000DF0BFFA00287FF477AE0222002304A836
:105110000DF088FA00287FF46FAE9DF8A530012BC2
:1051200014BF302220220CA904A80DF09DFA76E6C7
:105130009DF8760102F02CFC289B9B07D6D50DF23A
:10514000771002F051FCD1E7AC0A00202DE9F041C4
:10515000D2B0134605460A4602A804A9FFF71CFC74
:10516000044640B9049BD9034DD57C480CF06EFC35
:10517000031E04DAF124204652B0BDE8F081BDF8E8
:1051800020209A4253DCBDF8141011449942C4BF48
:105190009B1AADF814300CF063FA10B901200CF032
:1051A00057FA012212A928460DF06BFA08B1122411
:1051B000E1E70023012212A80DF034FA034600288B
:1051C000F5D1BDF81420129E12A80DF01FFA002888
:1051D000EDD13378614843F040033370BDF81430AB
:1051E000BDF8202012990CF04FFB0028C2DB129B67
:1051F000BDF8142012A91344284612930DF052FA58
:105200000028B8D0D3E7BDF82030554D8BB9554BA9
:10521000BDF822201A80288002F048FD70B9079A54
:10522000BDF820304F4E13443288934237D90224C0
:10523000A1E72A889A42EFD004249CE7049B5A06EF
:1052400040F183801B0640F182802022FF2112A8BA
:1052500010F062FC0C23ADF86830BDF82030ADF8DA
:105260006A30DDE9060100230DF16E02ADF86C3005
:1052700013F0E6FF3C4B1B78002B6AD09DF82430DE
:105280000DF12502462112A802F060FB08B9332473
:1052900071E7102002F084FB0028C0D1F7E70CF082
:1052A000DFF910B901200CF0D3F9BDF820202F4808
:1052B000B2FA82F35B090093DDE906130CF018FBE8
:1052C0000028FFF657AF2A88079B134432889BB209
:1052D00093422B807FF44FAF103B338013F08CFF51
:1052E000DFF8888000273588BD4219DC12A813F04A
:1052F00099FF1E4810233A4616A90CF0C5FA00285B
:10530000FFF638AF102216A912A812F04CFE10BBFF
:10531000124916480CF0DAFB0028BFF62CAF29E73B
:10532000ED1BB5F5807FA8BF4FF480752B463A463C
:1053300012A940460CF0A8FA0028FFF61BAFA9B24C
:1053400012A813F067FF2F44CDE7362413E7142487
:1053500011E734240FE73D240DE700BF9051020010
:105360000A0900200C090020AC0A00209851020014
:1053700070B54C4B03221A704B4B90B00446FF2281
:105380001A7002F0F7F98CB948480CF05FFB00285E
:105390000CDB474A4748092306210CF03BFB002859
:1053A00002DB002010B070BDF120FBE720220021BD
:1053B0000DEB020010F0B0FB012500233E480095E4
:1053C0001A4619460CF094FA0028EDDB3A480323FC
:1053D00008AA00210CF02CFB0028E5DB002337484D
:1053E00000951A4619460CF083FA0028DCDB0024ED
:1053F000304800942346224621460CF079FAA04218
:10540000D2DB2C48042308AA29460CF011FBA04249
:10541000CADB28482346224602210CF009FBA042A1
:10542000C2DB20210DEB010013F092FD2023214867
:105430000DEB030204210CF0FBFAA042B4DB2021A7
:105440000DEB010013F084FD20231A480DEB03023D
:1054500005210CF0EDFAA042A6DB194B03AA03F1DB
:105460001006154618685968144603C40833B34239
:105470002246F7D11B7823701122294608A810F084
:105480006FFD0123009309481123002208A90CF0A5
:105490002FFA002888DB20210DEB010013F050FDCE
:1054A0007FE700BFAC0A0020AB0A00209051020049
:1054B000A20A0020A1510200AB510200B351020028
:1054C000FC5F020070B58389202B05464FF0000475
:1054D00004D067238C71CB71204670BD0F4A1048F1
:1054E00014706FF02F0151714FF0FF31092391714A
:1054F000D1711172062153709470D47014710CF034
:1055000097FA002807DBAB892A6805482146BDE8E1
:1055100070400CF08DBAF120DFE700BFA20A002036
:10552000A151020007B58389B3F5906F06D9002019
:1055300067238871CB7103B05DF804FB01220092F0
:105540000168024800220CF0D3F9F4E7A1510200EF
:1055500010B509230A6805480C4606210CF05AFAD2
:105560000028A4BFA080002010BD00BFA1510200F0
:1055700070B58689092E054605D0002467238C71F5
:10558000CB71204670BD02680548334606210CF0F9
:105590004FFA296804463246024810F0E1FCF0E771
:1055A000A1510200A20A00202DE9F041CEB04C48E2
:1055B000032302AA00210CF02DFA0028C0F28C80EF
:1055C0009DF80A309A0703D100204EB0BDE8F08163
:1055D00043480CF03BFA9DF809204FF4967402FB07
:1055E0000442904219DB3E482346A2F5967203A975
:1055F0000CF04AF900286FDB9DF815316BB90122D8
:105600008DF815219DF80920009335482346624303
:1056100003A90CF06DF900285EDB32480CF016FA95
:10562000002859DBDFF8BC8000264C27B0FBF7F4DC
:10563000A64218DB9DF80A3029489B0742BF9DF817
:10564000083003F1FF338DF808309DF80A3023F05D
:1056500003038DF80A3002AA032300210CF0E8F9B5
:105660000028B1DA38E007FB06F54C232A4603A9E7
:1056700040460CF009F900282EDB9DF80930DDE9E1
:1056800014C1C3F1200EA3F120002CFA03F201FA99
:105690000EFE21FA00F042EA0E02024312F0010F60
:1056A000A3F12000C3F1200218D0012424FA02F251
:1056B00004FA00F010439C4021EA00012CEA0404A3
:1056C0000023CDE91441009306484C232A4603A940
:1056D0000CF00EF90028ADDAF12076E70136A7E7E5
:1056E000AB510200B35102002DE9F047ADF5747DD6
:1056F000134606460A4603A89DA9FFF783F8044609
:1057000020B9FFF751FF002805DDC4B220460DF592
:10571000747DBDE8F0879DF87832072B44D8D622F7
:10572000DA40D20740D5AB4AAB4813702146032379
:1057300052AA0CF06FF90028C0F2C383A09A9DF81A
:1057400078329DF848518DF84831531CB3F5967F57
:1057500000F21D8422B19F990DF2491010F000FC57
:105760009E4B1B78002B00F01584A0999DF8AD335B
:105770000DF2AE32013152A802F0E8F808B9332434
:10578000C4E7042002F00CF90028F8D09DF8783224
:10579000013B062BBAD8DFE813F009003300B30051
:1057A0002D01CD02DC0299032546EFE702F002F954
:1057B0000028E4D1022205A930460CF062FF08B1AE
:1057C0001224A3E70023012205A80CF02BFF0346B7
:1057D0000028F5D12A4605A80CF024FF0028EFD1B7
:1057E0000222002305A80CF01DFF0028E8D1C5F116
:1057F0004002D31705A80CF015FF0028E0D150E2B5
:1058000002F0D8F80028BAD1002D00F0FB807448CF
:10581000744D0CF01BF94C2390FBF3F028600BF057
:105820001FFF10B901200BF013FF2D68DFF8B091B6
:10583000DFF8B4A1013D00274FF04C08002D4CDAF1
:10584000694B67481A680DA94C2308FB02F20CF05B
:105850001BF80028C0F23583032205A930460CF05E
:1058600010FF0028ACD10322002305A80CF0DAFEBB
:105870000028A5D1012209A905A80CF002FF0028E3
:105880009ED15A4909A8FFF784FA002898D11D9A99
:1058900015A909A80CF0EDFE002891D109A905A8C9
:1058A0000CF000FF00288BD10422002305A80CF087
:1058B000B9FE002884D120220DA905A80CF0D4FE41
:1058C00000287FF47DAF0522002305A80CF0AAFE76
:1058D00000287FF475AF3A468BE74C2308FB05F2AE
:1058E0000DA948460BF0D0FF0028C0F2EA82DDE99E
:1058F0001E3213431CBFCAF800500137013D9DE71B
:105900003B4B1B780A2B04D1324A1378023B012B04
:1059100004D9304B00221A703024F7E6324FDFF8FA
:10592000C4803D68DFF8B8A00323137001354FF041
:105930004C09D8F80030AB420EDD4C2309FB05F2D0
:105940000DA950460BF0A0FF0028C0F2BA82DDE995
:105950001E3213433CD03D60022205A930460CF0B4
:1059600090FE00287FF42CAF0322002305A80CF042
:1059700059FE00287FF424AF012209A905A80CF0E4
:1059800080FE00287FF41CAF184909A8FFF701FA30
:1059900000287FF415AF1D9A15A909A80CF069FE1F
:1059A00000287FF40DAF09A905A80CF07BFE0028A4
:1059B0007FF406AF0422002305A80CF033FE002874
:1059C0007FF4FEAE20220DA905A80CF04DFE14E7D1
:1059D0000135AEE720090020AB510200AC0A0020DF
:1059E000B35102001C0900201809002030510200A8
:1059F000AB0A0020A1A801F0E5FF074600283FF40C
:105A0000BEAE0DB92E2481E6B648B74D0CF01EF897
:105A10004C2390FBF3F028600BF022FE10B901201C
:105A20000BF016FEDFF8C882DFF8B89200222B6870
:105A3000C8F80020934217DD4C235A430DA948466D
:105A40000BF022FF0028C0F23C82DDE91E32134336
:105A500003D1D8F800200132E9E72022A1A90DA83E
:105A600012F0A1FA0028F4D1D8F800202B689A424D
:105A7000C8D0DDE91E129D4BC3E900129B48D0E956
:105A800000C54FF000086346AE4641464FF0FF3276
:105A900013F0010F07D008F101085FFA88F8B2F19E
:105AA000FF3F08BF0A4601315B08402943EACE7335
:105AB0004FEA5E0EECD1511C11D00121A2F120035E
:105AC000C2F1200E01FA03F321FA0EFE43EA0E039F
:105AD00091402CEA010125EA0305C0E90015844B39
:105AE00084481A604FF496735A4352A90BF0CCFEC7
:105AF0000028C0F2E6819DF852323A1D1A4405A9E9
:105B000030460CF0BEFD00287FF45AAE062200237A
:105B100005A80CF087FD00287FF452AE032209A9E6
:105B200005A80CF0AEFD00287FF44AAE724909A822
:105B3000FFF72FF900287FF443AE9DF8CE210DF535
:105B4000C77109A80CF090FD00287FF439AE6B49AD
:105B500009A8FFF71EF900287FF432AE0DF2CF112D
:105B600009A8FFF716F900287FF42AAE644909A8AE
:105B7000FFF70FF900287FF423AE84A909A8FFF7E7
:105B800008F900287FF41CAE09A905A80CF08AFDCD
:105B900000287FF415AE0722002305A80CF042FD73
:105BA00000287FF40DAE022209A905A80CF069FDBA
:105BB00000287FF405AE504909A8FFF7EAF800284D
:105BC0007FF4FEAD462252A909A80CF04DFD002835
:105BD0007FF4F6AD4B4909A8FFF7DBF800287FF406
:105BE000EFAD494909A8FFF7D4F800287FF4E8ADE4
:105BF00009A905A80CF056FD00287FF4E1AD0822A4
:105C0000002305A80CF00EFD024600287FF4D8AD55
:105C100009A905A80CF035FD00287FF4D1AD20A915
:105C200052A801F083FF002840F04B81DDF88A0183
:105C300001F0E4FE20A9814613F02EF80028C0F2FE
:105C4000A381099D314B013D53F8292031A92846F4
:105C500010F086F9DDF88A11CB1D2AD101222846E1
:105C6000FFF727F82844099009A905A80CF01AFDA8
:105C700000287FF4A5AD27BB00230A2205A80CF05D
:105C8000D1FC034600287FF49BAD9DF8692105A84F
:105C90000CF0C8FC00287FF493AD9DF85232002B25
:105CA00036D105A930460CF0FDFC00283FF42EAD9E
:105CB00086E50831D8D12846FEF79AFF05440995B4
:105CC000D2E70023092205A80CF0ACFC034600280B
:105CD0007FF476AD424605A80CF0A4FC0028CBD09A
:105CE0006EE500BFB35102001C090020100900201E
:105CF00018090020AB510200305102003F51020050
:105D000033510200495102004E510200506A020014
:105D100095A956A802F070F800287FF451AD0B2227
:105D2000002305A80CF07EFC00287FF449AD20225A
:105D300095A949E6994B1B780A2B7FF4EAAD984A5E
:105D40001378043B012B3FF6E4AD052313700027C5
:105D500094E60DF2C62001F035FE00283FF40FADA9
:105D6000002D3FF44FAE8F480BF070FE0028C0F2BC
:105D7000A8808D4EDFF82C8200224FF49673B0FB82
:105D8000F3F5EFB29742326016DD4FF496735A4343
:105D900052A940460BF078FD0028C0F292809DF891
:105DA000513213B132680132EBE74622A9A952A859
:105DB00012F0F9F80028F5D133689F423FF422AE83
:105DC0007848032320AA00210BF024FE002878DB6A
:105DD00033688DF881309DF88230724843F00203B9
:105DE0008DF8823020AA032300210BF021FE002829
:105DF00067DB32686B48002300934FF496730127EA
:105E00005A4352A98DF851720BF072FD002858DBED
:105E100066480BF01BFE051E53DB4C23B5FBF3F568
:105E20000BF01EFC10B938460BF012FCDFF87CA119
:105E30004FF00008EDB24FF04C0945452DDD09FB50
:105E400008F74C233A460DA950460BF01DFD0028DB
:105E500037DB20220DF2C6210DA812F0A4F890BB6A
:105E6000316800900122A1F12003C1F1200522FA3E
:105E700005F502FA03F32B438A40DDE91E5121EABE
:105E8000030125EA0205CDE91E5148484C233A4654
:105E90000DA90BF02DFD002813DB9DF88030414843
:105EA000013B8DF880309DF8823023F002038DF89D
:105EB000823020AA032300210BF0BAFD0028BFF690
:105EC00025ACF12422E408F10108B6E70DF2C62062
:105ED00001F078FD00283FF452AC002D3FF492AD64
:105EE00030480BF0B3FD0028EBDB4FF49673B0FBAA
:105EF000F3F50BF0B5FB10B901200BF0A9FB2A4E0E
:105F0000DFF8A0800022EFB29742326015DD4FF437
:105F100096735A4352A940460BF0B6FC0028D0DBDA
:105F20009DF8513213B132680132ECE74622A9A93B
:105F300052A812F038F80028F5D133689F423FF498
:105F400061AD9DF8CE319DF82A239A4202D00224F9
:105F5000FFF7DCBB0DF2EA210DF5C77012F023F854
:105F600005460028F3D10DF2EA21C3220DF5C770D2
:105F70000FF0F6FF32680B4800954FF496735A43C2
:105F800052A90BF0B5FC99E7FF24FFF7BFBB032430
:105F9000FFF7BCBB3424FFF7B9BB00BFAB0A00203E
:105FA00020090020AB51020018090020B351020063
:105FB0002DE9FF47DDE90C861F463368DDF8389090
:105FC000242B82460C46154603D8152004B0BDE8A4
:105FD000F0870146202220460FF0C2FF84F82050AF
:105FE00003A801F023FD002801DAF120EEE7039B6E
:105FF0006A061BBAC4F821304ED53368C92BE4D9E0
:106000002649102204F125000FF0AAFF002384F88E
:1060100035304623514684F83630202204F15900A9
:106020000FF09EFF9DF84030012B38BF012304F193
:106030007D0A00934A469DF83C30514604F13700F2
:1060400001F01AFD0028D0DB19F1070F05D101225C
:1060500049465046FEF72DFE05E019F1080F13D111
:106060005046FEF7C5FD7D302B060AD5336800EBA0
:106070000805AB42A9D34246394620440FF070FFD1
:10608000284630600020A1E7054BD3F805104945AC
:10609000ABD1D3F80120DCE72520E5E7EC5F020077
:1060A000A20A00202DE9F04FADF2445D134608909E
:1060B00009920AA80A46EBA9FDF7D8FF0DF12408BA
:1060C000044620B9FFF770FA002805DDC4B2204667
:1060D0000DF2445DBDE8F08F0BF0C2FA10B901205B
:1060E0000BF0B6FAEB9B13F0400219D0DDF8141553
:1060F00089B90BF0B5FA38B901200BF0EBFA012899
:1061000000F0C98002285DD001F0D0FD00280CBF4E
:1061100035243124DBE703F0C003402B00F0458336
:106120009DF8F03403F00C01082904BF23F00C03A0
:106130008DF8F0342AB19DF8F03423F00C038DF87B
:10614000F0349DF8F03403F00C02042A01D12C2421
:10615000BDE703F03002202A04BF23F030038DF89E
:10616000F0349DF8F0349D07F1D0012262F3010371
:106170008DF8F03401F09AFD48B1EB9B5C0606D433
:106180009DF8F03403F03003102B00F010839DF8DD
:10619000F03413F0300F17D1EB9B580614D40025C0
:1061A000DDF8EC34002B78D1EB9B5A0677D40BF05A
:1061B00057FA002877D101200BF08CFA01286AD019
:1061C000022870D1272482E701F070FD0028E6D074
:1061D000EB9B5906E3D5B44B1B78002B00F0E9820A
:1061E0009DF818350DF2F1422021ECA801F0AEFB2C
:1061F00008B933246BE7012001F0D2FB0028F8D066
:10620000FDA801F0DFFB0028F3D001F045FA0546B8
:106210000028EED0FDA801F0E7FBC1E701F032FA5B
:1062200080B3192453E70DF2DC400CF085FE002802
:1062300040F014810134DDF8EC34A342B4D995A9BF
:106240000DF2DC40FDF752FB2022FDA90DF2762075
:1062500011F0A9FE0028E6D14AA995A801F066FC34
:10626000C82106464AA812F06BFE002EC0F2FB8140
:10627000D9D19DF87532032B01D1002DD3D0EB9BE2
:106280005B06CBD40BF0ECF90028CAD101200BF04F
:1062900021FA0128C5D12D2419E70024CBE701F00C
:1062A000F1F9002883D001F001FA01F00BFA01F0B6
:1062B00015FA9DF83C459DF8193504F001041C447D
:1062C0009DF81B35002B18BF013414F0FF0435D0A6
:1062D00027AE00238C2231464AA80CF090F92246C2
:1062E0000CA94AA80CF0CDF90446002840F0B6806D
:1062F0009DF83C35DF0700F19A809DF81B357BB196
:106300006A490CA8FEF745FD0346002840F0A68028
:106310009DF81B250CA80CF085F9002840F09E8004
:106320009DF81935002B40F09B800CA94AA80CF071
:10633000B9F9002840F092804A9CA41B9DF81A35B8
:10634000002B00F09B809DF8F03403F03003102BFD
:106350007FF4FDAE042208980CA90CF092F90028F5
:106360007CD1012200230CA80CF05CF9002875D127
:106370004F490CA8FEF70DFD00286FD140F25713CE
:10638000C8F800309DF81B3504939DF8F034009454
:1063900003F03003002CA3F110010CBF40226FF07A
:1063A0003F024B424B41039342EA8502DDF8D83469
:1063B00042F00102CDE9018302F0FD0227AB95A96D
:1063C000FDA8FFF7F5FD044600287FF480AE022209
:1063D00000230CA80CF026F900283FD1D8F8003093
:1063E00007931A4695A90CA80CF03EF90546A8BBE0
:1063F0004FF4967A014652464AA80FF08DFB9DF85D
:10640000F03403F03003102B40F0318129480BF0B9
:106410001DFB0028C0F2278190FBFAF9DFF894B049
:106420002F4640264F452BD1402E60D15EE0412BB8
:1064300007D89DF8F04404F03004A4F11000444261
:1064400044411D490CA8FEF7A4FC38B904F114011D
:106450000CA80CF0F6F800283FF44FAF122436E6F3
:1064600016490CA8FEF795FC0028F7D115210CA8B9
:106470000CF0E7F800283FF458AFEFE703226AE793
:106480004FF496730AFB07F24AA958460BF0FCF941
:106490000028C0F2E8809DF831328BB1402E08BF51
:1064A0003E460137BEE700BFAC0A00206251020041
:1064B000BB510200AB5102006E5102008451020038
:1064C00020220DF5A571FDA811F06DFD0028E8D181
:1064D0009DF854349DF8AE219A42E2D10DF5B77182
:1064E0000DF2144011F05FFD0028DAD13E463F2E38
:1064F00000F3BB8046220DF28B214AA80FF030FD3D
:10650000C3220DF214410DF5B7700FF029FD9DF86F
:106510001A358DF8323200238DF833329DF83C3530
:10652000DA070CD5412BC3F346014FEA530206D8D4
:106530008DF833128DA80DF21C510FF011FD0027BC
:106540009D488DF83172032310AA39460BF062FA88
:10655000B842C0F288809DF8423097488DF841607B
:1065600043F001038DF8423010AA032339460BF0A3
:106570005FFAB84277DB4FF496738F48009703FBBE
:1065800006F24AA90BF0B4F9B8426CDB8B480BF069
:106590005DFA002867DBDFF824B24FF040094FF0C6
:1065A0004C0A90FBFAF7BD4207D10023CDE9253311
:1065B000B9F1400F18BF4D4619E04C230AFB05F214
:1065C00014A958460BF060F900284CDBDDE92532B0
:1065D000134305D1B9F1400F08BFA9460135E2E7E1
:1065E000202214A9FDA811F0DEFC0028F6D12022FB
:1065F000FDA914A80FF0B4FC2022F4A91CA80FF0E8
:10660000AFFCFC9B2493DDE925120120A6F12003B9
:10661000C6F1200C20FA0CFC00FA03F343EA0C0349
:10662000B04001431A4300274C23CDE925126348AB
:10663000009703FB05F214A90BF05AF9B84212DBDC
:106640009DF842305C4867F300038DF842309DF8B6
:10665000403001338DF8403010AA032339460BF047
:10666000E7F9B84203DAF12431E528242FE50322C3
:1066700000230CA80BF0D6FF00287FF4EFAE032216
:1066800010A90CA80BF0FDFF00287FF4E7AE4C49E1
:1066900010A8FEF77EFB00287FF4E0AE6FF0060244
:1066A0004FF0FF3310A80BF0BDFF00287FF4D6AEEB
:1066B000444910A8FEF76DFB00287FF4CFAE12F01E
:1066C0009BFDBDF81C1095A812F0A4FD2021ECA89C
:1066D00012F0A0FD95A812F0A5FD3B4B95AA10461F
:1066E000196801F04FFA0246C8F800000028BAD035
:1066F00095A910A80BF0B8FF00287FF4AFAE33497E
:1067000010A8FEF746FB00287FF4A8AE012214A9CA
:1067100010A80BF0B3FF024600287FF49FAE95A9A6
:1067200014A80BF0A1FF00287FF498AE149DA81CBC
:1067300001F0B2FA002896DB592305F8013C687095
:10674000031202302B7014A9054410A814950BF005
:10675000A9FF00287FF482AE10A90CA80BF0A2FFBD
:1067600000287FF47BAE9DF81A353BB908980CA938
:106770000BF098FF00283FF4AAAC6FE68DA94EA855
:1067800001F03AFB00287FF469AE052200230CA833
:106790000BF048FF00287FF461AE20228DA90CA8E1
:1067A0000BF062FF0028E1D058E614248FE4362471
:1067B0008DE434248BE400BFAB510200B3510200DE
:1067C000B7520200C2510200746A0200C6510200B0
:1067D0002DE9F04FADF2944D0D4606901C46079200
:1067E00000214FF496727BA807AE0FF095F93CB9E3
:1067F0009A4B1C70FEF7D8FE00283FDDC5B206E0BC
:10680000974B1B78022B07D0082B05D03025284644
:106810000DF2944DBDE8F08F904B1A78914B1B7898
:106820009A42F3D2FCF782FA8F4B1B68C01A47F2E8
:1068300030539842EAD88D4C636D002B40F00681AE
:10684000DFF8188298F80090B9F1000F00F050823C
:1068500098F80030864A8748D25C4FF496735A43C2
:106860007BA90BF011F80028C0F2968049A97BA8FB
:1068700001F05CF9002800F00C818DE02A463368B5
:106880007A4908A8FDF780FD05460028BFD10AF027
:10689000E7FE10B901200AF0DBFE744C236813F008
:1068A00040011BD0E26FA2B90AF0DAFE30B9012034
:1068B0000AF010FF012808D0022808D001F0F6F9EC
:1068C00000280CBF35253125A1E72D259FE7272579
:1068D0009DE703F0C003402B00F05F83664B674DDC
:1068E00000221A7094F858302A7003F00C0008281F
:1068F00004BF62F3830384F8583029B194F8583008
:1069000023F00C0384F8583094F8583003F00C024C
:10691000042A00F0448303F03002202A40F041832F
:1069200003F00302022A02BF012262F3010384F88A
:10693000583001F0BBF900283FF47DAF23685806BA
:106940007FF579AF4E4B1B78002B00F02C834D4A1E
:1069500094F880302021A2F1350000F0F7FF08B94B
:10696000332554E701232B7000F096FE0028F7D062
:10697000022001F015F80028F2D0434801F022F877
:106980000028EDD0404801F02FF854E749A97BA832
:1069900001F0CCF8051E01DAF12538E74FD19BF85C
:1069A000002001217BA801F059F8002847D09DF86C
:1069B0000C3223B9636D434568D12E2527E7122297
:1069C0007FA9C6A80FF0CCFA2A480BF03FF80028A0
:1069D000E2DB4FF4967AB0FBFAF7BD422FDA254896
:1069E0004FF496730AFB05F27BA90AF04DFF0028CD
:1069F000D2DB9DF8F5320BB10135EEE722482022BB
:106A00000DF20E2111F0CFFA0028F5D112227FA944
:106A1000C6A811F0C8FA0028EED1CBE708F10108AA
:106A2000636D4345C6D97BA94846FCF75FFF16490D
:106A300020220DF20E2011F0B6FA0028A6D048460A
:106A40000CF07AFA0028E9D01225E0E6DFF82CB045
:106A50004FF0000804F14409E2E700BFA10A00205A
:106A6000AB0A0020A00A00209C0A00206409002034
:106A700022090020AB5102006209002063090020B6
:106A8000AC0A0020BD09002068090020A64B0122A5
:106A90001A70DFF8C08298F800302BB1A24B1B7837
:106AA000012B94BF00230123A04AA14F13703B7810
:106AB00003BB94F8585005F00305012D1AD1236843
:106AC0005A0602D500F0DEFD58B90AF0C9FD40B9FA
:106AD00028460AF0FFFD01283FF4F7AE02283FF4F4
:106AE000F6AE944B01221A7000F0E0FD00F0EAFDD2
:106AF00000F0F4FD616D98F80020003918BF012105
:106B00007BA800F0ABFF00283FF457AF256894F84E
:106B10003531C5F300351D4415F0FF0521D00DF1C9
:106B200098098C2249460EA800230BF068FD2A46DE
:106B30000AA90EA80BF0A5FD002885D194F83531DF
:106B4000002B40F02B812368DB0400F138810AA977
:106B50000EA80BF0A7FD00287FF476AF0E9DA5EBE5
:106B600009059DF80C32002B636D14BF042203222B
:106B700033B93B7823B96C4B1B78012B88BF0132AA
:106B80009DF8F6320BB10132D2B206980AA90BF089
:106B900078FD00287FF458AF012200230AA80BF0EB
:106BA00041FD00287FF450AF022212A90AA80BF081
:106BB00068FD00287FF448AF5F4912A8FEF7E9F8A6
:106BC00000287FF441AF46227BA912A80BF04CFDB0
:106BD00000287FF439AF594912A8FEF7DAF80028E7
:106BE0007FF432AF564912A8FEF7D3F800287FF49D
:106BF0002BAF12A90AA80BF055FD00287FF424AF93
:106C00004C4A5048127840F27713336098F80030BD
:106C1000009542EA83022B1E18BF012342EAC312E9
:106C20009DF80D3204939DF80C32003B18BF0123F0
:106C30000393DDF82E320DF54678CDE90163D2B22B
:106C400026AB4146FFF7B4F9054600287FF4DFADD7
:106C5000022200230AA80BF0E5FC00287FF4F4AE22
:106C6000D6F8009041464A460AA80BF0FDFC0028E1
:106C70007FF4EAAE032200230AA80BF0D3FC00281D
:106C80007FF4E2AE3049202208EB09000FF068F9EA
:106C9000424649A9DDF82E02CDF8008009F1200313
:106CA00000F094FF4146024630600AA80BF0DCFC7D
:106CB00000287FF4C9AE9DF80C32002B40F0EE8026
:106CC000636D002B00F037819DF8F632002B40F009
:106CD0004C8106980AA90BF0E5FC00287FF4B4AEBD
:106CE0003B7801333B70FCF721F8184B18608EE5B8
:106CF00017480AF0ABFE051EFFF64EAE0A4FDFF84E
:106D000054A087F80090DFF848904FF4967304F190
:106D1000040BB5FBF3F5013D691C1DD13B78002B3D
:106D20007FF496AD49E600BFA00A002021090020AB
:106D3000A10A0020620900203051020049510200DE
:106D40004E51020068090020880900209C0A00209A
:106D5000AB510200630900204FF4967303FB05F268
:106D60007BA948460AF090FD0028FFF615AE9DF875
:106D7000F51289B99AF800207BA800F06FFE58B18F
:106D800020220DF20E21584611F00DF920B93B7862
:106D90005A1C3A70854AD554013DBDE784490AA87A
:106DA000FDF7F7FF00287FF44FAE9DF8F722BEA94C
:106DB0000AA80BF059FC00283FF4C5AE44E63B7826
:106DC000002B3BD094F8333194F81121012B62D180
:106DD00098F800300093774912AB7FA800F0CEFFFF
:106DE00000283FF70BAD94F8333194F8112100934C
:106DF000012B12AB18BF103A6F48194600F008FD7E
:106E00000028FFF6C9AD6D4A3B78127801339342F2
:106E100003D16948402112F093F869490AA8FDF7A7
:106E2000B8FF00287FF410AE94F8112112A90AA827
:106E30000BF01AFC00283FF48AAE05E6614B1B7884
:106E4000002B00F0AE8094F833115B4800F0A4FCF6
:106E500000283FF7D3AC94F833315B4D0193009594
:106E600094F81131A5F151022021A5F1910000F013
:106E700053FD00283FF474AD94F833310093A5F12D
:106E8000510394F811211946A5F1910000F00EFD6F
:106E9000002897D080E5103AD2B299E70422002367
:106EA0000AA80BF0BFFB00287FF4CEAD474E337825
:106EB000002B0CBF0122032212A90AA80BF0E1FB50
:106EC00000287FF4C1AD424912A8FDF762FF0028F7
:106ED0007FF4BAAD9DF872220DF2322112A80BF0A8
:106EE000C3FB00287FF4B0AD33783BB912A90AA8E0
:106EF0000BF0D8FB00283FF4E3AEA5E5354912A816
:106F0000FDF747FF00287FF49FAD0DF2732112A813
:106F1000FDF73FFF00287FF497AD2F4912A8FDF73A
:106F200038FF00287FF490ADADA912A8FDF731FF1E
:106F30000028DBD088E53B78002B7FF4C5AE1F4CE2
:106F40002378012B7FF6C0AE002305220AA80BF0A0
:106F500069FB034600287FF477AD22780AA80BF07E
:106F600061FB00283FF4B0AE6EE5BEA97FA800F03B
:106F700043FF00287FF468AD072200230AA80BF026
:106F800051FB00287FF460AD2022BEA90AA80BF0B7
:106F90006BFB00283FF49DAE56E5142537E42C2505
:106FA00035E42B2533E4342531E400BF22090020E9
:106FB0006E510200250A0020E5090020A00A0020E9
:106FC0008451020062090020760A00202109002075
:106FD000305102003F510200335102002DE9F041CF
:106FE000074694B014461E4601F1FF38002900F010
:106FF000DB8200F097FB3268651C29460023013ACA
:1070000068460BF0FCFA394611F8017B0D2F12D8B7
:10701000A7B17B1E0C2B11D8DFE813F012001B0068
:107020001000250010008D02920221001000A00225
:10703000AB02BC021000412F00F09082F12319E056
:1070400042466846FFF72EF82070002840F0828202
:1070500037E2002342466846FFF7BAFBF4E7002216
:1070600001231146F7E70D2204A968460BF009FB3E
:1070700010B1122323706DE20122002304A80BF04B
:10708000D1FA0028F5D103220CA904A80BF0F6FAD6
:107090000028EED1B0490CA8FDF77BFE0028E8D10E
:1070A000AE490CA8FDF775FE0028E2D1AC490CA84A
:1070B000FDF76FFE0028DCD10CA904A80BF0F2FA52
:1070C0000028D6D10222002304A80BF0ABFA002836
:1070D000CFD104220CA904A80BF0D0FA0028C8D103
:1070E000A0490CA8FDF755FE0028C2D19E490CA866
:1070F000FDF74FFE0028BCD19C490CA8FDF749FEC6
:107100000028B6D19A490CA8FDF743FE0028B0D15B
:107110000CA904A80BF0C6FA0028AAD10322002368
:1071200004A80BF07FFA0028A3D1102291490DEB9F
:1071300002000BF099FA00289BD10422002304A836
:107140000BF070FA002894D1062210A904A80BF0C5
:1071500098FA00288DD1884910A8FDF71AFE00285A
:1071600087D1152110A80BF06CFA002881D1834932
:1071700010A8FDF70EFE00287FF47BAF152110A8A4
:107180000BF05FFA00287FF474AF7D4910A8FDF77B
:1071900000FE00287FF46DAF00F088FD00F11401BF
:1071A000C9B210A80BF04DFA00287FF462AF754900
:1071B00010A8FDF7EEFD00287FF45BAF152110A8A5
:1071C0000BF03FFA00287FF454AF6F4910A8FDF789
:1071D000E0FD00287FF44DAF152110A80BF031FA27
:1071E00000287FF446AF694910A8FDF7D2FD0028BA
:1071F0007FF43FAF152110A80BF023FA00287FF48D
:1072000038AF10A904A80BF04DFA00287FF431AF75
:107210000522002304A80BF005FA00287FF429AF0B
:1072200040F21452002304A80BF0FCF900287FF46C
:1072300020AF0622002304A80BF0F4F900287FF405
:1072400018AF02220CA904A80BF018FA00287FF44A
:1072500010AF012200230CA80BF0E4F900287FF402
:1072600008AF022200230CA80BF0DCF900287FF401
:1072700000AF0CA904A80BF015FA00287FF4F9AEB2
:107280000722002304A80BF0CDF900287FF4F1AE0B
:107290000822002304A80BF0C5F900287FF4E9AE0A
:1072A0000822002304A80BF0BDF900287FF4E1AE0A
:1072B0004622002304A80BF0B5F900287FF4D9AECC
:1072C0000922002304A80BF0ADF900287FF4D1AE09
:1072D00002220CA904A80BF0D1F900287FF4C9AE52
:1072E0002B490CA8FDF755FD00287FF4C2AE2949B3
:1072F0000CA8FDF74EFD00287FF4BBAE0CA904A836
:107300000BF0D0F900287FF4B4AE0A22002304A8C1
:107310000BF088F900287FF4ACAEDFF8808098F895
:107320000030002B0CBF022203220CA904A80BF092
:10733000A5F900287FF49DAE022208A90CA80BF045
:10734000A0F900287FF495AE134908A8FDF721FDA8
:1073500000287FF48EAE23E0CA510200D151020012
:10736000DA5102006E5102006251020084510200A3
:1073700077510200EC5F020059510200E351020014
:10738000EC510200F65102000152020010520200BC
:107390002152020025520200B7520200A20A002028
:1073A0006FF006024FF0FF3308A80BF03BF90028FE
:1073B0007FF45FAE7E4908A8FDF7EBFC00287FF460
:1073C00058AE7C4908A8FDF7E4FC00287FF451AED4
:1073D00008A90CA80BF066F900287FF44AAE022237
:1073E00008A90CA80BF04DF900287FF442AE7249B1
:1073F00008A8FDF7CEFC00287FF43BAE6FF0070233
:107400004FF0FF3308A80BF00DF900287FF431AEE0
:10741000674908A8FDF7BDFC00287FF42AAE65493E
:1074200008A8FDF7B6FC00287FF423AE08A90CA835
:107430000BF038F900287FF41CAE98F80030002BD0
:107440004CD10CA904A80BF02DF900287FF411AE43
:107450000B22002304A80BF0E5F800287FF409AE06
:107460004FF48052002304A80BF0DCF800287FF4CE
:1074700000AE0E22002304A80BF0D4F800287FF4FD
:10748000F8ADC922002304A80BF0CCF800287FF443
:10749000F0AD0F22002304A80BF0C4F800287FF4FD
:1074A000E8AD2022002304A80BF0BCF800287FF4EC
:1074B000E0AD04A968460BF0F5F800287FF4D9ADDB
:1074C00020700099491B013131603C4B22781F70BC
:1074D000002A66D1002014B0BDE8F081022208A97C
:1074E0000CA80BF0CEF800287FF4C3AD324908A8F1
:1074F000FDF74FFC00287FF4BCADD8F8052008A8A4
:10750000D3170BF08FF800287FF4B3AD284908A8F3
:10751000FDF73FFC00287FF4ACAD264908A8FDF735
:1075200038FC00287FF4A5AD08A90CA80BF0BAF828
:10753000002886D09DE542466846FDF737FC83E586
:10754000FBF7F4FB42F21073984205D80120FDF7D7
:107550000FFF20700121B7E73020FAE74246684666
:10756000FEF7C2F82070D0B90099491B01310A27F3
:10757000AAE70AF075F830B901200AF0ABF8012843
:1075800004D0022804D0002323709AE72D2371E54C
:107590002F236FE542466846FDF7D8FD54E50121EB
:1075A000E5E7FF221A7095E74FF0FF3093E700BF41
:1075B000495102004E510200B7520200AB0A0020AE
:1075C00037B500230B714B718B716FF06F03CB716B
:1075D0000379802B0C4613D14379102B1BD140F239
:1075E0003C5301930A688189006801ABFFF7F6FC00
:1075F000019BA380002810DA0023A37169230BE00C
:10760000F3B94379032B18D00AD8012B0FD0022BE2
:1076100010D00023A3716D23E371002003B030BDAF
:10762000102BFAD0A42BF4D100F034FDE2E700F0E7
:1076300009FCDFE700F092FCDCE700F017FDD9E77A
:107640006E23E9E708B5322101200AF00FF8002087
:1076500008BD0000074B10B51870074B01241C70C3
:10766000FBF764FB054B00F5EA4030301860044B33
:107670001C7010BDB40A0020B50A0020B00A00201A
:10768000B60A0020024B187808B1024B18787047F0
:10769000B60A0020B40A0020024B187808B1024B49
:1076A00018787047B60A0020B50A0020034B1B78F3
:1076B00013B1034B00221A70704700BFB60A0020B6
:1076C000B40A0020034B1B7813B1034B00221A703D
:1076D000704700BFB60A0020B50A0020044B1B7893
:1076E00023B1044A137823F010031370704700BFCE
:1076F000B60A0020B70A0020054A00231370054A85
:107700001370054A1370054A1370054A13707047C9
:10771000B80A0020B70A0020B60A0020B50A0020E7
:10772000B40A002008B5084B1B785BB1FBF7FEFAE2
:10773000064B1B68984205D9FFF7B8FFBDE8084023
:10774000FFF7DABF08BD00BFB60A0020B00A00206C
:107750000149002011F070BAD90A002008B5044888
:10776000202111F0F5FBBDE80840FFF7C5BF00BFC1
:10777000A10B002008B5FFF7EBFFBDE80840FFF7BD
:10778000EDBF0000024B03491A680EF0E9BB00BFD1
:10779000506A02001D0B002030B5034602468BB034
:1077A00004460D460020174911F092FA002826DB06
:1077B000012D07D122462021204611F041FD002055
:1077C0000BB030BD02AD2022002128460EF0A4F9F6
:1077D0002023224619462846009511F042FB0094CA
:1077E0002846094A0F232021203411F03AFB074A8A
:1077F00000940E232021284611F033FBDFE70120FF
:10780000DEE700BFD90A00202952020039520200E7
:107810002DE9F0438FB089461746002105461C220A
:1078200005A81C46DDF858800EF076F901238DF886
:107830001430164B0C9301AE154B09961021B8F17C
:10784000010FCDE906978DF82C100D930894304662
:1078500018D111F075FB05A80A9510F019FAB8F1C6
:10786000020F05460AD13A46214604F110000EF0F7
:10787000A7FA1022314620460EF072FB28460FB0C0
:10788000BDE8F08311F064FB2035E4E7357C0100AE
:10789000497C010007B50B46009203492022FFF7FF
:1078A000B7FF03B05DF804FBA10B0020F0B58FB06B
:1078B00006460C46154600211C2205A81F460EF060
:1078C0002BF901238DF81430114B0C93114B0D93B0
:1078D000149B01A81022012B09908DF82C200BD1AC
:1078E000114611F02DFB05A8CDE906450A9608972B
:1078F00010F092FA0FB0F0BD0F2D06D921460EF010
:107900002FFB2036103D1034EDE74FF0FF30F1E74C
:10791000357C0100497C010070B58AB0DDE90E5666
:10792000022E02D1202928BF202102AC009411F0A0
:1079300098FA012E0CBF102220222946204610F072
:1079400032FBB0FA80F040090AB070BD2DE9E74182
:1079500098460C4B054618780E46174670B1FBF753
:10796000E5F9094B00F5EA40303018602A46CDE9C8
:107970000078064833462021FFF7CEFF03B0BDE86C
:10798000E08100BFB60A0020B00A0020A10B002051
:10799000024A137803431370704700BFB70A0020F0
:1079A000034B1B78034214BF01200020704700BF27
:1079B000B70A0020024B1878431E584258417047BE
:1079C000B80A002008B50146064803783BB12022DA
:1079D000013010F0E8FAB0FA80F0400908BD01204B
:1079E000FCE700BFB80A002001460348012200F866
:1079F000012B20220EF0B4BAB80A002010F1080FB3
:107A00000BD0C31D0BD0084B1A7852B1D3F80530F8
:107A100098420CBF032009207047042070470020C3
:107A200070470920704700BFA20A002010B5024627
:107A3000044604230848012109F0ECFF00280ADB72
:107A4000236805480133236022460423012109F0FD
:107A5000EFFF00EAE07010BDA151020090F8213064
:107A6000022B04D1002A18BF012108467047032BBE
:107A700008BF1146F7E700002DE9F0430446BDB00A
:107A80001046C4F842200F461946FFF7B7FF0928F1
:107A9000054644D09DF8103184F8201084F8213038
:107AA0002048202302AA042109F0B4FF002833DB78
:107AB00004F110090AAE1021484611F049FA1223C8
:107AC0004A46202102A8009611F0CBF90DF16C086E
:107AD0002023194604F122023046CDF8008011F02F
:107AE000C0F91022414620460EF03AFA31462846A7
:107AF00011F0D2F80028DDDB202102A811F020FAD5
:107B0000094B414653F8252038460EF029FA3046F5
:107B1000C82111F015FA00203DB0BDE8F0834FF008
:107B2000FF30F9E7A1510200506A020073B501F17C
:107B3000440605460C46124820233246042109F02B
:107B400069FF00281ADB122305F1100220213046BC
:107B5000009411F086F9202305F1220219462046EF
:107B6000009611F07EF910222946304610F01BFADB
:107B700020B12046C82111F0E3F9012002B070BD08
:107B8000A151020070B5B4B005460E460E48144629
:107B9000202302AA002109F03DFF002811DB2A461C
:107BA000334602A90094002010F0D6FFC82102A895
:107BB00011F0C6F922462146202010F075FB34B0A2
:107BC00070BD0020FBE700BFA15102002DE9F0418C
:107BD0008AB017469846FFF711FF0928109D0E46F8
:107BE000044619D0042811D111F056F8002813DBEF
:107BF000009543463A463146204610F0ADFF002836
:107C00000ADB224B18690AB0BDE8F08103282AD1AB
:107C100011F042F8002802DA4FF0FF30F3E702AA31
:107C200031461B4810F0A2FB11F02EFC202102A8C7
:107C300011F058FC38461FFA88F111F053FC284621
:107C400011F098FC134B009553F824702A463B46DC
:107C50003146204610F080FF0028DDDB032C0DD1DB
:107C60000A4BD868CFE711F0C7FA38461FFA88F1F7
:107C700011F0D0FA284611F0D5FAE3E72A46294652
:107C8000F8B20AB0BDE8F04110F00EBB2C6A020059
:107C90007B6B0200746A020001464FF49063024855
:107CA000002209F0F1BD00BFA151020007B5012378
:107CB0000DF107020221044809F0ACFE003818BF9C
:107CC000012003B05DF804FBA151020013B50B467F
:107CD000044691B90A460C48022109F0A9FE002881
:107CE00009DB08238DF80730074801230DF107024F
:107CF000032109F09DFE02B010BD024611F0A0FA6A
:107D000010232246E7E700BFA15102001FB5044639
:107D1000102308486A46022109F07CFE002807DB90
:107D200010222146684610F03EF9003818BF0120A5
:107D300004B010BDA151020007B501230DF10702E7
:107D40000321054809F066FE0028A8BF9DF807003A
:107D500003B05DF804FB00BFA151020007B5012389
:107D60008DF807000DF107020321034809F060FEBA
:107D700003B05DF804FB00BFA15102002DE9F04300
:107D80008BB002AC80460E461A489DF848901746C4
:107D90001D4622462023052109F03CFE00281CDB5D
:107DA000B9F1000F08D0224620231178013B6FEA79
:107DB000010102F8011BF8D1102342462021204680
:107DC000009411F04EF820230095324619462046C3
:107DD00011F047F8402F03D000200BB0BDE8F0832E
:107DE000202320350095F2181946204611F039F865
:107DF000F2E700BFA151020037B520230A4605462D
:107E00000C460F48052109F005FE002815DB6178B6
:107E10002378A2784B405140A27F23705340A37730
:107E2000E278E37F61705340E377204600941023AB
:107E30002A46202111F015F8002003B030BD00BF04
:107E4000A15102002DE9F0438389402BAFB00446D5
:107E50000F4608D000238B716723FB710024204656
:107E60002FB0BDE8F08309F0FBFB98B909F0F8FBEF
:107E700018B9C821022009F0F9FB09F0DDFB20B98F
:107E80006FF07A03BB716923E7E7002009F0DAFBA2
:107E900009F00CFC2568D7F8008005F120062022A7
:107EA00031460DF192004FF001090EF059F8CDF86E
:107EB000009000236FF006020CA91CA8FFF7DCFD60
:107EC000041ECCDB11F098F90024494603A88DF874
:107ED0000C4011F09FF93046202111F09BF9284603
:107EE000202111F097F9052388F80030042388F841
:107EF000013040220CA9462508F1020008F1430692
:107F00000EF02EF82A461CA988F8425030460EF092
:107F100027F822460F484FF4906308F1890109F0D1
:107F2000B3FC041E9BDB29461CA811F073F9412108
:107F300008EB090011F06EF904A811F073F9064B73
:107F400062191968324404A8FFF71CFE89340444FE
:107F5000BC8083E7A1510200746A02002DE9F0435E
:107F6000838906680D68872BADF5117D07460C46A1
:107F700009D06FF07F03A3716A23E37100200DF530
:107F8000117DBDE8F08396F84030462B03D00023E6
:107F90008B716723F1E706F12008202206F16301C7
:107FA000404606F141090FF0FEFF0028E1D108A983
:107FB0004846FFF7BBFDC0B20028DAD1BB79072BDA
:107FC00004D16FF07A03A3716923D6E709F048FB67
:107FD00078B909F045FB18B9C821022009F046FB21
:107FE00009F02AFB0028ECD0002009F02BFB09F057
:107FF0005DFB40F2571307AA07936FF006010023B9
:10800000CDE90121CDE90333009301223AA940468D
:10801000FDF7CEFF07460028D3D111F0EDF825215A
:108020003AA811F0F7F82021304611F0F3F8404655
:1080300011F0F8F8052242A928460DF091FF0A4BED
:1080400005351B680095424608A9384610F084FDA6
:10805000C82108A810F074FF2A462946202010F0F5
:1080600023F90530A08089E7746A020008B50B4641
:10807000818929B100229A716722DA71002008BD36
:1080800006225971186802491A710DF069FFF5E767
:10809000CA51020010B50B46002406220A714C7129
:1080A000186802490DF05CFF204610BDCA5102005D
:1080B0002DE9F84300230B714B718B716FF06F0347
:1080C000CB7143791D2B0C4617D0A42B5ED183793D
:1080D000042B01D1C5792DB16FF07903A3716A2307
:1080E000E37107E02A49206805220DF039FF0523D6
:1080F000237165710020BDE8F8838379002BEBD1F3
:10810000C779002FE8D10B6819221A700B684FF05D
:10811000010883F801800B6802259D700B68DD70F3
:108120000B683A261E710B685D710B684FF00409ED
:1081300083F8069008680730FAF7F0FF236883F8A1
:108140000B90236883F80C80236841225A732368BC
:1081500003229A732368DD7323681D7423685E7499
:1081600023680D229A742368DD7423681D752368C3
:108170005E7523680E229A752368DD7523681D7667
:1081800023685E761A2323716771B3E76D23A7E72F
:1081900048520200014B00221A707047C10B0020A8
:1081A000034B987BA0F1FF0358425841704700BF32
:1081B000C20B002007B583795BB1012B08D06FF0AB
:1081C00079038B716A23CB71002003B05DF804FB47
:1081D000FF23054905488B730123009300220F23D9
:1081E00009F086FBC017F0E7C20B00204E520200D8
:1081F00007B5012300930C490C481323002209F012
:1082000077FB01300CDB09484FF4806109F0DCFB9F
:1082100001304FF0FF30A8BF002003B05DF804FB31
:108220004FF0FF30F9E700BF1C600200535202001C
:10823000174B37B500221A70044658B11549164835
:108240000F220DF08DFEFFF7D3FF002814DA4FF058
:10825000FF301AE0114809F0F9FB0F280546EDD16F
:108260000F4809F0F3FB0028E8DD0B490B482B46CB
:10827000224609F009FB07E001230093064907485D
:108280000F23002209F034FBC01703B030BD00BF3C
:10829000C10B00200D600200C20B00204E520200F4
:1082A000535202008379042B03D1C3792BB90020E8
:1082B000704713B9C2790C2A04D06FF079038B711F
:1082C0006A2304E08289012A03D88B716723CB716A
:1082D000EDE703681A78E12A06D15B78032B0AD10F
:1082E000064B01221A70E2E72AB95B78012B02D112
:1082F000024B0222F6E76FF07D03E0E7C10B00209E
:1083000038B5C28852BA92B2B2F5806F05460C46B3
:1083100004D90023A3716723E3710AE08368B3F5EE
:10832000806FF6D814490978012904D002290ED0AB
:10833000F9B100200AE0D1180F29EAD821680F48C6
:1083400009F0A2FA002811DA4FF0FF3038BD0C49CD
:10835000497B21B16FF07D03A3716923DCE7D1185C
:10836000B1F5806FD5D821680648E9E7AB68A380EE
:10837000DFE76FF07A03EFE7C10B00204E520200F7
:10838000C20B00205352020037B5C28852BA92B2D3
:10839000B2F5806F04D900238B716723CB7109E09C
:1083A0008389B3F5806FF6D80F4C2478012C04D95B
:1083B000022C07D0002003B030BD6FF07A038B7120
:1083C0006923EBE7094CA47B14B16FF07D03F6E75A
:1083D0009D18B5F5806FDEDC00940168044809F053
:1083E00087FAC017E7E700BFC10B0020C20B0020CF
:1083F0005352020010B500230B714B718B716FF05B
:108400006F03CB714379B02B0C460BD0D62B0CD01D
:10841000A42B0DD1FFF746FF00280BDA0023A37130
:10842000692306E0FFF76CFFF6E7FFF7ADFFF3E720
:108430006D23E371002010BD00F18D02072012F8BA
:10844000013D0133DBB213700BB90138F7D20130B3
:108450004FF0FF3018BF00207047F7B506461546AD
:108460001A4690F842309DF820700C4603F00F0336
:1084700096F841100094012B00F14400A1F1020193
:1084800010D12B4610F091FC14204FB1204410F86D
:10849000013C03F00F03E018E25C02F07F02E254BB
:1084A00003B0F0BD022B2B4603D110F0DAFC2020E4
:1084B000EBE710F032FD4020E7E700002DE9F04F38
:1084C0008379A5B006460D460BB9C47934B16FF077
:1084D0007903AB716A23EB7100200BE0DFF8BC90ED
:1084E0002D48032389F8003009F0B0FA002804DA97
:1084F0004FF0FF3025B0BDE8F08FDFF8A480DFF843
:1085000098A08D23B0FBF3F74FF08D0BB368A34217
:1085100006D998F80020974204D8002389F8003043
:10852000AC80D9E78D2302FB0BF26946504609F077
:10853000ABF90028DCDB9DF80020B168D31C234494
:108540008B4205D94FF0FF33AB716123EB71E7E745
:1085500098F80030013388F80030002AD6D02B6814
:1085600072221A552B689DF80020234401325A705C
:108570002B689DF84220234404F1030B9A7028686D
:108580009DF800200DF1010158440DF0E9FC9DF823
:1085900000405C44B8E700BF58520200E40B0020E2
:1085A000DB0B002007B50023009301F185020823AF
:1085B00000F18501024809F09BF903B05DF804FB66
:1085C000585202002DE9F0411D4690F88430DB0737
:1085D00004460F46164602D40020BDE8F081082A62
:1085E00011D100F18508294640460EF021F90028F6
:1085F0000CDC2946324640460DF0B2FC3946204696
:10860000FFF7D0FFE8E74FF0FF30E6E76FF001003B
:10861000E3E700002DE9F04FC379012BB9B006461E
:108620000C4604D96FF07903A3716A2314E07B48E8
:1086300009F00CFA051E04DA4FF0FF3039B0BDE83E
:10864000F08FDFF8E88198F8000060BBB389012B58
:1086500005D80023A3716723E3710020EEE731689A
:108660000A78742A02D06FF07F03DDE74A786C4FF6
:1086700002F1FF3CBCF1070F3A7001D93870F2E704
:10868000901C9842E5DC674802310DF069FC3B78AC
:10869000B28902339A42DCD3F379002B624B0CBFD0
:1086A000012202221A70DFF880A18D234FF0000909
:1086B000B5FBF3F30393B3684B4507D998F8007003
:1086C000039BBB4205D8584B00221A70A4F80490B3
:1086D000C3E78D2317FB03F750483A4614A909F066
:1086E000D3F80028A8DB9AF800109DF85020022942
:1086F00014BF40210421531D0B44B1684B448B42ED
:1087000005D94FF0FF33A3716123E371DEE798F8D9
:108710000030013388F80030002ACCD02368712261
:1087200003F8092023689DF850204B4409F1020BFF
:108730005A7020680DF1510158440DF011FC9DF85C
:1087400092309DF8505003F0F003102B5D440ED191
:10875000236877225A5523682B4401225A702368D4
:108760009DF893202B4405F103099A70A3E79DF827
:10877000D49019F0020902D023687C22EAE7DFF8DE
:10878000A0B0284B9BF80020394614A8FFF71AFF29
:10879000002804DA6FF07D03A37169235CE79AF87F
:1087A00000309BF800202168022B05F1030005F141
:1087B000010705F1020B1AD176234B5523680521D9
:1087C000D95523689DF8931003F80B1027680123EF
:1087D0000744009304A9134B14A8FFF73EFE04229C
:1087E000014638460DF0BCFB05F1070963E7752328
:1087F0004B550C4BCDF80090014414A8FFF72DFE0B
:1088000023680130D85523689DF8932003F80B2086
:10881000236813F80790D9444DE700BF585202006F
:10882000D90B0020D10B0020E40B0020DB0B002033
:10883000024A00231370024A13707047E40B0020B1
:10884000DA0B00201FB50446FFF7F2FF68B10123E1
:108850000093002313481A46194609F049F80028E6
:108860000ADA4FF0FF3004B010BD0E4809F0EEF800
:108870000028ECDB2046F6E700230A481A460221CE
:1088800009F0D6F80028ECDB08210DEB010010F010
:108890005FFB082303480DEB0302032109F0C8F82E
:1088A000C017E0E75852020070B58D26B0FBF6F312
:1088B00006FB1303B8B004460D461BB16FF0010070
:1088C00038B070BD1D4809F0C1F80028F6DBA042A1
:1088D000F4D91A483346224614A908F0D5FF0028D7
:1088E00002DA4FF0FF30EBE79DF85030002BE5D077
:1088F0009DF8923003F0F003102BF2D114A8FFF78B
:108900009BFD0028EDDB214614A8FFF74BFE082253
:108910000DF1D5010DEB02000DF022FB01230093B8
:10892000082202AB04A914A8FFF797FD0422014610
:1089300028460DF015FB9DF89300C1E75852020040
:108940002DE9F04FB24F00266FF06F030E714E719C
:108950008E71CB710C4639784379BBB0054651B95D
:10896000A42B00F07083A32B00F00B836FF07D032A
:10897000A371692348E2552B00F0C58316D8013B4B
:10898000DAB2042A03D90023A3716D233CE2042B3D
:10899000F9D801A252F823F0CB8900006B8B0000BC
:1089A000198C000087890000CF8C000003F15F0262
:1089B000D2B2042AE7D8A23B032B00F20F82DFE8F1
:1089C00013F01502E002420398038379002B40F074
:1089D000D88390F80790B9F1000F40F0D2838389D3
:1089E000012B06D84FF4CE4301E046F68423E38002
:1089F00025E3D0F8008098F80020712A02D04FF4C7
:108A0000D543F4E798F801707A1E3F2AF7D8BA1DCB
:108A10009342E7DDBA1C18F80220732AEFD1FA1C42
:108A200018F802A0AAF103023F2AE8D83E1D08EB7D
:108A30000602039218F8062002F0F001102901D076
:108A40002029DCD102F00F02013A022AD7D8039A7A
:108A50005278043A042AD2D85644B3420CD918F8B2
:108A60000620782A08D1721C9342BBD918F80290CC
:108A7000B9F1030FC3D802360022B342CDE9062272
:108A800019D918F806207A2AACD1721C92B29342F6
:108A9000A8D918F80220042AB1D11029AFD1711D2C
:108AA00089B28B429EDDB11C18FA81F107A80DF046
:108AB00057FA0636B6B2AB89B34293D1554808F09F
:108AC000C5FF0028C0F2C78008F102038D2502937C
:108AD000B0FBF5F64FF0000BB0465E4525D146459C
:108AE00001D1632E81D802998DF858703A460DF164
:108AF00059000DF035FA03998DF899A052460DF101
:108B00009A000DF02DFA082206A90DF1DD008DF86E
:108B1000DC900DF025FA002300938D2303FB08F26F
:108B200016A93C4808F0E4FE92E03A488D2305FB84
:108B30000BF216A908F0A8FE0028C0F28C809DF860
:108B40005830BB4208D102993A460DF159000DF058
:108B50006FFE002800F026839DF8583013B9464573
:108B600008BFD8460BF1010BB7E78379002B40F023
:108B70000883C679002E40F004838389012B7FF699
:108B800031AFD0F8009099F80020712A7FF437AF08
:108B900099F8018008F1FF323F2A3FF630AF08F123
:108BA00002029342FFF41EAF1A4808F04FFF071E5F
:108BB00051DB8D23DFF85CA0B7FBF3F709F1020965
:108BC0005F433546AF4202D146F684130FE78D234B
:108BD0002A4616A9504608F057FE00283BDB9DF8B0
:108BE0005830434512D1424649460DF159000DF027
:108BF0001FFE064650B9284602F008F900282ADB75
:108C00008DF8586000968D232A4689E78D35D9E77F
:108C1000DA0B0020585202008379002B40F0B18219
:108C2000C379002B40F0AD8282894AB1012A3FF41A
:108C3000D9AE05682B78732B7FF4E1AE6B7863B9FE
:108C400001233B7000231A46B948022108F0F0FEC8
:108C5000002880F2F48100238AE6112B7FF4CFAE46
:108C6000152A7FF7BFAEEB7C742B7FF4C8AE2B7D4B
:108C700003F1170842457FF7B5AE03F11501695CB2
:108C800075297FF4BCAE03F1160115F80190B9F116
:108C9000140F7FF4B4AE03F12B018A427FF4A2AE2D
:108CA0000DF1580AEE1C05F1150210213046CDF8E1
:108CB00000A010F07AF84A4605EB080150460FF084
:108CC00072F9002880D1387010233246BCE78379CE
:108CD000002B40F05682C379002B40F052828389EA
:108CE000022B7FF67FAE06683278712A7FF487AE5A
:108CF00096F8019009F1FF323F2A3FF680AE09F164
:108D00000405AB427FF66EAE09F10202B25C712A35
:108D10007FF475AE09F1030216F8028008F1FF3204
:108D20003F2A3FF66CAE08EB05029342FFF45AAEC1
:108D30007F4808F08BFE00288DDBB31C4FF08D0BB5
:108D40002E440293B0FBFBF54FF0000A2F46554529
:108D50001AD1BD423FF438AF8D256F4374482B467E
:108D60003A4616A908F090FD0028FFF674AF424677
:108D700031460DF159008DF858800DF0F1F80023BF
:108D800000933A462B46CBE669488D230BFB0AF24B
:108D900016A908F079FD0028FFF65DAFBD420DD1A0
:108DA0009DF858304B4509D102994A460DF15900BA
:108DB0000DF03EFD002814BF2F4657469DF8583051
:108DC000434508D1424631460DF159000DF030FDC2
:108DD000002800F0E7810AF1010AB8E7554B0022AC
:108DE0001A7021462846FFF769FB31E7AF7917B9BA
:108DF000EB79012B02D96FF079030DE0AB89022BDF
:108E000004D80023A3716723E37118E12A6811785D
:108E1000712904D06FF07F03A3716A23F4E75678B9
:108E2000721E3F2AF6D806F1020A5345E9D340489C
:108E300008F00CFE0028FFF60EAF4FF08D0BB0FBD4
:108E4000FBF8B84502D16FF07B0391E50BFB07F906
:108E500037488D234A4616A908F016FD0028FFF66C
:108E6000FAAE9DF85830B34201D00137E9E72968DE
:108E7000324602310DF159000DF0DAFC0028F4D130
:108E80009DF8DC309B0708D508F0EAFB28B908F00C
:108E900021FC013801287FF669AD9DF89A3003F076
:108EA000F003202B48D1AA89F11C9142A9D22B684A
:108EB00013F80A007428ADD15F5C791E0729A9D880
:108EC000311D01EB070842459BDB19443A4604A8D3
:108ED0000DF046F8AB89434593D304AB3A46494677
:108EE00016A8FFF76FFB0028FFF640ADEB7922686C
:108EF000002B38D076231370236805225A70012383
:108F0000256800933A4606A904AB16A8FFF7A5FA10
:108F100003350146042228460DF022F823689DF807
:108F20009B209A7023685B780233A38087E000BFA0
:108F300058520200DB0B0020102B7FF48CAE16A8D9
:108F4000FFF77AFA002802DA6FF07A0310E5494653
:108F500016A8FFF727FB08220DF1DD0104A80CF08D
:108F6000FFFF0827C2E775211170216800933A4678
:108F700004AB033116A8FFF770FA2368013058706C
:108F8000CCE7AB79002B7FF436AFEB79002B7FF485
:108F900032AFAB89022B7FF634AF2D682A78752A61
:108FA0007FF438AF6A78142A7FF434AF182B7FF639
:108FB00028AFAA7D742A7FF42DAFEE7D06F118024A
:108FC00093427FF41EAF7F48102306AA022108F0C7
:108FD00021FD0028FFF63FAE3FF435AF16AB7A4ACD
:108FE00000931021082306A80FF0DFFE1422A91C0D
:108FF00016A80EF0D8FFB0F100080CBF0123002323
:109000003B707FF407AF16AB05F1180200931021F7
:10901000334606A80FF0C9FE102106A80FF090FFF6
:10902000236875221A70236814225A70206816A9C2
:1090300002300CF095FF1623237184F80580002080
:109040003BB0BDE8F08FAB79042B45D1ED79002D15
:109050007FF4D1AE5D4B18689A8816909B79ADF875
:109060005C2016A9072220688DF85E300CF078FF8E
:109070002268544808230732032108F0CBFC00285B
:10908000FFF6E9AD0F2323714E486571012306AA4F
:10909000022108F0BFFC0028FFF6DDAD02D101235C
:1090A0003B70CCE7484808210FF052FF236846493F
:1090B0007422DA73236808221A74206811300CF0C5
:1090C0004FFF23687B225A76226801239376226819
:1090D000D376A3880D3328E7002B7FF48CAE0029CC
:1090E0003FF444AC3A4A137021462846FFF792FAFF
:1090F000AEE5384B1B78032B3FF473AE013B012BDD
:109100003FF622AFF0E78379013B012B39D8C379D1
:10911000012B36D88389012B7FF664ACD0F800B0E0
:109120009BF80020712A7FF46AAC9BF8018008F15B
:10913000FF323F2A3FF663AC08F102029342FFF48C
:1091400051AC204808F082FC0028FFF684AD0BF1FA
:10915000020B4FF08D0AB0FBFAF7B7423FF434AD83
:109160000AFB06F917488D234A4616A908F08CFB1E
:109170000028FFF670AD9DF85830434504D0013605
:10918000EBE746F6862332E4424659460DF1590094
:109190000DF04EFB0028F2D19DF89A3003F0F00359
:1091A000202B02D146F6851321E4A879EB790093B0
:1091B00001389DF858200DF159034946C0B201F01D
:1091C00001FE45E558520200DC0B00203060020031
:1091D000DB0B0020E40B00200A461423002108F0DA
:1091E00019BC0A461423002108F022BC0A460423B5
:1091F000012108F00FBC0A460423012108F018BC25
:1092000007B50023ADF804308DF8063001AA03231A
:109210009321034808F00CFCC01703B05DF804FB71
:109220005D52020070B503780C2253430D460D4980
:10923000CC5C064601341944224628460CF090FEC8
:109240003378032B04D8B378012B03D113236B702D
:10925000204670BD022B01D11223F8E74FF0FF34F6
:10926000F6E700BFC86002002DE9F0413D4B9B7856
:10927000ADF5A36D05460C4623B96FF07D03A371D0
:10928000692309E083793F2B02D1C379FF2B09D0F1
:109290006FF07903A3716A23E37100200DF5A36DCC
:1092A000BDE8F08181890668012903D80023A371F4
:1092B0006723F1E733784D2B02D06FF07F03E9E7A6
:1092C000013601AB6A460139304608F03EF9009B91
:1092D000002BF2D10128F0D9019AA989531C03442B
:1092E0008B42E3D116F80280B31808F15C02D2B2C7
:1092F000142AE2D81C4951F82270002FDDD05A7888
:109300000AB1032AD9D1023202A938469E1808F0C0
:1093100041FF00281ADB2B68AA89F31AD21A3146BA
:1093200002A808F047FD421CC0D0831CC5D000280D
:1093300001DA0023A3E702A9384608F047FF002816
:109340004FF4A26102A804DA0FF0FAFD4FF0FF30EB
:10935000A4E70FF0F5FDB8F1B60F9ED1FFF750FF6F
:109360009CE700BF4E0000203C60020008B508F0FA
:1093700077F920B9BDE80840192108F077B908BD90
:109380002DE9F0415B4FADF5A36D3B7805460C46EA
:10939000164632B1D90713D46FF07D03A371692348
:1093A00040E09A07F8D5544F02A9384608F0F2FE7B
:1093B000002816DA4FF0FF300DF5A36DBDE8F081FF
:1093C0004E48012302AAC42108F024FB0028F1DB47
:1093D0009DF808301BB93B7823F001033B70484FE0
:1093E000E2E79DF80C30033B012B22D808F038F956
:1093F000F8B9DFF81C81F9F799FCD8F800308342FE
:1094000007D2C01A3F4B1B784FF47A7253439842ED
:109410000FD3002008F05EF90138012805D8002399
:10942000A3716623E3710020C6E7F9F77FFCC8F853
:1094300000009DF8093023B96FF07703A3716A2308
:10944000F0E79DF80A30DB0702D46FF07A03A5E756
:10945000FFF78CFF9DF808309A1F022A0DD82A4981
:10946000AA8951F8233005215B00B3FBF1F39A423E
:109470000BD90023A3716723D4E7032B05D8234915
:10948000AA8951F823309A42F3D102A9384608F04C
:109490008BFE00288EDBAA892968236802A808F0C1
:1094A000D1FE051E86DB4FF4A26102A80FF048FD35
:1094B000A580002EB7D001AC10480323224693218B
:1094C00008F0A8FA0028FFF675AF0DF10701A142D8
:1094D00006D011F8013D0133DBB20B70002BF6D042
:1094E000064803232246932108F0A2FA00289ADABC
:1094F00060E700BFE80B00206F5202005D520200DF
:1095000066520200E50B0020506A0200746A0200F5
:109510004000002070B56C4B1B789A07ADF5A46D28
:1095200005460C4604D46FF07D03A371692324E043
:10953000664804A908F02EFE002871DB9DF814305F
:10954000033B012B21D808F08BF8F0B9604EF9F7F6
:10955000EDFB3368834207D2C01A5E4B1B784FF491
:109560007A725343984210D3002008F0B3F80138C0
:10957000012807D80023A3716623E37100200DF5AD
:10958000A46D70BDF9F7D2FB30609DF8113023B99E
:109590006FF07703A3716A23EFE79DF812309B0702
:1095A00002D46FF07A03C0E7FFF7E0FE474804A952
:1095B00008F0FAFD002833DB9DF81000831F022B12
:1095C00036D8454BAA8953F8203001339A4208D245
:1095D0004FF4A26104A80FF0B3FC0023A37167232A
:1095E000CBE729680B783BB14FF4A26104A80FF0D8
:1095F000A7FC6FF07F03CDE70DF10B05009501315E
:10960000236803AA06A80FF090FD00284FF4A2617A
:1096100004A808DA0FF094FC9DF80B30002BE8D179
:109620004FF0FF30ABE70FF08BFC039BA380A5E767
:109630000528F5D8AB89072BCAD92A681378A62B39
:10964000D2D193787F2BCFD1D378492BCCD15379FA
:10965000862BC9D1204B517853F8203003281BD8D2
:109660009D1DA942C0D11579D91C8D42BCD19179DB
:1096700001339942B8D1D379042BB5D108210A44DA
:10968000236806A90FF024FB002811DA4FF4A26129
:1096900004A80FF055FCC3E75D1DA942A4D11579BC
:1096A000991C8D42A0D1917999429DD10721E6E77D
:1096B0009DF81020094B53F82230A3804FF4A2618B
:1096C00004A80FF03DFC59E7E80B00207852020097
:1096D00040000020E50B0020506A0200746A02007E
:1096E000F0B5C379ADF2145D05460C4613B16FF0C9
:1096F000790317E08289022A08D0052A06D08B71E7
:109700006723E37100200DF2145DF0BD2B681B7818
:109710005C33DBB2142B03D82B4A52F8237027B9E1
:109720006FF07F03A3716A23EBE76946384608F0C0
:109730003BFD002802DA4FF0FF30E4E7AB79802BE5
:109740002ED1FFF713FE684608F056FD0028F2DB25
:109750006946384608F03AFD0028ECDB23687F2292
:109760001A70236849225A70216801220231684622
:1097700008F0B4F94FF4A261064668460FF0E0FB2A
:10978000002ED8DB0236A680AB79802BBAD10F49E8
:1097900038460CF0C5FE0028B4D1FFF731FDB2E722
:1097A000812B0BD19DF80130002BD7D14FF4A26152
:1097B00068460FF0C5FB6FF07703B3E74FF4A26183
:1097C00068460FF0BDFB92E73C6002006652020063
:1097D000044A00231370044A9370044A9370044AA5
:1097E00013707047E80B0020590000204E00002045
:1097F000E60B002030B5ADF2345D0446FFF7E8FF1C
:1098000070B100230125854800951A46194608F0D5
:109810006FF800280BDA4FF0FF300DF2345D30BDE9
:109820007E4808F013F90028EBDB2046F5E77B487B
:109830008DF809502B460DF10902FC2108F0F8F8CB
:109840000028E8DB002375481A465E2108F0F0F88E
:109850000028E0DB002371481A465B2108F0E8F895
:1098600004460028D7D1034602462D216B4808F054
:10987000DFF80028CFDB39238DF80A3067482B4604
:109880000DF10A02352108F0D3F80028C3DB634844
:109890008DF80B402B460DF10B02C42108F0C8F8DF
:1098A0000028B8DB142103A80FF04AFB4FF4A26292
:1098B000214608A80CF030F9594B5A48089308A9DA
:1098C00008F084FC0028A6DB564803A9FFF789FCB2
:1098D0000028A0DB534803A9FFF78DFC00289ADB82
:1098E000022351488DF8223008A908F06FFC0028A7
:1098F00091DB4D4803A9FFF774FC00288BDB4A4835
:1099000003A9FFF778FC002885DB4848012408A953
:109910008DF8224008F05AFC0028FFF67CAF43483F
:1099200003A9FFF75EFC0028FFF675AF3F4803A9C7
:10993000FFF761FC0028FFF66EAF3848142303AA36
:10994000FF2108F075F80028FFF665AF33481423AF
:1099500003AAFE2108F06CF80028FFF65CAF2F4840
:10996000142303AAFD2108F063F80028FFF653AF83
:109970002F4A2A4800231370FB21234608F058F889
:109980000028FFF648AFFFF73BFC0028FFF643AF87
:109990000023284800941A46194607F0A9FF00281A
:1099A000FFF639AF0023244800941A46194607F001
:1099B0009FFF0028FFF62FAF0023204800941A468F
:1099C000194607F095FF0028FFF625AF1C491D48F2
:1099D0000323062208F058FC0028FFF61CAF1A49A2
:1099E0001A480323082208F04FFC0028FFF613AFA3
:1099F000002217480323114608F046FC0028FFF612
:109A00000AAF00238DF80930044823460DF10902FE
:109A1000FC2108F00DF8C017FFE600BF5D52020000
:109A20000600010066520200785202006F520200E6
:109A3000E50B0020815202008A520200935202007C
:109A40002F500200590000209C5202004E000020BE
:109A5000440000202DE9F04300230B714B718B7102
:109A60006FF06F03CB710C4601798BB0054629B1BD
:109A70006E23E37100200BB0BDE8F0834379884A80
:109A8000A52B0CD101231370864801230DF10F0281
:109A9000FC2107F0BFFF002834DA002305E010782E
:109AA00080B9CC2B04D16FF07A03A3716923E0E76E
:109AB000CA2BE9D1AB797F2BE6D1EB79212BE3D10E
:109AC0000223E0E7012817D1CC2BECD0CA2B09D117
:109AD000AB797F2B02D1EB79212BF1D0724B002196
:109AE000197007E0DA2BF9D1AB797F2BF6D1EB793E
:109AF000212BF3D10023C6E7CC2B1EBF6A4B11707C
:109B00001970C1E79DF80F206B79012A0AD1442B07
:109B100000F0B380A42B00F08C806FF07A03A37167
:109B20006223A6E7882B01F0868021D82C2B00F039
:109B30003A860CD8242B00F0FD852A2B01F060809A
:109B4000202B00F081850023A3716D2391E7842BE6
:109B500001F07380F7D8442B00F08C80472BF2D1B2
:109B600021462846FFF7BCFD054607F09FFD8EE025
:109B7000DA2B00F04C8640D8CA2B00F08A8026D819
:109B8000A42B56D0A52BDED1A979474A0023022960
:109B9000137051D8EB79042B4ED1AB89062B7AD1B7
:109BA0002B68187860280FD1587804280CD1987841
:109BB0005C2809D1D878022806D118797F2803D1EA
:109BC0005B79212B00F037856FF07F033FE0CC2BD2
:109BD000B9D1AB797F2B2FD1EB79212B2CD1AA894D
:109BE000002A58D130490B780133DBB2012B0B70BE
:109BF00040F024854FF4906390E3DB2B00F0FA876C
:109C0000E62BA0D1AB79BBB9EB79ABB9274D284690
:109C100008F0FDFB0028FFF640AF03D0AB78002B27
:109C200000F0598501238DF8203008AAFC2100F0AE
:109C30007CBEAB79042B02D06FF0790307E0EB799F
:109C4000002BF9D1AA89062A04D06FF07D03A371F5
:109C50006A230EE7164928680CF0EAFD0028F4D1C3
:109C6000144A10480123FB2107F0D4FE0028BFF658
:109C700001AF12E7002A3FF416AFAB79002BDBD11E
:109C8000EB79002BD8D10120FFF7B4FD0546002D5C
:109C9000EDE7AB8983B10023A3716723E9E600BF39
:109CA000E60B00205D520200E70B00204E00002072
:109CB000B8600200E50B00207A48ED8804A908F09E
:109CC00069FA6EBA0028B6B2FFF6E7AE764806A982
:109CD00008F060FA0028FFF6E0AE744808A908F022
:109CE00059FA0028FFF6D9AEB5F57A4F00F07E8319
:109CF000FA2E32D8B5F5DC4F00F0E2806E2E0BD88C
:109D0000B5F5BC4F66D0B5F5CA4F7CD0B5F59E4FC2
:109D100052D06FF077039AE7B5F5444F00F0118306
:109D2000B5F55E4F00F03683B5F5F44FF1D12368F9
:109D30005F487A221A70236805225A70236893219B
:109D4000997022680323D3702268043207F062FE00
:109D50000028FFF6A2AE072338E042F27F139D42AF
:109D600000F0CC8247F621739E4211D845F25F0382
:109D70009D423AD045F25F239D423DD040F20123FF
:109D80009D42C6D14B4A236812781A7001231DE008
:109D900046F27F639D4200F0CD8247F27F439D42B1
:109DA000B7D1236881221A70236801225A70236870
:109DB00020229A70032309E03F49206810220CF00A
:109DC000CFF820680A30F9F7A9F91023237100238E
:109DD00063714FE6226836483F235E2107F01AFE82
:109DE0000028FFF65AAEA08044E621683048FF23E1
:109DF000002207F049FDF3E7304920680A220CF001
:109E0000AFF80A23E2E72368294865221A7023681D
:109E100000225A7023685B2199702268272304323C
:109E200007F0F8FD051EFFF638AE2368DD70ADB211
:109E30002B1D22689BB25F26D6546B1D22689BB2F5
:109E40002D21D154AF1D2068BFB27A1C02440823D3
:109E5000174807F0DFFD0028FFF61FAE236807351F
:109E6000D85510FA85F52368ADB235215E556B1CC7
:109E700022689BB2AE1CD154B6B22068721C024458
:109E800001230B4807F0C6FD0028FFF606AE236845
:109E90000335985510FA85F5ADB22368AA1E5A709D
:109EA000A580E7E566520200785202006F52020078
:109EB0005D520200E50B0020B8600200AE600200B7
:109EC0002368D7496E221A7023684FF0820883F8FE
:109ED0000180236800279F702368DF7023684F226A
:109EE0001A71236810225A71206806300CF038F875
:109EF00020681030F9F712F92368CA495F229A7571
:109F000023685222DA7523680A261E7620683246B4
:109F100019300CF025F82368C3497F2583F82350B6
:109F20002368662283F824202368082283F82520EA
:109F3000206826300CF014F82368BC4983F82E50B2
:109F40002368742283F82F202368032283F83020AB
:109F50002368812283F831202368012583F8325059
:109F60002368202283F833202368732283F8342067
:109F7000236883F83580236883F83670236883F874
:109F800037702368C02283F83820236883F839604B
:109F9000206832463A300BF0E3FF2368C12283F891
:109FA0004420216804A84531FFF73CF90028FFF65A
:109FB00074AD80B200F146034530226880B2C22100
:109FC0001154216806A811FA83F19EB2FFF72AF90D
:109FD0000028FFF662AD3218216892B2C32088547F
:109FE0002168531911FA83F108A89EB2FFF71AF9F4
:109FF0000028FFF652AD06442368B6B2C421995535
:10A00000731922689BB20720D0542268B01C12FA40
:10A0100080F22B46864807F0FDFCF71C0028BFB2F3
:10A02000FFF63BAD236883484022DA55331D216893
:10A030009BB2B51DCA54731D21689BB2ADB2CA5400
:10A0400008F0E5F90028FFF628AD236858557A484E
:10A0500008F0DDF9F71D0028BFB2FFF61EAD23683A
:10A06000D855764808F0D3F906F108050028ADB2B6
:10A07000FFF613AD2368585506F1090322687048AE
:10A080009BB2C521D15406F10A0321689BB206F1A7
:10A090000B023C26CE54216811FA82F195B2FFF7EB
:10A0A0009BF80028FFF6F9AC2168284411FA80F1EA
:10A0B00085B26448FFF790F80028FFF6EEAC2168FF
:10A0C000284411FA80F185B25F48FFF785F800282F
:10A0D000FFF6E3AC2B18226855489BB2C621D15439
:10A0E0009A1C013321689BB295B2CE542168142387
:10A0F00011FA82F2FF2107F08DFC0028FFF6CDACAB
:10A1000021682A1895B24A4811FA82F21423FE21D6
:10A1100007F080FC0028FFF6C0AC21682A1895B231
:10A12000434811FA82F21423FD2107F073FC002842
:10A13000FFF6B3AC2B1822689BB2CD21D1549A1CE8
:10A14000013321689BB20C20C85421683C4811FAA5
:10A1500082F195B2FFF74AF80028FFF69EAC21681D
:10A16000284411FA80F185B23648FFF73FF80028FD
:10A17000FFF693AC2168284411FA80F185B2324889
:10A18000FFF734F80028FFF688AC2B189BB2226842
:10A19000DE21D1545A1C216892B2062088549A1CA0
:10A1A000216892B201208854DA1C21689DF81100C0
:10A1B00092B2022688541A1D216892B20220885455
:10A1C0005A1D21689DF8195092B28D549A1D21682C
:10A1D00092B203258D54DA1D21689DF8215092B268
:10A1E0008D5403F10802216892B2D6258D5403F1F3
:10A1F0000901256889B203F10A0268549DF8141018
:10A20000042998BF114892B298BF4156206888BF70
:10A210004FF0FF31815403F10B02216892B217E035
:10A22000B8600200AE600200A66002009C600200FE
:10A230005D52020059000020440000204E00002022
:10A2400066520200785202006F520200376002002C
:10A250002020885403F10C02216892B2D720885440
:10A2600003F10D01206889B2022545549DF81C10A8
:10A27000042998BF534803F10E0298BF4156206845
:10A2800092B288BF4FF0FF31815403F10F01206873
:10A2900089B22025455403F11002216892B2D820DA
:10A2A000885403F11100256880B203F112012E5485
:10A2B0009DF82400042898BF424D89B298BF2856C3
:10A2C000256888BF4FF0FF30685403F11301206800
:10A2D00089B220254554A3F124012068C1F3072544
:10A2E00080F83650206880F837102168100A88708E
:10A2F00021681433CA70A380FFF7BCBB324B1A78B5
:10A300003AB9216831484FF4906307F0BDFA00284C
:10A3100067E5012A05D14FF49063002221682C489B
:10A32000F3E7022A7FF4F5AC4FF490630022216832
:10A330002848EAE72849206808220BF011FE082384
:10A3400044E5226825480123C42107F063FB002867
:10A35000FFF6A3AB22682248402353702268937013
:10A360002268D37008F053F80028FFF696AB2368F4
:10A3700018711C4808F04BF80028FFF68EAB2368D4
:10A380005871194808F043F80028FFF686AB236897
:10A390009871E0E4236801221A7023689DF8112067
:10A3A0005A70236802229A7023689DF81920DA7087
:10A3B000236803221A7123689DF821205A7106230D
:10A3C00004E500BF37600200E70B00208152020065
:10A3D0008A52020093520200A66002005D520200FF
:10A3E00059000020440000204E0000202368C54989
:10A3F000C1271F702068072201300BF0B1FD2368D0
:10A40000C14901259D7023681F7220680722093009
:10A410000BF0A6FD2368BD499D7223681F74206858
:10A42000072211300BF09CFD2368B9499D74236805
:10A430001F7620680A2219300BF092FD2368B54977
:10A4400013269E76236883F8237020680722243021
:10A450000BF086FD2368B04983F82560236883F8F4
:10A460002B70206807222C300BF07AFD2368AB4953
:10A4700083F82D60236883F8337020680B22343012
:10A480000BF06EFD2368A6494FF0160983F835904E
:10A49000236883F83F7020680C2240300BF060FD89
:10A4A0002368984983F841602368C22783F84C7079
:10A4B000206807224D300BF053FD2368924983F842
:10A4C0004E50236883F854702068072255300BF0F3
:10A4D00047FD23688D4983F85650236883F85C70E4
:10A4E000206807225D300BF03BFD2368884983F824
:10A4F0005E50236883F8647020680A2265300BF090
:10A500002FFD236883494FF0120883F86680236883
:10A5100083F86F702068072270300BF021FD2368EC
:10A520007D4983F87180236883F87770206807225B
:10A5300078300BF015FD23687A4983F87980236819
:10A5400083F87F7020680C2280300BF009FD2368AF
:10A55000734983F88180236883F88C7020680C220B
:10A560008D300BF0FDFC2368664983F88E802368EC
:10A57000C32783F89970206807229A300BF0F0FC0B
:10A580002368614983F89B50236883F8A170206891
:10A590000722A2300BF0E4FC23685C4983F8A35047
:10A5A000236883F8A97020680722AA300BF0D8FC32
:10A5B0002368574983F8AB50236883F8B17020684B
:10A5C0000A22B2300BF0CCFC2368524983F8B36006
:10A5D000236883F8BC7020680722BD300BF0C0FCF4
:10A5E00023684D4983F8BE60236883F8C4702068EF
:10A5F0000722C5300BF0B4FC2368484983F8C660D5
:10A60000236883F8CC7020680B22CD300BF0A8FCB7
:10A610002368434983F8CE90236883F8D870206874
:10A620000C22D9300BF09CFC236883F8DA606FF0C1
:10A630001A03FFF7CBBB1170FFF71CBA022B7FF494
:10A6400068AB4FF4906372E6AA79531EDBB2FD2B20
:10A650007FF6F2AAEB79812B0CD1334B1B7803F0F8
:10A66000FE03314931480B70FF2A0FD1002383705C
:10A67000FFF700BA822B04D12B4B1B7803F0FD03AC
:10A68000EFE7832B7FF4D8AA2948EDE7AA8972B9AE
:10A690008378002B7FF4EEA907F0B9FE0028FFF6BF
:10A6A000FCA900F5C7404030E080FFF7E3B9296816
:10A6B00008ABD2B207F00CFE471C3FF4EEA9C61C53
:10A6C0003FF4E9AA9DF820301BB96FF07C03FFF737
:10A6D000ECB9023003D16FF07D03FFF7E6B9EB79F7
:10A6E000812B06D1104A137843F001031370FFF752
:10A6F000C1B9822B7FF4BEA90B4A137843F0020341
:10A70000F4E700BF106102001C6102002861020032
:10A71000C8600200D4600200E0600200F86002003D
:10A72000EC60020004610200E80B002059000020E8
:10A730004E000020AA79002A7FF47EAAEB79812BB3
:10A740002CD1BA4BBA4F1A70384607F05DFEAA8971
:10A7500029688242A8BF0246064608ABD2B23846F4
:10A7600007F0B6FD411C3FF498A99DF82030002B5E
:10A77000ABD00230AFD0AA8996423FF78CAA2968A5
:10A78000921BD2B23144384607F012FE431C3FF40C
:10A7900084A903307FF46EA9FFF77DBA832B7FF481
:10A7A0004BAAA44FD0E7AB7913F0FD067FF444AA7F
:10A7B000EA79812A7FF440AA23BB9F4807F024FE50
:10A7C0000646002887D0AA8929688242A8BF024687
:10A7D000D2B2994808AB07F07BFD421C3FF45DA95B
:10A7E0009DF82030002B3FF470AF02303FF473AF80
:10A7F000AA89B242FFF64FAA29688D48921BD2B2AD
:10A800003144C1E78B4B9B78002BF1D163E7894B37
:10A810009B78002B3FF45FAFEF887BBA9BB2D82BBD
:10A8200046D8C02B0DD8B7F5B64F78D0B7F5BC4F8A
:10A830007FF402AAAB893F2B3FF62DAA2A685E213E
:10A8400073E0C13B172B3FF6F7A901A252F823F0A2
:10A850007DA900007DA900007DA9000065AA000077
:10A86000399C0000399C00007BAA00008DAA0000E2
:10A870009BAA0000A9AA0000B7AA0000C5AA000070
:10A88000399C0000D3AA0000E5AA0000F3AA00004A
:10A89000399C0000399C000001AB0000399C00008D
:10A8A000399C000023AB000065AB0000A7AB0000A3
:10A8B00043F25F5297423CD045F63572934210D82E
:10A8C00040F201239F4200F08B8142F65F539F428A
:10A8D0007FF4B2A9AB89082B3FF6DDA92A682D21A8
:10A8E00023E045F25F039F422AD042F27F139F424A
:10A8F0007FF4A2A9AB89B3F5906F3FF6CCA94F4E78
:10A9000032785ABB0121009129684D4806F0F0FFCA
:10A910000028FFF6C2A800233370FFF7ABB8AB895D
:10A92000272B3FF6B8A92A685B21464807F080F834
:10A9300011E0AB89012B3FF6AEA92A683521F4E777
:10A94000AB89FF2B3FF6A7A90122009229683D4859
:10A95000002206F0CDFFC517FFF799B9012A04D1EF
:10A960000092296838480022D0E7022A7FF4D1A952
:10A9700001220092296835480022C7E7AB89013BD4
:10A980000C2B3FF688A9DFF8D0800026AB8918F899
:10A99000022C9A4206D00136092E08F10C08F5D196
:10A9A000FFF712B929680B78012B0DD18B78002B9A
:10A9B0007FF40AA94B780C2B0FD0102B33D0082B27
:10A9C0007FF402A9062509E0013A013140460BF067
:10A9D0002FFF0028DFD1F5B200E00725B7F5414F82
:10A9E0003CD01B4E1B4BB7F5424F08BF1E4608A973
:10A9F000304607F0CFFB0028FFF64FA89DF8203027
:10AA0000AB423FF437A8B7F5424F29D1042D3FF4AC
:10AA1000DBA800238DF820508DF8213008A930469E
:10AA200007F0BDFB97E70825D8E700BFE80B00203B
:10AA3000590000204E00002044000020E70B0020B9
:10AA4000815202005D5202008A52020093520200BB
:10AA50006F52020078520200CA600200814EC6E7BF
:10AA6000052DD4E7AB89012B7FF415A92A6811784D
:10AA700001293FF6A9A8C42157E7AB89142B7FF41D
:10AA80000AA929687748FEF7ACFB64E7AB89142B69
:10AA90007FF401A929687448F5E7AB89142B7FF48A
:10AAA000FAA829687148EEE7AB89142B7FF4F3A864
:10AAB0002A68FF2139E7AB89142B7FF4ECA82A68B8
:10AAC000FE2132E7AB89142B7FF4E5A82A68FD212B
:10AAD0002BE7AB89042B7FF4DEA829686148FEF7D9
:10AAE0008AFB38E7AB89042B7FF4D5A829685E4838
:10AAF000F5E7AB89042B7FF4CEA829685B48EEE725
:10AB0000AA895B4852B1037893423FF6C4A84378C0
:10AB10009342FFF4C0A82968D2B235E607F0A1FC41
:10AB200019E7AB89022B7FF4B6A84E4808A907F0B5
:10AB300031FB0028FEF6B1AF9DF82430042B04D879
:10AB40004C4AD356022B3EF4AEAF2B681B78022B37
:10AB50003FF63AA8484A434852F823308DF824304B
:10AB600008A95DE7AB89022B7FF495A83E4808A9A8
:10AB700007F010FB0028FEF690AF9DF82430042B60
:10AB800004D83C4AD356022B3EF48DAF2B681B7879
:10AB9000022B3FF619A8384A334852F823308DF873
:10ABA000243008A93CE7314808A907F0F3FA002847
:10ABB000FEF673AF9DF82430042B04D82D4AD356EB
:10ABC000022B3EF470AF2B681B78022B3EF6FCAFD5
:10ABD000294A264852F823308DF8243008A91FE767
:10ABE000AB89012B7FF457A82A681178234A11708A
:10ABF000FB219AE621462846FEF736FBFFF746B8CA
:10AC0000AB799E2B0AD1EB799A2B7FF415A8012200
:10AC100021462846FEF7B4FBFEF7A6BF802B7FF443
:10AC20000BA8EB79862B7FF407A821462846FEF770
:10AC300071FCFEF799BF0022EAE7AB79002B7EF4A6
:10AC4000FBAFEB79002B7EF4F7AFA96840F23C53E1
:10AC500099423FF620A820680EF07AF9AB68FFF71A
:10AC60004ABB00BF66520200785202006F520200D7
:10AC7000440000203760020090600200E50B0020D5
:10AC800038B505460078087001280C4608D002281F
:10AC900007BF95F846304B70B0FA80F0400938BDD8
:10ACA0006A794A70A01CA91D0BF05AF96B7995F8C6
:10ACB00046201C44D81CA270F1E7000013B50446DE
:10ACC00070B10D488E210EF03BF9012300930A4923
:10ACD0000A488E23002206F00BFEC01702B010BDFA
:10ACE000064806F0B3FE8E280346EAD1024903481F
:10ACF000224606F0C9FDF0E7E90B0020A55202004C
:10AD000070B5084E0D4630460968FFF7B9FF29684F
:10AD10000446014406F14700FFF7B2FF0444AC804B
:10AD2000002070BDE90B002073B58479013CE3B2CB
:10AD3000012B054604D96FF079038B716A2304E077
:10AD4000838933B900238B716723CB71002002B054
:10AD500070BD0268107820B1022812D06FF07F0316
:10AD6000EBE7012BEED12B6814491B7814484722DE
:10AD7000544300220B55012300938E2306F0B8FDA7
:10AD8000E5E7022BDED95278202ADBD8D01C83429B
:10AD9000D8D10A48472606FB040663427270296828
:10ADA00003F047030233184402310BF0D9F82B6843
:10ADB000727813449B7886F84630D4E7E90B00207C
:10ADC000A55202002DE9F0410E4C9DF8188047274E
:10ADD00007FB00FC04EB0C0528460126C5F8011012
:10ADE000063019466A7104F80C600BF0B9F885F862
:10ADF0004680214606960448BDE8F0418E23002295
:10AE000006F076BDE90B0020A552020013B51149EA
:10AE10000B78012B0CD1D1F80120824208D10022FD
:10AE20000A7000938E230C4806F062FD02B010BD3C
:10AE300091F84730012B4FF0000208D18C6C84420E
:10AE400005D181F84720009302498E23EBE7104695
:10AE5000ECE700BFE90B0020A55202000128F7B57E
:10AE60000D460CD0022806D11A4C2078012808D0B3
:10AE7000022827D008B14FF0FF3003B0F0BD164CC8
:10AE8000F3E7D4F8010001A9FDF70EFD0028F2DB7D
:10AE9000019B29181BBA0A460A26AA4209D1002397
:10AEA0000B7094F84630002BE7D00D232B54013063
:10AEB000E3E7B3FBF6F706FB1733303302F8013D47
:10AEC0003B46EAE76278A11C28460BF049F8607817
:10AED000E7E700BF300C0020E90B002070B5ADF5AE
:10AEE000A26D04460E46154600214FF4A262684644
:10AEF0000AF012FE09238DF800306946012320462E
:10AF00008DF802608DF803508DF8043007F05EF97B
:10AF1000C0170DF5A26D70BD0348002100F8011B9C
:10AF200010220AF0F9BD00BF930C0020112822D096
:10AF30001DD8072821D002D808B303281FD0174BEB
:10AF40001A78F2B15A7882421DD09A7882421CD087
:10AF5000DA7882421BD01A7982421AD05A79824218
:10AF600019D09B7983420CBF032009207047142815
:10AF7000E5D10220704700207047062070470A2064
:10AF80007047092070470420704707207047082049
:10AF90007047052070470120704700BF770C0020E4
:10AFA00070B58579ADF5A26D0C4625B16FF07903CA
:10AFB000A3716A2303E0868936B18D716723E3713B
:10AFC00000200DF5A26D70BDC3799A2B0CD02ED840
:10AFD000812B04D81A0631D46FF07703E8E703F128
:10AFE0007E02D2B2012AF7D87E33654ADBB252F82C
:10AFF00023000028DAD0694607F0D6F80028C0F20E
:10B000009B809DF80030092BE6D022680123137045
:10B01000226853709DF8003022680A2B65D8DFE85B
:10B0200003F06396A49990938E9C9F64A2009B2B3F
:10B0300038D003F16402D2B2022AD4E7514A524D09
:10B04000802B08BF1546812101236A46E81C06F0C3
:10B05000E1FC002870DB284607F0EEF9064628469A
:10B0600007F0D5F9021E67DB216801230B70216808
:10B070004B702168FF20887021680520C870216806
:10B080000B7123689DF8001059712368062199718E
:10B0900023680221D97123681E7223685A720A2517
:10B0A000A5808DE7394801236A46812106F0B2FC6C
:10B0B000002841DB22680123137022685370226844
:10B0C0000321917021680222CA7021680A712268E6
:10B0D00056712268937122680521D171226813721A
:10B0E00023689DF80020D9E7112595702268022376
:10B0F000D3702268137123689DF803205A71236866
:10B100009DF804209A7123680322DA7123680122D2
:10B110001A7223689DF801105972236804219972EC
:10B12000216868460B3106F0D9FC00281FDA4FF47D
:10B13000A26168460DF004FF4FF0FF3041E707259C
:10B14000D3E7134B5D78D0E7114B1D79CDE7104B5A
:10B150005D79CAE70E4B9D79C7E70D4B9D78C4E733
:10B160000B4BDD78C1E70325BFE71425BDE700F1F0
:10B170000B054FF4A26168460DF0E2FE90E700BFB8
:10B18000346102006F00002064000020AA52020017
:10B19000770C002008B506F063FA20B9BDE8084036
:10B1A000192106F063BA08BD70B53B4B1B78ADF5AD
:10B1B000A26D05460C4643B96FF07D038B71692380
:10B1C000E37100200DF5A26D70BD8389042B03D8B7
:10B1D00000238B716723F3E7837993B9C3797E33B7
:10B1E000DBB21C2B0DD82D4ADA40D20709D50268F4
:10B1F0001178AC2905D19178802902D1D278012A21
:10B2000004D06FF07F03A3716A23D9E7244A52F870
:10B2100023606946304606F0C7FF002802DA4FF087
:10B22000FF30CFE72B681879FFF780FE09288DF8EB
:10B230000000E6D0FFF7AEFF684606F0DDFF00280D
:10B24000EDDBAA892968053A0531684606F0CAFC93
:10B2500028B14FF4A26168460DF072FED1E769464D
:10B26000304606F0B3FF0028D9DB23687F221A702E
:10B27000236849225A70216801220231684606F08B
:10B280002DFC4FF4A261054668460DF059FE002DD5
:10B29000C5DB0235A58094E7920C00200300001D59
:10B2A0003461020070B5294B1B78ADF5A26D0546DF
:10B2B0000C4623B96FF07D03A37169230FE0C279B7
:10B2C00002F17E03DBB21C2B05D8214951F8236023
:10B2D0000EB19B2A08D16FF07903A3716A23E37141
:10B2E00000200DF5A26D70BD6946304606F05CFF8A
:10B2F000002825DBA879FFF719FE09288DF8000042
:10B30000E9D0AA892968684606F0A6FC421C03D148
:10B310000023A3716723E2E7831C02D16FF07F0350
:10B32000DBE7002801DA0023C6E76946304606F06D
:10B330004DFF00284FF4A261684604DA0DF000FECC
:10B340004FF0FF30CDE70DF0FBFDC9E7920C002078
:10B3500034610200CB78012B0CD0032B084B9B7877
:10B3600002D03BB901207047002BFBD0054B1B7866
:10B37000002BF7D1034B01221A700020704700BF49
:10B380006F000020910C00202DE9F04F8389ADF271
:10B39000345D05460C461BB90023A371672307E003
:10B3A00003681B787C2B09D06FF07F03A3716A239D
:10B3B000E37100200DF2345DBDE8F08FC27902F137
:10B3C0007E03DBB21C2B05D8A64951F82380B8F1C7
:10B3D000000F02D16FF07903E8E79B2A13D183793C
:10B3E0000BB1032BF6D108A9404606F0D3FE002886
:10B3F000C0F2C4809DF8201009290CD16FF07A03A7
:10B40000A3716923D4E7984A42FA03F3DB07EAD52C
:10B410006FF07703CAE7A879FFF788FD8142D9D199
:10B42000002302AF05AEC7E90033C6E90033CDE91A
:10B430000033BB60B360A989286801AB6A46013953
:10B44000013006F082F8009B002BA5D1019B01334F
:10B450009BB2A9898B4221D39DF82430023B012B5A
:10B4600045D806F0FDF8002841D1F7F75FFC9DF8BC
:10B470002430032B08D17D4B1B68984204D9C01A95
:10B4800043F69723984232D9002006F023F9013879
:10B49000012828D80023A371662389E7286803F1CF
:10B4A0000109C35C83F08002022A1FFA89F9A3F123
:10B4B000800A02D9852B7FF477AF01AB6A46A1EBF6
:10B4C0000901484406F041F8009B26F81A00002BB9
:10B4D0007FF462AF019B99441FFA89F9484427F829
:10B4E0001A9083B2B5E7F7F721FC604B18603B88F0
:10B4F000B7F80290002B40F0C180B9F1000F00F0C6
:10B50000F580B6F802A0BAF1000F00F0BA80BA8850
:10B51000002A00F0B680B288002A40F0B280FFF71F
:10B52000FBFCE87908A9FFF715FF10B16FF07D0368
:10B5300066E79DF82030032B23D84D4A52F823307C
:10B540009A453FF629AF08A9404606F02DFE00288F
:10B5500014DBFFF71FFE9DF820309A1F022A39D80E
:10B5600022682968083249440AA80DF07BFD0028AA
:10B5700011DA4FF4A26108A80DF0E2FC4FF0FF30A1
:10B5800018E79A1F022ADED83A4A52F823309A4521
:10B590007FF402AFD7E723687C221A7023689DF8F6
:10B5A000201082225A70344B206853F82130191D24
:10B5B000090A81702068D9B20D1DC570206802711A
:10B5C000206842712268180A907122680833D1718C
:10B5D000A38040E0052BD1D8032B254E15D856F873
:10B5E00023302868A3EB0A034B4400EB09015246C1
:10B5F00018440AF0E5FB9DF82030286856F823101F
:10B600004844A1EB0A010DF09BFC23689DF8202023
:10B61000296856F822200433494408A806F012FE8F
:10B620000028ABDB9DF82030032B06D8226816F8E3
:10B630002300043211460CF037FE23687C221A7076
:10B640002268C3B2991C51702268822191702268CD
:10B650000430D370A0804FF4A26108A80DF070FCF4
:10B66000A7E600BF34610200FCFFFFE27C0000207F
:10B67000746A0200506A02002C6A0200B9F1000FDD
:10B6800034D0B6F802A0BAF1000F2FD1FFF744FC76
:10B690008E4B83F800A0EB799B2B7FF447AF236898
:10B6A0008B4D7C221A7023680A225A7023688122EB
:10B6B0009A7023680821D970206804300DF048FC86
:10B6C0000C23237184F805A0012308A940462B70A0
:10B6D00006F06AFD0028FFF651AF20680AAA691C2F
:10B6E00004300CF082FC0028B5DA42E7B988002962
:10B6F00000F0E780B288002A00F0AE807448067837
:10B70000012E02D0FFF708FC10E7EB799B2BF9D153
:10B71000082AF7D12B68013019440CF044FC0028AA
:10B72000F0D1FFF7F9FB694B1E7042E6B9F1000F4B
:10B7300049D0B6F802B0BBF1000F44D0644802789B
:10B74000022ADFD1EA799B2ADCD1BAF1080FD9D1DC
:10B7500029685246194401300CF025FC06460028A1
:10B76000D0D1BBF1080F03D0FFF7D6FBA67115E6C9
:10B7700023687C221A7023680A225A702368822266
:10B780009A70236883F803B00C236071237108A9B1
:10B79000404606F009FD0028FFF6F0AE2168286853
:10B7A0000AAA043148440CF020FC0028FFF6E1AE60
:10B7B0004FF4A26108A80DF0C3FBFFF7ADFB434BAC
:10B7C00001221A70F5E500297DD0B388002B7AD1CB
:10B7D0007F89002F77D07689002E74D0FFF79CFBED
:10B7E000E87908A9FFF7B6FD00287FF49FAE9DF821
:10B7F0002020384B53F82230032A98BF01339E4251
:10B800007FF4D2AD404606F0CFFC0028FFF6B6AE7E
:10B81000FFF7C0FC9DF8200023682A68032898BF22
:10B82000013704333A440AA90DF052FA0028FFF612
:10B83000A0AE23687C221A709DF82020264B216838
:10B8400053F82230DAB2901C487021688220887048
:10B8500021680433CA70BBE6002BB9D0B6F800A04B
:10B86000BAF1000F7FF462AFFFF756FB174B83F876
:10B8700000A0EB799B2B7FF459AE154D284602238F
:10B8800000F8013B08210DF063FB23687C221A704D
:10B8900023680A225A70236880229A70236808223B
:10B8A000DA700C23237184F805A008A9404606F03D
:10B8B0007BFC0028FFF662AE21680AAA0431681CEE
:10B8C0000FE7002BCAD1FFF727FB6DE5920C002094
:10B8D000930C0020506A0200746A0200084A094969
:10B8E00000231370084A1370084A9370084A937033
:10B8F0004FF0FF320A6007490A60074A1370704729
:10B90000920C0020840C0020910C00206F0000207D
:10B9100064000020800C0020880C002030B5ADF2BF
:10B920009C5D0446FFF7DAFF60B98D4806F08EF89B
:10B93000002807DB8B498A480723224605F0A4FF2D
:10B94000C0170BE000230124874800941A461946CB
:10B9500005F0CEFF002804DA4FF0FF300DF29C5DB9
:10B9600030BD0023814800941A46194605F0C0FFF7
:10B970000028F1DB00237E4800941A46194605F0A2
:10B98000B7FF0028E8DB00237A4800941A461946DE
:10B9900005F0AEFF0028DFDB0023774800941A464D
:10B9A000194605F0A5FF0028D6DB00237348009454
:10B9B0001A46194605F09CFF0028CDDB002370488D
:10B9C00000941A46194605F093FF0028C4DB6D4B1E
:10B9D00004AA03F1300518685968144603C40833F3
:10B9E000AB422246F7D118681B79206023711521DC
:10B9F00005A80DF0ADFA012300936348352300221A
:10BA000004A905F075FF0028A6DB604B12AA03F11C
:10BA1000380518685968144603C40833AB422246F7
:10BA2000F7D118681B792060237110210DF1670090
:10BA300001240DF08DFA564800943D23002212A9EE
:10BA400005F056FF002887DB524802222146FFF707
:10BA500045FA002880DB504802222146FFF73EFAD3
:10BA60000028FFF679AF4D4802220421FFF736FA8D
:10BA70000028FFF671AF4A4822462146FFF72EFA0A
:10BA80000028FFF669AF474802220421FFF726FA93
:10BA90000028FFF661AF444802220421FFF71EFA96
:10BAA0000028FFF659AF4FF4A262002122A80AF045
:10BAB00033F83E4B3E492293182224A88DF88C403F
:10BAC0000AF04EFA3B4822A906F080FB0028FFF658
:10BAD00043AF38488DF80F4023460DF10F02812106
:10BAE00005F0A6FF0028FFF637AF3349334803239C
:10BAF000082206F0C9FB0028FFF62EAF3048234687
:10BB00000DF10F02812105F093FF0028FFF624AF0D
:10BB10002C492D480323082206F0B6FB0028FFF627
:10BB20001BAF2A4823460DF10F02812105F080FF4B
:10BB30000028FFF611AF0B4909480C7022224A7009
:10BB400005228A705122CA7052220A7153224A7108
:10BB500054228A7107230094002205F0C9FEEFE603
:10BB6000B3520200770C0020BB520200C452020004
:10BB7000CD520200D6520200DF520200E75202000C
:10BB8000EF52020021620200F652020056620200E9
:10BB9000FE520200065302000F5302001853020027
:10BBA000215302002A530200315302000A0102010C
:10BBB00009620200AA520200385302006F000020FE
:10BBC000720000209C5202006400002067000020E8
:10BBD0002DE9F04300230B714B718B716FF06F03F4
:10BBE000CB71037985B005460C464BB1102B02D1C1
:10BBF0004379DB2B04D00023A3716E23E3713AE178
:10BC00006B79B94FDB2B4FF0FF380DD0B74AC02B03
:10BC1000C2F8008012D13B68434540F030816FF09C
:10BC20007A03A3716923E9E7B14BC7F800801B7859
:10BC3000002B40F00F826FF07D03F2E7DB2BC7F89B
:10BC4000008022D8472B00F075820CD8242B00F0FE
:10BC500096812C2B00F0D581202B00F03881002319
:10BC6000A3716D23CAE7A42B3CD0CB2B71D0872BBB
:10BC7000F5D121462846FFF787FB054605F016FD5E
:10BC8000002D80F2F8800023CBE7ED2BE7D9EE3BC7
:10BC9000112BE4D801A252F823F000BF83C20000A8
:10BCA0005FBC00005FBC00005FBC00005FBC000028
:10BCB0005FBC00005FBC00005FBC00005FBC000018
:10BCC00079C2000057C200005FBC00005FBC0000EA
:10BCD000B3C100005FBC000029C200001DC200000B
:10BCE0003FC10000AB79042B01D1ED7915B16FF0A4
:10BCF00079034BE07E4B1D707E4B1D707E4B9D701B
:10BD00007E4B9D70FFF708F923687D4961221A7008
:10BD1000236811225A7023684F269E7023680622DA
:10BD2000DA70206804300AF01BF92368754979221B
:10BD30009A7223680722DA7223681E732368052229
:10BD40005A7320680E300AF00BF9132323716571C2
:10BD500091E0AB793F2BCAD1EB79FF2BC7D1AA89F0
:10BD6000012A01D80023D0E12B6819785C2902D080
:10BD70006FF07F030AE05978881C9042F2D10129C4
:10BD800031D19B787E2B04D06FF07D03A3716A23A1
:10BD900034E722685B491370236812225A702368C3
:10BDA0004F229A7023680B22DA7020680522043033
:10BDB0000AF0D6F820685249062209300AF0D0F875
:10BDC000236851495F22DA7323682F221A7423688B
:10BDD00002225A74206812300AF0C2F81423237128
:10BDE0000023637147E00329CED1052ACCD19A788C
:10BDF0005F2AC9D1DA78C12AC6D11B79092B06D1AD
:10BE00003D4B9B78002B3FF416AF082303E0013B2A
:10BE1000DBB20D2BB8D83D4A52F82390B9F1000F90
:10BE2000B2D0484605F012FE061EFFF62CAFABD08E
:10BE3000AB6821680022484605F026FDB0F10008F5
:10BE4000FFF621AFB6EB0805A4F8048003D1A57175
:10BE50006FF06F03D2E62E48494609F03FFBFF2DF5
:10BE6000C7F8008004DD4FF0FF33A3716123C5E6FE
:10BE700005F5C245E580002005B0BDE8F083DFF898
:10BE8000909099F80030002B3FF4FDAE484605F045
:10BE9000DDFD061EFFF6F7AEAB683A68216848463E
:10BEA00005F0F2FC0028FFF6EEAE3B68A0801844D7
:10BEB0003860301A05D1C7F8008089F80000A071F9
:10BEC000C6E7FF28CFDC00F5C240E080D3E7A979C0
:10BED0004B1EDBB2FD2B7FF60AAFEB79802B19D01E
:10BEE0006FF0770352E700BF800C0020840C002025
:10BEF000920C0020910C00206F00002064000020B4
:10BF0000FE61020004620200FC610200C4610200E2
:10BF1000880C0020FF29AA8907D1002A7FF422AFCC
:10BF2000B24B9A70B24B1A70A5E762B9AF488378EA
:10BF3000002BA0D106F06BFA0028FFF6A4AE00F5A6
:10BF4000C7404030C1E7082A7FF40CAF2968A748F2
:10BF50000DF10F0306F0BCF9411C3FF494AE9DF8BF
:10BF60000F3013B96FF07C035BE6023004D103F5A8
:10BF7000C7434033E3807EE79D4B0022D3E7AB7994
:10BF8000002B7FF4B4AEEB79802B04D0812BA7D1AA
:10BF9000984F994E01E0994F944EAB89102B7FF446
:10BFA000E1AE082229680DF10E03304606F090F943
:10BFB000421C3FF468AE9DF80E30002BD2D0023008
:10BFC000D5D0296808221144304606F0F1F9431C07
:10BFD0003FF459AE03303FF4C5AE28680822394615
:10BFE00010440AF025FCB0FA80F040098DF80F00EB
:10BFF00001230DF10F028121F01C05F019FDC51779
:10C000003EE6AB79002B7FF472AEEB79802B7FF4A8
:10C0100067AFAB89102B7FF4A5AE296876480DF188
:10C020000F03082206F054F9461C3FF42CAE9DF88D
:10C030000F30002B96D0023099D029686B48082227
:10C04000114406F0B5F9411C3FF41DAE03307FF4F6
:10C0500012AF87E6AB793F2B7FF449AEEB79FF2B2C
:10C060007FF445AE664F3B685A1C42D1AE89042E20
:10C070007FF678AE29680B785C2B7FF479AE4B782D
:10C08000032B7FF481AE8B785F2B7FF47DAECB7872
:10C09000C12B7FF479AE0B79013BDBB20D2B3FF660
:10C0A00073AE584A52F82380574A32F81390B8F1C9
:10C0B000000F3FF469AE053E4E453FF753AE0123F6
:10C0C0000093002233460531404605F011FC00285C
:10C0D000FFF6D9AD2B79DB067FF5CDAE4E45BFF629
:10C0E000CAAEA9EB0606414648483E6009F0F6F99B
:10C0F000C1E6464E3278002A3FF4C5ADAA89934284
:10C1000006DA0023C7F800803370A371672375E552
:10C110009B1A29683B60304605F024FC0028FFF696
:10C12000B2AD2B7913F010037FF4A5AEC7F80080F1
:10C130003370A0E621462846FFF736F89DE5AB7937
:10C14000FF2B7FF4D4ADEB79FF2B7FF4D0ADAB891F
:10C150001B2B7FF407AE29680B78032B7FF408AE06
:10C160004B789B2B7FF404AE8E78182E7FF400AEB4
:10C17000274B1B78002B3FF45EAD01272548009725
:10C1800033460022033105F0B3FB0028FFF67BADF8
:10C1900028682149324603300AF04AFBB0FA80F0A1
:10C1A00040098DF80F003B461A480DF10F0281211E
:10C1B00023E7AB79002B7FF49AADEB79002B7FF46A
:10C1C00096ADAB89002B7FF4CDAD084806F01FF982
:10C1D00000283FF730AD084806F019F900283FF76E
:10C1E0002AAD0120FFF79AFB45E600BF6F00002053
:10C1F000910C00209C520200640000203853020081
:10C20000840C0020C4610200A8610200880C002098
:10C21000920C0020AA520200096202002146284620
:10C22000FFF740F805462BE5AB79002B7FF45FADB7
:10C23000EB79002B7FF45BADAB89002B7FF492ADE3
:10C2400022680521117022680421517022689370C0
:10C2500003222271C5E5AB79002B7FF448ADEB7961
:10C26000002B7FF444ADAD89002D7FF47BAD2068B9
:10C27000F6F754FF042369E521462846FEF790FEB1
:10C28000D0E71B4B1B78002B3FF4D5ACAB795A1E83
:10C29000012A3FF62CADEF79002F7FF428AD012B5A
:10C2A0000CD12168134807233A4605F0EDFA00281F
:10C2B000FFF6E9AC072323716771DCE5AE89072E31
:10C2C0007FF450AD29680B78012B3FF651AD012367
:10C2D0000093084833463A4605F00AFB0028FFF66B
:10C2E000D2AC29680448324609F03AFEC3E500BFE3
:10C2F000920C0020B3520200770C00200C4B8222DB
:10C3000081281A7014BF00220722C3F801201122CD
:10C310009A7210221521DA7200221A7359739A73D5
:10C32000FE211A7401221872D9735A72704700BF25
:10C330002412002070B5174A174C0146E379507952
:10C3400003F0030330B143F040030520134AE371C7
:10C35000D37170BD8E0706D5D2F801501DB143F0E0
:10C3600040030120F2E74D0707D5157A567A354389
:10C3700003D043F040030820E8E70907E6D5D07969
:10C38000117A527A084310431CBF43F04003072040
:10C39000DCE700BFCA0C002024120020DC0C0020C7
:10C3A00008B50B20FFF7C6FF38B9044A0449D37912
:10C3B00003F00303CB71D371812008BD2412002048
:10C3C000DC0C0020014B024A1A607047A40C0020CC
:10C3D000E60C00202DE9F041064600200D461446EB
:10C3E00000F0EAFAD8B90020BDE8F081002CFAD1BB
:10C3F000B8F10108F7D00120F6F79EFC214620464F
:10C4000007F0BEFD3B78002BF0D164B106232A462D
:10C41000314600203B7000F0FBFAC0B2E4E7054F64
:10C420004FF03308EEE715F03F0F14BF022303234C
:10C43000EDE700BFC50C002010B50121002007F07A
:10C440009FFD11480021F6F75DFC0346A8B90F498E
:10C450000F484C798979817180220270C2710A215A
:10C46000012243708370C37003714471027243727E
:10C47000FFF7B0FF0448F6F753FCBDE8104005484D
:10C4800040F2DC51F6F7BEBCC00C0020CA0C002004
:10C490003F12002039C40000F8B5424E3378012B1A
:10C4A0000446D8B24BD005286CD008B914B9347002
:10C4B0000020F8BD092CFBD93B4D3C4F0A222946F0
:10C4C00000F094FA3A4A6879A97950719171394A21
:10C4D000D5F8013050710A3CA4B291712A78A34278
:10C4E00038BF9CB26F2A3C8020D1022004F0E8FFC4
:10C4F00060B100243A88D5F801309A4219D3002C53
:10C500002D4B0CBF022201221A70D1E7D5F8013061
:10C51000082B06D8294C3A882146002000F066FAFC
:10C52000E8E7274B1C68002CF5D1E2E7082BF1D98E
:10C53000DFE7002C0CBF052301233370B8E71A494D
:10C540001A4DD1F80120082A84BF1D4B19682B8889
:10C5500003EB040098BF0A318242194407D92246EE
:10C56000002000F043FA2B8823442B80A0E738BF3B
:10C57000D41A2246002000F039FA00233370012239
:10C580000D4BC1E7094A08491388D1F8011023442B
:10C590008B4201D213808BE7002333700222064BBB
:10C5A000B2E700BFC60C0020CA0C0020C80C002057
:10C5B000DC0C002024120020C40C0020D40C00202D
:10C5C000A40C002070B51E4DD5F80130082B88BF93
:10C5D0001C4B4FF001008CBF1E6805F10A06FFF7E7
:10C5E000A9FE0446E8B9D5F801201748174D92B2C4
:10C5F000314604F0A1FD002814DA67232C716C7118
:10C60000AC71EB71AB88124A991CC2F80110E98831
:10C610001344080A9872D9720023D3710D4A8120FD
:10C62000D37170BD0C4840F2DC51F6F7EBFB2946A4
:10C63000054804F06BFE21462046F6F7E3FBE1E7F0
:10C64000CA0C0020A40C0020B00C0020A80C002074
:10C65000DC0C00202412002039C40000084B094AD9
:10C6600000201860084B1870084B1870084B1360B6
:10C67000084A1360012203F8032C074BDA71704754
:10C68000C00C0020B00C0020C60C0020C40C002000
:10C69000E60C0020A80C002024120020F8B5574E0C
:10C6A0003378002B3ED0564F3A78613A00230E2A59
:10C6B00000F2A080DFE802F08A08489E5D9E9E9E00
:10C6C000949E8C858A9E6A004E4C07206370A370EE
:10C6D000E3702371FFF72EFE054650B9FB794A4FF0
:10C6E0000BB3E37903F0030343F04003FB71E37101
:10C6F000072580232370257200236372414CD4F8F0
:10C70000015042480121ADB2F6F7FCFA05F10A01E9
:10C71000002289B22046FFF75DFE3C48F6F700FB99
:10C7200000233370F8BD04F003FF3949112204F1EE
:10C730000A0009F015FC1123A570E5702571FD7143
:10C74000E57163708125D4E70B20FFF7F3FD2D4CD5
:10C7500030B904F0EDFE2C4A0123D371E37181203E
:10C760008123237000236370A370E3702371207210
:10C77000C3E7FFF715FE234B81221A7000225A707F
:10C780009A70DA701A7118725A72B7E73378022BFE
:10C79000D9B20DD11B4B59706421997280210022AE
:10C7A000197081219A70DA701A71DA721972EBE7D6
:10C7B000FFF708FF144C8022227000222072627260
:10C7C0009DE7FFF7EDFDFFF799FD97E70020FAE7FA
:10C7D0000C4A8321117053709370D370137106E06B
:10C7E000084A802153709370D370137111701372C3
:10C7F000537283E7034A8121ECE700BFC40C002099
:10C80000CA0C002024120020DC0C0020C00C0020E8
:10C810009362020010B9022004F062BE704708B5AE
:10C8200028B900F0D7F8BDE80840FFF735BE08BDCD
:10C8300010B50B4C2378032B08D102230022237060
:10C84000BDE810401146104600F0E2B82078831F82
:10C8500058425841FFF7DEFF0023237010BD00BF90
:10C86000C50C00200120704710B5054C042220465D
:10C87000002109F051F9201DBDE8104007F044B92E
:10C880004C12002013B5084C90220021204609F0DC
:10C8900043F9002300934022012304F11001201DDD
:10C8A00007F09AF802B010BD4C120020F7B51346FD
:10C8B0004A790B2A06460AD18A7942B9CA7932B92D
:10C8C0000A79C2EBC2043F34A4B29C4203D90024CB
:10C8D000204603B0F0BD174D6F78AB78002FF6D12E
:10C8E000002BF4D18B782B700B78CF1897F801C000
:10C8F000BCF1210F09D1C95C6B1C0193AB1C0093E7
:10C900003944022307F07CFA38B94FF0E023D3F81A
:10C91000F03DDB07DBD500BED9E7A9780029D7D0E9
:10C92000402305F15002304607F0A6FA0028CFD187
:10C93000EBE700BF4C12002070B504468178002060
:10C9400007F0C6FA054668B9201D07F07AF83F28B7
:10C9500008D9A17804F1500228464023BDE8704070
:10C9600007F08ABA70BD000010B5124C0A4619468D
:10C97000A37893420DD18AB2201D04F1500107F033
:10C98000BDF80020FFF74BFF2046FFF7D5FF012041
:10C990000AE06378934208D04FF0E023D3F8F03DEB
:10C9A000DB0700D500BE002010BD0020FFF740FFD0
:10C9B000EDE700BF4C120020054B902202FB003334
:10C9C000587818B19878003818BF0120704700BF18
:10C9D0004C12002008B59022042302FB00330248C9
:10C9E000184407F00CF808BD4C12002000EBC00002
:10C9F00070B5064E0401201D92B2304407F045F890
:10CA000005463019FFF798FF284670BD4C120020EC
:10CA10002DE9F04180460F46144607F0E5F8C8B10D
:10CA200007F0EAF80546A8B90C4E902303FB086608
:10CA3000717807F013FA68B17178A3B23A462846C4
:10CA400007F01AFA38B94FF0E023D3F8F03DDB07CE
:10CA500000D500BE00242046BDE8F0814C12002025
:10CA60000123037000487047A4620200024B034890
:10CA70001B684021184700BFDC1200201C18002052
:10CA800070B5094C06460D4620464022002109F0AB
:10CA900043F8BF23A38001232660A371E571BDE89D
:10CAA0007040FFF7E3BF00BF1C1800202DE9F84FCE
:10CAB0001F4CDFF88090164607460D4640220021A5
:10CAC000204609F029F865F07F05392E2571354695
:10CAD00028BF3925330A174963712A46E01D2760AC
:10CAE000A67109F03DFAFFF7C1FF4FF0000B04F10A
:10CAF000040804F1050AAE425FFA8BF70BF1010B53
:10CB000001D8BDE8F88F3C220021404609F004F826
:10CB10002771771B3B2FA8BF3B2709EB05013A463E
:10CB200050463D4409F01CFAADB2FFF79FFFE2E723
:10CB30001C180020081300202DE9F04104460D4682
:10CB400007F052F8B0B9BDE8F081013EFBD00021FA
:10CB5000084607F015FA0120F6F7EEF839780029B3
:10CB6000F3D101233B7022462B460846BDE8F04135
:10CB700006F0A0BA014F3326F0E700BFE012002014
:10CB800038B5094C054640222046002108F0C4FF74
:10CB9000064BE5711B682360BB23A3800123A371AF
:10CBA000BDE83840FFF762BF1C180020F8120020D3
:10CBB000044B054A186000231373044A1370044A97
:10CBC00013707047DC120020F8120020E0120020E1
:10CBD000F7120020F7B57D4C237B012B05460AD1C7
:10CBE000F6F7A4F8A368984205D9002320682373B8
:10CBF0000521FFF745FF764E337803F0FF006BB158
:10CC0000744B186820B1421C0AD11A79862A07D0C1
:10CC10000B21FFF735FF00200023337003B0F0BD78
:10CC2000227B012A04D12168884201D00621F0E745
:10CC300093F9047019792060002F3FDA35B9012A81
:10CC400004D1862902D025730421E2E75F799A791D
:10CC500002EB072292B240F214539A42A28001D909
:10CC60000321D6E7392A4FF0010328BF3922237365
:10CC70006173002358495948E280A37309F070F9A1
:10CC8000F6F754F800F54870A0600023A1883370CF
:10CC9000E3888B42BFD14FF0FF33A360637B813BBE
:10CCA000102B00F28E80DFE803F0818C238C8C65E2
:10CCB0008C878C8C8C8C8C8C8C508E00002AAAD00B
:10CCC000A37B5A1C9942A27302D000232373BBE7B3
:10CCD000E388A78841484249FF1A3B2FA8BF3B275A
:10CCE000BAB2184409F03CF9E3881F44E780CCE766
:10CCF00015B10621206840E0032901D80321F9E796
:10CD00003848237C0371637C4371A37C8371E37C8B
:10CD1000C371B4F8153005725BBA83814572324B2A
:10CD2000C572324D03600122073B294682722B6097
:10CD3000FAF746FCAA88E988A318080A0232187490
:10CD4000597492B2617B206811E0002DD1D1002985
:10CD5000D4D0224D40F2145301932A4601AB284609
:10CD6000FAF73CF9BDF8042055F8100C9021FFF7B4
:10CD70009DFE04E0206835B10621FFF781FE00200A
:10CD80000023237348E7431C0ED104210DEB01005F
:10CD90000CF0DEF8019BA3614FF48173E36104237F
:10CDA00084F820301122CDE70190F3E72068002DB0
:10CDB000E2D10A468121DAE70DB9FAF743FC0022F5
:10CDC000C0E7012196E70120DAE700BFF812002052
:10CDD000F71200201C180020231800200813002040
:10CDE00021180020E91200200F130020E11200207A
:10CDF000014B00221A707047E0120020002070479B
:10CE000010B50C46204311460AD1064C22783AB997
:10CE10003F2B05D90448402209F0A2F801232370D2
:10CE200010BD00BFF71200201C1800200346084662
:10CE300013B9D1B2FFF7DCBF012B02D1D1B200F0A0
:10CE4000DFB8704710B40446084611461A46BDF8CC
:10CE500004301CB95DF8044BFFF7D0BF012C03D19F
:10CE60005DF8044B00F0CDB800205DF8044B70472E
:10CE700010B40446084611461A46BDF804301CB9E1
:10CE80005DF8044BFFF7BCBF012C03D15DF8044BE8
:10CE900000F0B9B85DF8044B70470000054A032361
:10CEA000137000235370044A1370044B01221A704C
:10CEB000704700BF64180020631800208618002007
:10CEC000024A00231370024A13707047861800202C
:10CED00063180020F8B5444C2578ADB904F08EFBFA
:10CEE00090B104F0A9FBE0B1404E3146FDF7B6FF2A
:10CEF000002816DD3E4B35541D7001232370284653
:10CF0000BDE8F84004F09EBB2578022D4FD005F017
:10CF1000FD05012D05D1364F344E3B78F35C0BB93E
:10CF20002370F8BD284606F0A9F80028F9D03B7810
:10CF30003049F35C304A032B0CD100230B70B8232B
:10CF4000137002252B4B12782946012006F0ECF8CD
:10CF50000223E5E7A3F1310008280DD8133BDBB22B
:10CF600018060B7045BF022003F07F0300231070EA
:10CF70004CBF0B701370E5E7302B14D0A3F16100A8
:10CF8000192801D85D3BEAE7A3F14100192803D82D
:10CF90003D3B63F07F03E2E70D3BDBB2712B04D82E
:10CFA0001648C35CDCE72723DAE70023D8E7012033
:10CFB00006F064F80028B4D00D4E0C4831780E4BC2
:10CFC000415C002203291A7018BF0121094B06BFDA
:10CFD0002946012008461A7006F0A6F83378013376
:10CFE000337003239CE700BF8618002064180020DC
:10CFF000631800205D1800205C180020BC6202004D
:10D000007047002070477047064BFF221A70064B8E
:10D01000064A1B681360064A1360064B00221A601A
:10D02000704700BFA4180020A40C00209418002012
:10D030008C18002088180020F8B5F5F777FE1C4BF7
:10D040001C4D1B68C01AB0F5FA6F09D995F900306C
:10D05000042B05D1032004F043FAFF232B70F8BD05
:10D0600095F90030012BFAD1134F144E3A883168EC
:10D070001348144C04F060F8002813DA00232371DD
:10D080006371A3716723E371A2883168931C3B80AD
:10D09000E3881B0A8B54A28833681344E2885A70D1
:10D0A0000023DBE70648214604F030F9ECE700BF37
:10D0B00088180020A4180020A2180020A40C00202A
:10D0C000941800208C180020084B93F90020022AA5
:10D0D00007D0032A03D1032901D101221A700120AC
:10D0E00070470329FBD10422F8E700BFA4180020F1
:10D0F00037B54A78012A05460C4603D0022A08D0E3
:10D10000002015E00B4A137803B0BDE8304007F06B
:10D110003BBA8B88072BF3D107490DF1060008F0C5
:10D120001FFFBDF80630054A2146284607F02CFAB5
:10D1300003B030BD30630200506302004863020058
:10D1400070B50C460546F5F7F1FD244B1860637881
:10D15000012B28D0022B39D00BB1002070BD204EFE
:10D1600096F900305A1C01D0042BF6D1032004F0AC
:10D17000A7F90028F1D104233370E38840F23C5230
:10D180009342EAD86BB1174A21461268284607F045
:10D19000FBF9E279A37943EA0223134A13800323BC
:10D1A00033700120DAE70E4E96F90030002BD4D10F
:10D1B0000D4BE2881B88934228BF1346094A21463B
:10D1C0001268284607F0E0F90223E9E7044A012340
:10D1D0002146284607F0D8F9E3E700BF8818002069
:10D1E000A4180020A40C0020A21800200129134636
:10D1F00001D0FFF769BF127802F06001402904D125
:10D2000012F01F0203D0012A04D0002070471946F3
:10D21000FFF76EBF1946FFF793BFF0B59DF81450A6
:10D220009DF81860884200D3F0BD4478042C04D0E7
:10D23000052C04D004782044F4E78270FAE787785C
:10D240000671FF2F14BF2C461C468470F2E70000C5
:10D25000004870474965020020B10128024818BF04
:10D260000020704701487047CB6402002765020028
:10D270002DE9F347334CDFF8F0803349334E04F1A6
:10D2800009050922204608F06BFE31492022284674
:10D2900008F066FE98F801304FF0400ACDE9003AF8
:10D2A00004F12907327843F0800339462846FFF716
:10D2B000B4FF002527490922384608F051FECDE980
:10D2C000005504F132092B46727849463846FFF77B
:10D2D000A4FF21490922484608F042FE1F49362290
:10D2E00004F13B0008F03CFE1D490E2204F17100E0
:10D2F00008F036FE98F80030CDE9003A04F17F07D7
:10D30000B27843F0800339464846FFF786FF154957
:10D310001922384608F024FE98F802300822CDE998
:10D3200000323846F27843F0800304F19801FFF7A9
:10D3300074FF0423237120469823A370E57002B084
:10D34000BDE8F0871F19002033640200BA190020DD
:10D35000AB640200896402004A6402005364020064
:10D360003C64020092640200B719002010B5054C1D
:10D3700005493922204608F0F3FDF5F781FE2077B4
:10D38000204610BDE6180020FA63020030B50328DD
:10D3900087B018D81D4B53F820401CD0204608F009
:10D3A0004FFBC0B21A4B1F2828BF1F2021181A4656
:10D3B0008C4223D10130C0B2400040F44070108054
:10D3C000134807B030BD1038C3B2032B1BD8114B24
:10D3D00053F82040E2E702A8F5F7A0FE9DF80B30D5
:10D3E00001939DF80A3000939DF808209DF80930BC
:10D3F000094903A807F0AAFF03ACCFE714F8015BC3
:10D4000023F8025FD4E70020DBE700BF9000002094
:10D41000A6180020800000204153020008B507F044
:10D420000BFFF5F7FDFD08BD04F0C8B87047704765
:10D4300070470368013304D04068431C5842584188
:10D4400070470120704710B504680B689C4209D0F2
:10D4500040684968884205D08C4203D0181A18BF2A
:10D46000012010BD0020FCE710B5D1E900320468AE
:10D470009C4202D14168914206D0944206D1406854
:10D48000C31A5842584110BD0120FCE70020FAE7BA
:10D4900040F30903B3F1FF3F08BF0130C0F30900B7
:10D4A0000430704710B5031F0439083053F8042FB7
:10D4B00051F8044F834282EA04021A60F6D110BD8B
:10D4C0000346006830B95A682AB99868B0FA80F003
:10D4D000400970470020704708B503681B0D0246DD
:10D4E00013F4E06005D0101DFFF7ADFFB0FA80F037
:10D4F000400908BD00B97047884201D00068F9E7CB
:10D500000120704710B5C36E426D1944891AB1FBF2
:10D51000F3F203FB1211836D8B420AD94C09406E62
:10D5200001F01F0150F8243001228A40134340F8D3
:10D530002430002010BD000030B5184A0368184C94
:10D5400011F0805F18BF144683EA010525420DD013
:10D5500043F30904013409D001EA0204114A1A40D4
:10D5600042F09F4242F4E002944203D10023036060
:10D57000012030BD0A0D02F4E064B4F5806F05D1DE
:10D58000C3F38924C1F389218C4201D20020F0E742
:10D5900052B203EB82230360F8E700BF00FCFF7F79
:10D5A00000FC0F7000FC0F00024608B50846FFF7AC
:10D5B0006FFF136803441360002008BD0368013344
:10D5C000036000207047000008B5036BC3F3090235
:10D5D00042B9002910DA0F4B0F4A41F294210F484B
:10D5E00007F056FFB2F5FF7F06D9002904DD0C4B8A
:10D5F000094A41F29521F2E71944C1F30903003BBE
:10D6000018BF012321F0004141EAC37101630020EA
:10D6100008BD00BF9253020052660200C8530200C8
:10D62000FD5302002DE9F04F87B0DDE91149049365
:10D63000836E139EDB690292A2199A4280468A4643
:10D640000AD8C36E2BB9049B013B05933EB9304603
:10D65000B3E0109A9342F6D86FF05300ADE0BAF100
:10D66000000F3FD0DAF80030109A93423AD1DAE94D
:10D67000015305EB030BA34534D9A54211D8ABEBFD
:10D68000040BB345DAF80C1028BFB346651B4846B7
:10D690005A46294408F064FCD9445C44A6EB0B06C6
:10D6A000D4E72D1BB54228BF3546029B109A1B6854
:10D6B00093421DD1029BD3E901130B44A34217D916
:10D6C000A14211D81B1B9D4228BF1D46029BDB684F
:10D6D000611A48462A46194408F042FCA9442C44E1
:10D6E000761BB3E73546E0E7091B8D4228BF0D46A0
:10D6F000049B9E4220D3D8F868004369B4FBF3F240
:10D7000003FB1242C2B9B34216D8B5FBF3F203FBD6
:10D710001253A5EB030BCDF800B0039343681099A7
:10D720001F4622464B46B847002846D1039B5B1B49
:10D73000D9445C441E4489E7D8F86C3043B1109A50
:10D74000934205D81E4B1F4A6B211F4807F0A0FECD
:10D75000029A109B1360D8F8683002995A69B4FB9A
:10D76000F2F302FB1343E21A4A60D8F868500599B5
:10D77000D5F814C001EB0C002044B0FBFCF10CFB0D
:10D780001101401AE9691B1B884294BF1B185B18E2
:10D79000A96A8B4228BF0B4602998B60D8F86800B3
:10D7A0000093CB6845681099A847002803DD074B14
:10D7B000044A7621C9E73FF449AF07B0BDE8F08FCE
:10D7C00033540200A3660200C853020061540200F1
:10D7D0002DE9F04F9A46D1E9038387B006463C30E5
:10D7E00091460F460593FFF777FEC9F3892B044650
:10D7F00058B1BBF1000F78D0F36B3D4CC3F38922D5
:10D80000CAF389239A4288BF0024059D2846FFF762
:10D810003FFE031D434534D80423A8EB00080393BF
:10D8200005ABCDE901833B68009332460423002118
:10D830003046FFF7F7FE30BB059B1BBA6B4023F069
:10D8400000430593BBF1000F23D02A0D02F4E063DF
:10D85000B3F5806F1DD1AAEB0403C3F38920C5F390
:10D860008921884215D323F07F4323F4700323F4E6
:10D870007F7323F0030343F0804343F48013AB42F0
:10D8800004D16FF0010007B0BDE8F08F52B204EB95
:10D890008224AAEB0401694011EA0901B5D145F3DC
:10D8A00009030133EDD0129BC5F30909994528BF3F
:10D8B0009946119B0293109BCDF80C90043343447E
:10D8C00001933B68009332464B463046FFF7AAFE71
:10D8D0000028D8D1129BA3EB0902119B014603EB50
:10D8E000090008F019F96019CDE75C468DE700BF23
:10D8F00000FCFFFF1FB5C3F309040294069C0194CA
:10D9000000240094FFF764FF04B010BD30B587B069
:10D9100003AD094B00951446084AFFF7EBFF0028BA
:10D9200004DA831C00D1002007B030BD2946204610
:10D93000FFF7B8FDF7E700BF0C00F07F0000F07FB5
:10D9400030B5134687B00268044604AD0820916ED6
:10D9500003900295586801901B680093CB691046AC
:10D9600002F11001FFF75EFE30B9211D2846FFF7D6
:10D970006AFD003818BF012007B030BD10B5836EB6
:10D980001B6B044613B9C06808F08CFBA36E5B6B7D
:10D9900013B9E06908F086FBA36E9B6B13B9606E48
:10D9A00008F080FB002010BD08B5C36E8B4206D87E
:10D9B000084B094A4FF48A71084807F069FD806EE8
:10D9C000C3689847002804DD054B034A4FF48B7168
:10D9D000F2E708BD475702007E660200C853020006
:10D9E000615402002DE9F04F0024ABB0CDE90A44A8
:10D9F0000493BDF8DCB0BDF8E030BDF9E4A00690BA
:10DA000089460593A0460498FFF742FDD9F80C30EB
:10DA100087189F4235D20423039309ABCDE90173E4
:10DA2000069AD9F800300093002104231046FFF72E
:10DA3000F9FD002840F02081099B049A1BBA5A4046
:10DA400042F0004309930493D9F800300A933B1D38
:10DA50000B930AAE0999369B81EA08021A40884B5B
:10DA60001A4054D1369BC3F38923002B00F0AA80BF
:10DA7000022C16D9834B844A844840F29F3107F028
:10DA800007FD359B002B40F3F580349B1B68099301
:10DA9000349B5E6808333493359B013B35931746BE
:10DAA000D8E73C25654305F1A8036B44049843F887
:10DAB000700C349843F86C0C359843F8680C369821
:10DAC00023F85CBC43E91908059823F85A0C3A98E6
:10DAD00043F8540C3B9823F858AC43E91401DDE9B2
:10DAE0000A0143F8486C43E91E97443B83E803006E
:10DAF00005F1A8030DEB0305A5F14C033B93644B23
:10DB00003692013490463A939246059293463A46AD
:10DB100079E7B2F5817F1CD10025099BC3F3090287
:10DB20009542F4D2B1687268C3F38923534441EA41
:10DB30008321337803F5407341EA0351DDE93A303C
:10DB400098470028C0F2988006F10C06DFD1013515
:10DB5000E3E703EB8A213246DDE93A3098470028B3
:10DB6000C0F28A80D3D0002C00F086802AAA013C23
:10DB70003C2303FB042353E9110153F8702C049256
:10DB800053F86C2C349253F8682C359253F8642C6B
:10DB9000369233F85A2C059253F8542C3A9253F893
:10DBA000502C3B9253F84C2C09920AAA53E91E9729
:10DBB00082E8030053F8608C33F85CBC33F958AC4E
:10DBC00053F8486C369A099BC2F3892232B1C3F3E9
:10DBD00089225A459BD305998A4298D2C3F30A52A7
:10DBE000002A94D040F201118A4292D1284A079328
:10DBF0003A9B93428BD03C222AAB02FB0435002196
:10DC0000A5F1780007F088FF049B45F8703C349B31
:10DC100045F86C3C359B45F8683C369B25F85CBC68
:10DC200045E91938059B25F85A3C3A9B45F8543C80
:10DC30003B9B45F8503C079B25F858ACC3F3090BB8
:10DC4000C3F389230BF10102A3EB0B0353440592A9
:10DC5000104A0FFA83FA0023CDE9353234934FF09E
:10DC6000FF3345E91E970134B1464FF00058049345
:10DC700000274CE7002076E72BB0BDE8F08F00BF0F
:10DC80000000F07F6C54020028660200C8530200B6
:10DC900039D5000000FC0F602DE9F04F87B0154624
:10DCA000826E119C139ED2698946A1199142074642
:10DCB0004FD8DFF8A4B06FF0010A03F1FF380EB9B6
:10DCC000304643E02B68E868023318D1D5E90112E9
:10DCD0000A44944213D28C4211D3121BB242A4EBD9
:10DCE000010128BF324601441298059208F038F924
:10DCF000059A129B134412931444B61ADFE7C5F831
:10DD000000A0BB6E5B69B4FBF3F203FB1242A21AE4
:10DD10006A60D7F868C0DCF814E008EB0E0323440F
:10DD2000B3FBFEF10EFB11315B1ADCF828108B42BD
:10DD300028BF0B46AB604946CDE901030092109B1A
:10DD40005A463846FFF744FD0028B8DA07B0BDE868
:10DD5000F08F6FF05300F9E700FCF7FF2DE9F04F6B
:10DD600087B00646119F884691469A4600240DF1D9
:10DD7000100BA74203D8002007B0BDE8F08F3D1B71
:10DD8000109B082D28BF0825E318CDE900A3CDE995
:10DD900002B5A9EB0403424600213046FFF742FCDE
:10DDA0000028E9D1129B2A461868594603F0A8F9C1
:10DDB000129B2C441860DCE72DE9F04F97B0164613
:10DDC0000A93C36E126807460D4633B1934240F280
:10DDD000B58071688B4240F2B18000214FF0040899
:10DDE0000EABCDE901130092CDF80C8043463A46C4
:10DDF0003846CDE90E11FFF715FC044610B110F1BD
:10DE0000540F5BD1CDF80C800FAB4FF0000802939C
:10DE1000CDF80480736800933A460423414638469F
:10DE2000FFF700FC0F9B044600284BD010F1540F65
:10DE300044D1414656F821302B6081F0010307930D
:10DE400056F823306B6016AB03EB81014FF0FF34C3
:10DE500051F8203CAB600023EB6002230893AA4AF0
:10DE600092E8030010AB83E80300042205F10801E7
:10DE70004FF0FF3003F044F900230C90A1460693C5
:10DE8000099305934FF0FF389B464046FFF700FB90
:10DE90000422BB6E039283440DAACDE901B22A6825
:10DEA0000092DB693A4600213846FFF7BBFB064685
:10DEB00090B116F1540F00F025813446204617B07A
:10DEC000BDE8F08F0E9A9B1A002BD4BF00210121D0
:10DED000B0E701230893C2E70C9804220DA903F0D0
:10DEE0000FF90D9B0C901BBA88EA030ABAF1000FD8
:10DEF000CDF834A025DA4FEA185303F4F063A3F504
:10DF0000A06673427341EA68002A40F009810799CC
:10DF100016A800EB8101D5E9002351F8201CA96067
:10DF200008990129C5E90032D3D178497848CDE96B
:10DF30000021784940F2425208F0B8FC6FF05304D7
:10DF4000BCE75046FFF7A4FABB6EDA6900EB0B039F
:10DF5000934200F2D7804FEA1A5101F4F061B1F513
:10DF6000A06F2B680BF1040833D10421039114A98D
:10DF7000CDE9018100933146134638463A46FFF712
:10DF800051FB0646002894D1149A0C9B9A4240F00B
:10DF9000B9800D9BF86A1B0D04220CA98AEAC37A8A
:10DFA00003F0AEF8F8620D98FFF772FA059BAB82AA
:10DFB000109BAB615844119BEB61C5E9030A099BB7
:10DFC000EB754FF0FF330C934B464C46D0469946C9
:10DFD0005BE70CA90438CDE9008002913846394648
:10DFE000FFF7BCFE064600287FF463AF0D9B286850
:10DFF000190D11F4E06C1CD1059AC3F389239A42E0
:10E0000001D8013305930D99209B0A982A684B404B
:10E0100003400B9360D1CDE91428DDE9223014AA26
:10E020009847061E0B9B54DA16F1540F3FF46BAF62
:10E0300043E7BCF5806F1DD1059A48B242FA81F1E1
:10E040008AB20592344A09EA020242F09F4242F43F
:10E05000E002934202D149F00049D4E7B9F1FF3F11
:10E06000D1D0C3F38923C9F389229342CBD809EBDA
:10E070008029C8E7BCF5C06F13D101F00103082265
:10E080000993BB6E039210AACDE90182009031463C
:10E09000DB693A463846FFF7C5FA06460028B2D093
:10E0A00007E7C1F30A0240F2FF539A42ABD10822BC
:10E0B000BB6E039212AACDE901820090DB693A4659
:10E0C00031463846FFF7AEFA54301BD00123069391
:10E0D00099E70D9B03D199464B46A14675E70F4A38
:10E0E00089EA03010A4052B1022EF5D1C9F389220F
:10E0F000C3F389218A42EFD343F00049ECE74FF0A4
:10E10000FF39E9E70023FEE6C86602003852020044
:10E1100073540200C853020000FC0F0000FCFF7F94
:10E120000021A97513B3B96E8869B2FBF0F300FB47
:10E130001323DBB9069BCBB14FF0FF33149314AB21
:10E140000293129BCDE900233846CA692B683946F1
:10E15000FFF704FE20B110F1540F01D00446ADE6E4
:10E16000DDE91332981A43424341AB75294607F162
:10E170003C00FFF7B1F988B1FB6BC4F38922C3F30C
:10E1800089239A4204D144F00044219B43B912E010
:10E19000611CFAD09A4288BFA4F58064219B3BB1F0
:10E1A000AA8AC4F38923934228BF1346219A138075
:10E1B000002CBFF683AEAB8AC4F38924A34294BF7C
:10E1C00000246FF0010479E62DE9F04F00230125CA
:10E1D000C2E90635244BDFF8A8B00746884693E825
:10E1E00003008BB00DF1140A8AE8030014462E4692
:10E1F00004F118094846FFF71CF910B16FF001004F
:10E200000DE051464846FFF72FF958B1174B184912
:10E21000184841F2732208F049FB6FF053000BB02D
:10E22000BDE8F08FAE4205D1A3690593E36906937B
:10E2300075000646D8F800300893D8F804300993E2
:10E2400007AB03930C4B02930023CDE900B34A467E
:10E250000A4B0797214638460136FFF7ADFD0028E7
:10E26000C6D0831CC4D0DAE7C86602003852020068
:10E27000C8530200A854020041D90000FF03F07FF8
:10E28000080000201FB50023CDE9023301934FF0B1
:10E29000FF330093FFF790FD05B05DF804FB00002D
:10E2A0002DE9F34700230124C2E906341E4B07463B
:10E2B000884693E80300E94689E80300924625462C
:10E2C00002F118063046FFF7B4F810B16FF0010004
:10E2D0000DE049463046FFF7C7F858B1134B1449D3
:10E2E000144841F2322208F0E1FA6FF0530002B014
:10E2F000BDE8F087A54207D1DAF818300093DAF8C4
:10E300001C3001936C000546414630460135FFF74D
:10E310009AF80028EBD0324651463846FFF7B2FF54
:10E320000028CFD0E3E700BFC866020038520200E1
:10E33000C8530200A85402002DE9F04F8DB01668B2
:10E3400006928146884605931BB1059A40F2FF3339
:10E350001380D9F82030C8F81830D9F82430434C4D
:10E36000C8F81C304249304607F07AF83518404961
:10E37000284607F011FB0128074605EB000623D1CC
:10E380003C490246284608F053FA0028EAD0B24633
:10E390004FF0010B3649504607F062F88244344989
:10E3A000504607F0F9FA0246B8B1022811D1079099
:10E3B0003149504608F03CFA079A50B9BBF1010BBD
:10E3C00009D10AF10206CDE70228E0D12A49024626
:10E3D000D8E70BF1010B9244DCE72B78002B3DD002
:10E3E000069B1D60C4F30A53022B3BD1C4F389245E
:10E3F00040F2FF339C4208F1180A23D10DF1240B9F
:10E400002F21284606F0C4FF059B1C4ACDF80CB00E
:10E41000002818BF0023CDE9013200974FF0F043E8
:10E42000524641464846CDE909950B97FFF7C4FC93
:10E43000041E13DB96D198F81730002BE0D16FF053
:10E4400001040BE00E4B0F4ACDF800A043EA8423F1
:10E4500041464846FFF74EFA041ECFDA20460DB07B
:10E46000BDE8F08F6FF01304F8E700BF00FC2F0049
:10E470006A540200D4540200D3540200EDE40000B8
:10E480000800002000FC0F702DE9F04F87B0074610
:10E49000129E884691469A4600240DF1100BA64222
:10E4A00001D800201BE0351B109B082D28BF082534
:10E4B000E318CDE900A3CDE902B5A9EB0403424678
:10E4C00000213846FFF7AEF848B9119B2A461919C2
:10E4D000584608F0ADF9002804D005DA012007B04D
:10E4E000BDE8F08F2C44DAE70220F8E730B5134698
:10E4F0008268C1F3090585B0AA4228BF2A46029264
:10E50000416801915968009101681B6804460846FA
:10E51000FFF7BAFF28B9A368AB4202D034BF01208D
:10E52000022005B030BDF8B5C6690D68083EB54299
:10E530000F4613D3B5FBF6F0013816F07BFB841CB5
:10E54000A5EB8404B4FBF6F4204616F073FBA5EBB0
:10E55000800504FB16553D602046F8BD0020FCE711
:10E560002DE9F04F89B00646DDF84C8005920F4644
:10E570004BB94FF0FF32C8F80020149A0020136006
:10E5800009B0BDE8F08F846E013B07A920460793D0
:10E59000FFF7C9FF12A905462046FFF7C4FF4FF059
:10E5A000040A81460DF1140BA945059A03D3129B69
:10E5B000C8F80020E1E7A5EB0904B4FA84F495FA61
:10E5C000A5F3B3FA83F3C4F11F049C4228BF1C4691
:10E5D000A300CDE90023CDE902BA04233A46002185
:10E5E0003046FFF71FF80028CAD10123A340ED1AD7
:10E5F000DAE700002DE9F04F9046CE6A4A6BB2424E
:10E6000085B007460C465CD2B61A9E4228BF1E460D
:10E61000DFF8B4B0B14601F1400AB9F1000F01D101
:10E62000304618E0226B510304D5BB6EE16BDB6909
:10E6300099421BD1D202636B10D404F13C020292C6
:10E6400004F13802CDE900325146D4E90A233846B4
:10E65000FFF786FF30B105B0BDE8F08F6FF0010223
:10E66000C4E90E23236B43F480232363BB6EE26B68
:10E67000DB69216B01929D1A4D4528BF4D4611F46F
:10E680008011CDE9028515D0A2884BEA8222009242
:10E6900004F1080152463846FFF7FEFA0028DAD1A5
:10E6A000636B2B446363E36B2B44E363A844A9EBE4
:10E6B0000509B2E7A26B009238465246FEF7B2FF58
:10E6C000ECE70020C7E700BF000010202DE9F04F65
:10E6D00089B00646DDE9120A0F4690461D4688B30A
:10E6E0000138059005A9B06EFFF71DFF0DF1180B5D
:10E6F000044614982946D04720BB1CB304F00109F6
:10E70000C9F102039B00CDE90050CDE902B34246B6
:10E7100039463046FEF786FFA0B9E54305F001050E
:10E72000A84207DB08AB03EB8505023C55F8085C03
:10E730004C44DEE706991498D04703460120002B8D
:10E74000EED0184609B0BDE8F08F00002DE9F04F7B
:10E7500093B004460D46164600211C220AA80593D4
:10E7600007F0DAF9554B93E803000DF1180A8AE82F
:10E77000030001271197B84640F2022B10A8FEF7BC
:10E7800058FE20B1A76A002F6AD138460DE05146E5
:10E7900010A8FEF769FE58B1494B4A494A4841F270
:10E7A000D41208F083F86FF0530013B0BDE8F08F77
:10E7B000B845109905D1119B06914FEA4807079378
:10E7C0008046304608F10108A8470028EDD111998C
:10E7D0003046A8470028E8D110AA0AA92046FFF72A
:10E7E00051FD0028E1D18146BDF83C201FFA89F394
:10E7F0009A42C3D9354B03EA892308AA43F0005350
:10E80000009243F00803324A0AA92046FFF772F843
:10E81000002804DA831CC8D109F10109E4E7BBEB45
:10E82000105F4FEA10530CD1099B0093CDE90156BC
:10E83000089B224600212046FFF748FF0028EBD026
:10E84000B3E7059A002AE7D0B3F5007FE4D1089931
:10E850003046A8470028A8D109993046A847EDE7D7
:10E86000BB79012B01D03F688DE73B6B03F4881324
:10E87000B3F5803F13D03B6B03F49013B3F5003F27
:10E88000F1D1CDE901567B6B0093BB6B224607F1BA
:10E8900040012046FFF71AFF0028E4D085E7CDE9C4
:10E8A0000156FB6A0093BB6A224607F140012046ED
:10E8B000FFF70CFF0028DED077E700BFC866020034
:10E8C00038520200C8530200A854020000FCFF03A3
:10E8D00000FC0F7038B5C26D436D1344C26EB3FBBC
:10E8E000F2F102FB1133826E4365D36A016EDB00E5
:10E8F00000258B4294BF83658165C5650446D26A55
:10E90000406E294607F008F90549012322462046B2
:10E91000FFF71CFF18B1C4E91655E36E236638BD36
:10E9200005D50000F7B504460D460126A36DD4E9D0
:10E9300017209A420ED1002839D1626D20490091EA
:10E940001344204920484FF4287207F0AFFF6FF0BE
:10E950001B0024E00138511C2066676EE1655009F8
:10E9600002F01F0157F8200006FA01F10142DED142
:10E97000636D1344E26EB3FBF2F102FB11332B60C3
:10E98000A66D0125E36DB34217D0616E5A0903F0FD
:10E990001F0051F8222005FA00F0104001D103B009
:10E9A000F0BD0133E365236E013B2366EAE72046B1
:10E9B000FFF790FF0028B9D0F1E70020EFE700BF94
:10E9C00038520200C8530200D65402007FB50C46EC
:10E9D00004310646FFF7A6FF054680BB21463046B8
:10E9E000FFF7A0FF054650BB2246042342F8080F5C
:10E9F000CDE902230190226800920146324630465A
:10EA0000FEF710FE10B110F1540F1BD1B36E5A6A0D
:10EA1000002A0BDDA368013242F00102013B1344DE
:10EA2000B3FBF2F102FB11329B1AA3604FF0FF33EC
:10EA30000422C4E903230022C4E90523E361284634
:10EA400004B070BD0546FAE707B5002304490193F9
:10EA500001AAFFF77BFE00B9019803B05DF804FB43
:10EA6000BDD5000010B50C46826AE068FF2107F0B2
:10EA700053F84FF0FF33236010BD000038B58166B6
:10EA80000B6AC3664D69044635B95F4B5F4A41F274
:10EA900025015F4806F0FCFC8A6922B95D4B5B4AA0
:10EAA00041F22601F5E7886A20B95B4B574A41F2EB
:10EAB0002701EEE7B0FBF5F305FB130323B1574B3A
:10EAC000524A41F22B01E4E7B0FBF2F302FB1303DD
:10EAD00023B1534B4D4A41F22C01DAE7CB69B3FB2A
:10EAE000F0F200FB123222B14E4B484A41F22D01A6
:10EAF000CFE77F2B04D84C4B444A41F23001C8E7A2
:10EB00004B6A23B9494B414A41F23C01C1E70B6BC7
:10EB1000ABB1E360A36E5A6BE2B1E261A06E214635
:10EB2000FFF7A0FFA06E04F11001FFF79BFFA36E9B
:10EB3000D86AB0B93E4B354A41F25A01A9E707F00D
:10EB4000A9FAE0600028E5D12046FEF717FF6FF034
:10EB50000B0058E0986A07F09DFAE0610028DDD1CB
:10EB6000F2E7410702D19B6B9A0704D0314B274A49
:10EB700041F25B018DE74BB16366A36EDA6BFF2A4E
:10EB80000AD92D4B214A41F2680182E707F082FA47
:10EB900060660028F1D1D7E7002A08BFFF2222676C
:10EBA0001A6C002A04DA254B184A41F26E0170E70C
:10EBB00008BF6FF0004262675A6C40F2FE318A4231
:10EBC00004D91F4B114A41F2740162E7002A08BFC1
:10EBD0000A46A2679A6CDB699A4204D9194B0B4A20
:10EBE00041F27A0155E700204FF0FF33C4E90833C2
:10EBF000C4E90A00C4E90F00C4E90C00C4E912002A
:10EC00006064A063206538BDFD540200AF66020059
:10EC1000C8530200165502002F5502004955020044
:10EC200079550200A9550200DA550200F655020096
:10EC3000125602002F560200835602009D56020013
:10EC4000BE560200D95602002DE9F0430D46096870
:10EC50009846CB1C85B00646174603D9002005B060
:10EC6000BDE8F083C36E994205D31C4B1C4AB32107
:10EC70001C4806F00DFC806EAC6882691444013CAF
:10EC8000B4FBF2F302FB1343E41A0094D0F80890AB
:10EC9000EB686A68C847002803DD134B104AB721A8
:10ECA000E6E7DCD1B8F1000F04D1B06E2946FFF7DA
:10ECB000D9FED3E74FF0FF333B600294EB6801933A
:10ECC0006B6800932B68224639463046FFF7DCFB21
:10ECD0000028C4DBE9D06FF05300C0E708570200FA
:10ECE00065660200C8530200615402002DE9F74F27
:10ECF000DDE90C9519F1020FDDF83C800193074620
:10ED00000C46924608D0C36E4B4505D82E4B2F4A71
:10ED1000E8212F4806F0BCFBBA6ED26905EB080368
:10ED2000934206D84FF0000BB8F1000F05D14046D2
:10ED300033E0284B254AE921EBE723684B452FD1E7
:10ED40006068A8422ED8BB6E9E6A0644AE4229D99E
:10ED5000761BE3680E99464528BF4646281A324678
:10ED6000184407F0FDF86368A2683544EB1A934233
:10ED700038BF1346A360BA6E926A9A4205D00E9BC2
:10ED800033440E93A8EB0608CEE7019B524621467A
:10ED90003846FFF759FF0028F1D003B0BDE8F08FE7
:10EDA000013304D00C4B094A4FF48371B1E7C4F826
:10EDB0000090BB6E9A69B5FBF2F302FB1353EB1A9A
:10EDC000C4E9013BB0E700BF2957020072660200A8
:10EDD000C853020060570200835702002DE9F04F2C
:10EDE000044687B00D4605A92046FFF79BFD064661
:10EDF00058B9DDF8148020464146FEF7D5FD064699
:10EE0000002853D010F1540F56D0304607B0BDE85B
:10EE1000F08F2A6BCDF80C900DF1130A12F4801FBD
:10EE2000CDE9017AA3EB07031CD0AA88294941EA5E
:10EE30008222009205F108015A462046FEF72CFF77
:10EE400070B9CDE902A9CDE900870123224604F17A
:10EE500010012046FFF74AFF60B110F1540F2BD08C
:10EE60000646D2E7AA6B0092594622462046FEF794
:10EE7000D9FBE5E70137EB6BBB42CAD8A36EE1696A
:10EE80009A6AE86C07F06CF823692B6463696B6419
:10EE9000A369AB64A06E04F11001FFF7E3FD2B6BD7
:10EEA000C5F8388043F400332B63AEE7074605F11D
:10EEB000400B4FF00109DEE7074B00930749084874
:10EEC000434640F6C24207F0F1FC4FF0FF332361A6
:10EED00089E700BF0000102038520200C85302002A
:10EEE000A65702002DE9F04F91B0CDE907230B6B37
:10EEF000DA0206460D462CD5089B486BB26EC11847
:10EF0000EB6A946A994238BF1946936CE3B140F2B8
:10EF1000FE32A2424FEAD30328BF2246934228BFC3
:10EF200013468B4215D2E863F36E336629463046AA
:10EF3000FFF754FF2B6B044640B143F400232B63CF
:10EF4000204611B0BDE8F08FD369E0E723F48013C9
:10EF50002B63089B049305F140030B93049B0BB9AF
:10EF6000089CEDE72B6B13F4003205D0B16EE86B13
:10EF7000C969884240F0AA80DB0200F1DF8005F118
:10EF800040030593BAB96B6BABB10F920FAA029213
:10EF9000013B05F1380201920093D5E90A23059956
:10EFA0003046FFF7DDFA044608B12B6BC5E705993B
:10EFB000B06EFFF757FDF36E3366AB6B09936B6B67
:10EFC00006930DA93046FFF7ADFC04460028ECD1AE
:10EFD000DDF8348030464146FEF7E6FC044678B161
:10EFE00014F1540FE1D15F4B00935F495F484346F2
:10EFF00040F68C3207F05AFC4FF0FF332B64E0E709
:10F00000069B1BB9C5F83880EB635BE0B76E069BC7
:10F010000EA9013B38460E93FFF785FA0E9B03F1CC
:10F020000109FB69CDF83890994572D1013090FA09
:10F03000A0FB099B0F93BBFA8BFB0BF1010AA146C6
:10F040000FAF4FEA89030A930423CDE902730A9BA9
:10F050000599CDE90083324601233046FFF746FE8D
:10F060000F9B04460028BBD1D94557D109F10109AE
:10F07000CA45E6D8C5F838804FEA8A03C4E7099B39
:10F080000093CDE9027BCDF804A0A9EB0A03324638
:10F0900000213046FEF7C6FA0446002885D1CDE9A6
:10F0A000027BCDE9008A0599012332463046FFF7FD
:10F0B0001DFE0446002893D10AF1010AD145DED88D
:10F0C000C5E90E892B6B43F400332B63B36EDF6904
:10F0D000EB6BFF1A049B9F4228BF1F46079B0397B9
:10F0E0000293EB6B0193AB6B00930B9901233246B8
:10F0F0003046FFF7FBFD044628B310F1540F7FF4B0
:10F1000054AF29463046FFF769FE04460028E5D093
:10F110004BE7A2464FF0010B0FAFCFE70422CDE93A
:10F1200002720A9A0146CDE9003230460423324683
:10F13000FEF778FA0446002898D036E76FF001030E
:10F14000AB636B6B60E76B6B3B446B63EB6B3B449C
:10F15000EB63079B3B440793049BDB1B0493F36E19
:10F160003366FBE638520200C8530200A65702007D
:10F17000F0B585B0CDE902231D464B6801930B68BD
:10F1800000930C4617460023024600F11001FFF7DA
:10F19000ADFD064640B9E0682A46394601F0B0FFA9
:10F1A0006368E0602B446360304605B0F0BD2DE934
:10F1B000F04F064687B010469946FEF769F94B684E
:10F1C00093464A69034493420C46804641D88B6873
:10F1D0002BF0004A8AEA03031BBA059305AA04230D
:10F1E0003046FFF7C5FF054678BBBBF1000FA8F11D
:10F1F000040720DA0DF1130B2FB30123CDE902B37D
:10F20000D9F80430043B4344DB1B0193D9F80030A8
:10F21000009332463B4600213046FEF703FA40B9E0
:10F2200001235A4621463046FFF7A2FF013F00283E
:10F23000E2D0054609E03B464A4621463046FFF704
:10F2400097FF0028F5D1C4F808A0284607B0BDE80C
:10F25000F08F6FF01B05F8E713460A46D0E900016E
:10F26000FFF7A5BF2DE9F0430B6B0C46590399B08E
:10F27000054608D5DA0258BF4FF0FF3223F4802349
:10F2800058BF22642363216B8B0303D4002019B081
:10F29000BDE8F08311F48011666BE76A4CD154220B
:10F2A00003A806F039FCA36ACDE90D370123CDE9A7
:10F2B0000F3695E80F0013AF87E80F004FF0FF37C8
:10F2C0002F60626BE36A9A421FD3DFF89090DFF8F9
:10F2D0009080214F01232A4604F140012846FFF780
:10F2E000B3FC68B310F1540FD1D1CDF80090414672
:10F2F000A36B40F61152384607F0D8FA214628464B
:10F30000FFF76CFD0028E5D0C1E701230DF10B02EA
:10F3100003A92846FFF76EF90028B8DB01230DF199
:10F320000B0221462846FFF7DDFD0028AFDB2B68E6
:10F330000133C6D01397C3E7B7422CBF6763666338
:10F34000A36BA362636BE362236B23F4003343F488
:10F350008033C4E90C3699E7A65702003852020000
:10F36000C85302002DE9F7431E460B6B17469A0758
:10F3700005460C4606D4234B234A244840F6076131
:10F3800006F086F85A0319D4216B0B051DD4D4F866
:10F3900034806B6F08EB06029A422FD811F40039C3
:10F3A00019D033463A4621462846FFF79BFD0028F0
:10F3B00008DB236B23F40023236303E0FFF752FFF2
:10F3C0000028E1D003B0BDE8F083E36A626B9342AA
:10F3D00088BF6363DBE7E36A9845E2D96363636BE5
:10F3E0009845DED901230DF10702214628468DF804
:10F3F0000790FFF777FD0028F1DAE3E76FF01A00D6
:10F40000E0E700BFC95702009E650200C853020032
:10F410002DE9F04F0D46816E6B688A69C969143316
:10F42000571E8B4294BFFF187F184FF0000AB7FB9E
:10F43000F2F302FB13738BB00446FF1AD1466FF050
:10F44000030B6E68BE4219D32B694FF0FF3208924E
:10F45000A9EB0302CDE9003208AE02962B6809F150
:10F46000040221462046FEF779FC002847D1089B7C
:10F47000534500F0B7806FF0530040E0ABEB06035C
:10F480003B44043640F2FE32934294BFF618B6185D
:10F49000BE424FF0FF0335D38DF81F30A26ED2E984
:10F4A0000632D21A964236D8012203920DF11F027B
:10F4B000CDE901622A680092002122462046FEF72B
:10F4C000B1F810B110F1540F19D1A36E9A690096DA
:10F4D0004FF0FF33099309ABCDE9012321462B6897
:10F4E00008922046FEF73AFC10B110F1540F06D1F5
:10F4F000444A08AB29462046FFF759FE58B10BB0E5
:10F50000BDE8F08FA7F11402964228BF1646BE420E
:10F510008DF81F30C2D29DF81F206B68E868D24377
:10F52000ABEB0308C2F3C01202F5A062B04448EA94
:10F530000258AB6848F47F2848F4406888EA03031F
:10F540001BBA089308AB1946042201F0D9FD082222
:10F5500008ABE860039202936B6801932B680990F3
:10F5600004F1100100932246002320460591FFF785
:10F57000BDFB0028C3D10599B9F1000F04D16B6818
:10F58000D5F80CA003F104099DF81F306E60DB4331
:10F590001B0603F0004383EA0803AB60BE424FF052
:10F5A000FF33EB6006D2A36E62699B6A13449E42EE
:10F5B000FFF447AF4FF0FF3323602246002320467D
:10F5C000FFF742FB00289AD1A06E036998470028F4
:10F5D00005DD0D4B0D4A0E48DD2105F059FF3FF4C6
:10F5E00030AF8CE70422CDE9009202962B682146C9
:10F5F0002046FEF7B3FB002881D1089B002B3FF487
:10F600007EAF38E708FCFF5F615402001C66020011
:10F61000C85302002DE9F04F97B0CDE90823836E5F
:10F62000BDF884805A6A8B68BDF888B00133002A1F
:10F6300004460D468B6028DC0026002700234FF08F
:10F64000FF32CDE91132CDE913236968A26E109122
:10F65000936C002B4AD0083B20461593FEF7A4F983
:10F66000002845D010F1540F40F0D7804FF0FF3301
:10F670002361FEB9714B00936B687149714840F684
:10F68000010207F013F9374615E0013242F001029A
:10F69000B3FBF2F102FB1133002BCDD1012610A9EF
:10F6A000284610931196FDF7CEFE0028C5D04FF0E6
:10F6B000FF332361012700264FF0010910A92846D6
:10F6C000CDE91069FDF7BFFE002840F0A9805B4B33
:10F6D00000936B685A495C4840F6060207F0E6F86A
:10F6E0006FF01B0099E006464F46A7E7D369B2E7E3
:10F6F0000DF14009042305F1080249462046FFF7B1
:10F7000037FD0028AED10BAB0793504B0693C8F1E1
:10F7100000031BB2CDE904B34D4B0293099B019347
:10F72000089B009302462099CDF80C804FF0FF33E0
:10F730002046CDE90B49FEF755F9002892D105F195
:10F7400018010846FDF775FE68B9EA7D0B46414988
:10F7500002F5C06241EA025220464946FFF727FD02
:10F7600000287FF47FAF0023CDE90D330F934FB90D
:10F7700004F13C010DA8FDF795FE04F130010DA840
:10F78000FDF790FE04F1480A51460DA8FDF78AFEE8
:10F790000D9B0DAA6FF30903294620460D93FEF732
:10F7A000B5F8002839D10DA8FDF78AFE40B92A4ADC
:10F7B0000DAB49462046FFF7FAFC00287FF452AF14
:10F7C00049462046FFF724FE00287FF44BAFA36E86
:10F7D000119A9969B2FBF1F301FB132333B11F4B6B
:10F7E0001F4A174840F2EF7105F052FED5E90010AC
:10F7F000EA60ABEB0808129AA5F81480C5E900018D
:10F800002A61A364CAE9013337B904F13C033034F7
:10F8100094E8070083E80700384617B0BDE8F08F8A
:10F82000291D2046FFF77EF800283FF45CAF10F159
:10F830001C0FF2D1002F3FF453AFFFE63852020005
:10F84000C8530200A65702001C58020059F20000DB
:10F8500000FC0F4008FC0F000CFCFF7FF657020075
:10F860000C6602002DE9F0438DB00C4604A9BDF8EA
:10F870005490054617469846FFF7A8F8064628BB59
:10F88000E37D8DF82730A3690A93E3690B93BDF8F4
:10F890005830CDE90193149B00933A46434604A99E
:10F8A0002846FFF7B7FE002814DB049F059AA761DE
:10F8B0000123E261E37505F120012046FDF7C3FD58
:10F8C00020B9B9F1000F01D1C5E9087230460DB079
:10F8D000BDE8F0830646F9E72DE9F04F97B093466F
:10F8E000209ADDF8848006460D461F4603EBC200D1
:10F8F000002140F2014440F2FF4C834240F08880F6
:10F90000002940F0B080AB7D002B40F0CD804FF05F
:10F91000FF333361B5F814904FF00008A9EB080AE3
:10F92000BAF1010F00F26E81B8F1000F1CD01FFA7E
:10F9300088F8CDE90189209B00953A462946304652
:10F94000FFF790FF0446002800F0448110F11C0FDF
:10F950005AD1A14B01936B6800932B689F49A04833
:10F9600040F6590206F0A2FFB36E5A6A002A3FDD44
:10F97000AB680132013342F00102B3FBF2F102FB4A
:10F980001133002B34D1109310A901232846119371
:10F99000FDF759FD804658BB3046FFF755F8041E69
:10F9A00077DBF36E1C1BB4EBD30F21D9DFF828A251
:10F9B000CDF800A0AB6889498A4840F66F0206F08E
:10F9C00075FFCDE90189209B00953A4629463046CE
:10F9D000FFF748FF0446002800F04F8110F11C0F8C
:10F9E00012D17E498048534640F6790206F05EFF08
:10F9F0000023CDE90053CDF80890209B3A462946D4
:10FA00003046FFF707FE0446002C80F2CB8040E032
:10FA10001A684FEA125EC2F30A52A24204D1AA8ABD
:10FA20000132AA82083368E762450CD1AA8A32B94A
:10FA30006E4B6F4A40F69101684805F029FD013A86
:10FA4000AA820121EEE70EF4E062B2F5C06FE9D1BF
:10FA50005A681268AA615A685268EA611A68C2F361
:10FA60000052EA75DEE7AB8A002B7FF44CAFB8F1A9
:10FA7000000F04D15F4B5E4A40F69E01DCE7424630
:10FA800029463046FEF70CFC044630B1831C3FF497
:10FA90003AAF204617B0BDE8F08F98F81730002B2A
:10FAA0003FF431AF02247DE0EA682B6810934FF0F9
:10FAB000FF31CDE913122B69B06E11921293816C54
:10FAC00001B3083915910BA907914B490691002103
:10FAD000CDE90411CDE9021120990B96CDE9007111
:10FAE0000DF1400829463046CDF83080FDF77AFF09
:10FAF000044648B114F11C0F3FF409AF14F1540F40
:10FB0000C7D104E7C169DCE706F13009CDE90D0092
:10FB10000F9049460DA8FDF7C5FC06F13C031946B8
:10FB20000DA806F1480A0993FDF7BCFC0DA8514643
:10FB3000FDF7B8FC0D9B0DA86FF309030D93FDF7BE
:10FB4000BFFC80B90DAA29463046FDF7DFFE04460A
:10FB500000289ED1294A0DAB41463046FFF727FBCE
:10FB600004460028C6D141463046FFF751FC044602
:10FB70000028BFD1B26E119B9169B3FBF1F201FB7A
:10FB8000123222B11E4B1A4A40F6E80154E7EB60EC
:10FB9000129B2B6199E80700099B83E80700B46476
:10FBA000CAE90144DBF800301093D6F82880DBF86E
:10FBB00004301193B8F1000F3FF46BAF08F108095E
:10FBC00010A94846FDF73FFC8246002857D0D8F8D8
:10FBD0000080EFE7C1469FE638520200C85302009A
:10FBE0006658020094580200C4580200525802009D
:10FBF000396602006158020059F200000CFCFF7FD8
:10FC0000F65702000023109310AB1FFA88F20793F7
:10FC1000494B069353421BB2CDE90493474B0293E1
:10FC2000209B0392CDE9007300224FF0FF33294659
:10FC30003046FDF7D7FE044600287FF4E5AEBAF162
:10FC4000FE0F15D8B36EDA69986CA2F1280190B155
:10FC500042089869431E1344B3FBF0F200FB1232D2
:10FC60009B1A8B42109A28BF0B469342BFF45CAE9E
:10FC700008EB5A0852E65208EBE78146B8E6AE4672
:10FC8000BEE80F00CC46ACE80F009EE80F00D94557
:10FC90008CE80F0008D040F2FF4140F20140209A6A
:10FCA000B8F80430924517D108F1200AB8F80430AA
:10FCB000B8F81C2093428AD398F81F10002986D0E8
:10FCC0009B1AA8F80430524649463046FEF7DAFA45
:10FCD0000028EBD00446DCE657F83A20C2F30A5C71
:10FCE0008C4518D1C2F389229A4206D14FF0FF33D6
:10FCF000C8E902330AF1010AD1E7FBD2013BA8F8B7
:10FD0000043098F80630022BF4D1D8F82830013BA3
:10FD1000C8F82830EEE78445ECD1C2F389229A4234
:10FD2000E8D80133A8F8043098F80630022BE1D166
:10FD3000D8F828300133EBE7A9D5000000FC0F40CC
:10FD40002DE9F04F866A9FB00546884691469A464F
:10FD5000002E66D1D8F8003006934646D8F8043015
:10FD600007930FCE0EAC0FC496E80F000EAF16AE81
:10FD700084E80F00CDE900A64B46424639462846A6
:10FD8000FFF7AAFD041E77DB06A94046FDF75BFBE3
:10FD900048B9BE46BEE80F00C446ACE80F009EE876
:10FDA0000F008CE80F00022C2CD105F148024146CF
:10FDB0002846FDF7ABFD044600285DD1169B98F858
:10FDC00017200693179B0793AE4B019002F5C06274
:10FDD00043EA02530A9308F118030B93012300939B
:10FDE00006AA0AAB31462846FFF776FD041E43DB20
:10FDF000B646BEE80F00BC46ACE80F009EE80F0018
:10FE00008CE80F000023DFF89892DFF890B205939A
:10FE1000012C00F0A680059B002B0CBF00240324BE
:10FE20002AE006F10800404501D1366890E74146D6
:10FE3000FDF709FB0028F8D1B379012BF5D1336B1D
:10FE4000DA02F2D5AB6EF26A9B6A9A42EDD9736B15
:10FE5000F363EB6E2B6631462846FEF7BFFF044680
:10FE600050B9336B23F48013336331462846FFF7D0
:10FE7000F9F904460028D8D020461FB0BDE8F08F1D
:10FE80000AF1080106A8FDF7DEFA08B9CAE902423C
:10FE90009AF80630022B07D10AF12C0106A8FDF7CB
:10FEA000D2FA08B9CAE90B42DAF800A074E00121DD
:10FEB0002846FDF789FB04460028DDD1314605F1CF
:10FEC0003000FDF709FB002800F08C802C6B179B9D
:10FED0000093C4F38924169B6B48CDE9014940F691
:10FEE0009F12594606F0E2FC2B6BC5F838A06FF361
:10FEF0009E23C5E90C3AC8F38923A34276D9A8F515
:10FF00008062169B0493089340F2FF339C4218BF13
:10FF10005E4BDDF85CA0CDF824A014BF43EA842337
:10FF200000230A930023CDE90B32019302230093AF
:10FF300008AA0AAB314628460D97FFF7CDFC041EF0
:10FF40009ADB012C54D1049B0594B646CDE9063AC0
:10FF5000BEE80F00BC46ACE80F009EE80F008CE83E
:10FF60000F000F9B02930E9B0193079B009340F69B
:10FF70007212069B4648CDF80C90594606F096FC46
:10FF800005F1200106A8FDF75EFADDE90E4208B989
:10FF9000C5E90842D5F828A0BAF1000F7FF470AF88
:10FFA000324606A92846FEF70FF9B0F10008BFF661
:10FFB0007EAF18F1020F40F08B80324606A928462A
:10FFC000FEF76EF90446B0B1831C7FF455AF18F10B
:10FFD000020F3FF420AF2F4B2F4A304840F6C2119A
:10FFE00005F056FA424640F2FF348AE7424688E777
:10FFF0004FF0010AE1E72B6BC3F30903002B38D163
:020000021000EC
:10000000314605F13000FDF767FA00284AD140F289
:10001000FF34169B0693179B079340F2FF339C42D5
:1000200018BF1A4B9DF86F2014BF43EA84230023A6
:100030000A93144B02F5C06243EA02530021CDE952
:100040000C3702230B910191009306AA0AAB3146AB
:100050002846FFF741FC041EFFF60EAFB646BEE889
:100060000F00BC46ACE80F009EE80F008CE80F00C4
:10007000CEE6CAF100012846FDF7A6FA044600289C
:10008000BED0F9E608FC0F002B5902000000F04F2B
:10009000EF5802006E5902008B660200C85302003E
:1000A000385202002C6B179B0093C4F38924169BD3
:1000B0000848CDE9014940F6D312594606F0F6FB4F
:1000C0002B6B6FF39E232B630023C5E90D33A0E751
:1000D0004446D1E62B5902002DE9F04F0446006B4F
:1000E000C0F30900A3B0884648B3DFF8B8910025F3
:1000F0001C2200210AA805F00FFD01238DF83F30D6
:100100001193002710A8FDF794F918B1002F61D0C2
:100110000025EDE710AA12A92046FEF7B3F870B942
:100120009DF83F30002B40F0A2801AAA10A920466B
:10013000FEF74AF8002859DA811C00F0958023B0B8
:10014000BDE8F08F236B4F494F48C3F3892A0B9BBF
:100150000093CDE901AB0A9B41F22E3206F0A6FBDB
:10016000236BA5636FF39E23C4E90C3540F2FF3384
:100170009A4565D0454B43EA8A2362E0B8F1000F07
:1001800075D0434B0193119B3E49009341F24E328F
:10019000109B404806F08AFB04F1480212A9204651
:1001A000FDF7B4FB0028CAD19DF85F203A4B02F559
:1001B000C06243EA0253069318AB079306AA2B4684
:1001C0000AA92046FFF7BCFD0028B8DB032808BFBA
:1001D000474697E70135022D8AD1216B494249B242
:1001E000204623B0BDE8F04FFDF7EEB9002D3ED11B
:1001F00004AE034600964A461AA92046FDF77AFB4C
:1002000000289CDB10A93046FDF72EF900282ED1DE
:10021000059B0293049B0193DFF874B0119B19496D
:1002200000931E48109BCDF80CB041F2233206F02B
:100230003DFB0AA904F13000FDF74EF9002881D1F9
:1002400000230693164B09960022CDE907230AA93D
:10025000022306AA2046FFF773FD0028FFF66FAFC2
:10026000032808BF01274DE70DB1012D86D00DF100
:10027000480CBCE80F000AAE0FC69CE80F0086E8E9
:100280000F003FE7C8530200D75902000000F04FAB
:10029000385202001E5A020008FC0F009359020057
:1002A00008FC0F6000FCFF7F10B50446FFF748FD17
:1002B000002806DB05D020460021BDE81040FFF7EE
:1002C0000BBF10BD30B5036B9B0595B0044630D510
:1002D0003B4B0193436A009305463A4955F8203F4A
:1002E000394841F2AE2206F0E1FA2A460CA920462E
:1002F000FDF7C8FF002861D1344B0693A36EDB697C
:100300000793E36E0893236F0993636F0A93A36FB8
:100310000B932F4B049306AB059304AA01230CA95E
:100320002046FFF7C1FF002848D1236B23F4007358
:100330002363E36B1A0D12F4E06F06D1012120460E
:1003400015B0BDE83040FFF7C7BE1D4A0292C3F3A7
:1003500089230193636C0093236C1A491D4841F271
:10036000D62206F0A3FAE36B40F2FF42C3F30A532E
:10037000934206D0184B194A124841F2DD2105F08C
:1003800087F804F140020CA92046FDF77BFFA8B9CD
:10039000E36BA063C3F38922236B6FF39E23C4E94D
:1003A0000C300F4B43EA8223CDE9063006AA012325
:1003B0000CA92046FFF778FF0028BFD015B030BD4C
:1003C00038520200C85302004B5A020001000200DA
:1003D000180010207F5A0200B05A0200FE65020089
:1003E0000000F04F73B514460E4600F14802214656
:1003F0000546FDF78BFA70B9E27D084B02F5C06245
:1004000043EA02530093183401236A4631462846D2
:100410000194FFF749FF02B070BD00BF08FC0F0058
:1004200070B50B6B1E0386B005460C463FD4FEF735
:1004300019FF226B20B142F40022226306B070BD86
:10044000D10334D504F108063046FCF7F2FF00284A
:100450002DD1D3025DBFD4E90A016B46C3E9000187
:10046000E26AA1884BBFE36C082240F2012040F20F
:10047000022042EA812242EA0052CDE90223226DA3
:10048000936843EA812343F08153049353680593AF
:1004900002AA022331462846FFF706FF236B18B154
:1004A00043F400232363C9E723F48033236300204C
:1004B000C4E770B505460C46FFF7B2FFAB6A0646C7
:1004C00005F128021BB19C42196808D11160236D07
:1004D0001B6813B9E06C05F0E5FD304670BD1A46A7
:1004E0000B46EFE770B58CB0164601911D4601AA88
:1004F000002304A90446FDF71FFF00281BDBC0F3FF
:10050000892040F2FF33984206D104F1200204A969
:100510002046FDF7B7FE70B9109906F5407641EA1E
:10052000065141EA8021CDE90215012302AA04A95E
:100530002046FFF7B9FE0CB070BD00002DE9F04772
:100540008AB013F0020F06460D460392984634D146
:10055000129B2B6505F1080700236B63EB63EB64CB
:10056000C5F830802B1D03AA39463046FDF7E4FE5E
:10057000041E06DAA21C17D1AA8840F2FF339A4261
:1005800012D00123AB71B36A2B60A31CB56257D1A3
:1005900018F4807F08D0039C204605F051FA336F91
:1005A000834213D26FF023042B6B43F400232B639D
:1005B00029463046FFF77DFF04E0FFF783FE04463F
:1005C0000028C5D020460AB0BDE8F087AB88644A51
:1005D000DFF8948142EA832240EA8320049240F4C7
:1005E0008010002248EA8323CDE90604CDE90832D1
:1005F0000592032304AA39463046FFF755FE10F151
:100600001C0F0446CED00028CED14446DFF85CA1B2
:100610004FF000084FF00C092B6D9A68424535D811
:100620001B68002B62D0EB64B06E05F14001FEF751
:1006300019FA40F20123B3EB145F61D00024C1E743
:1006400018F4007F40F08380240D012C40F082805C
:10065000AB8818F4806F4FEA832308D043F000542E
:100660002B6B43F4803344F480142B63CEE705F105
:10067000280243F00053009243F00803394A3946F8
:100680003046FDF737F9041EC0DA8DE72A6BD00734
:1006900006D42B6B2A6D99071DD408F10108BBE71E
:1006A0005868B5F804C009FB08F28118825C8B68B1
:1006B0004968009143EA8C2302F5407243EA0253F1
:1006C000394652463046FDF715F90028E1DA831C19
:1006D000DFD0044668E7526809FB08229168B26FD0
:1006E00091423AD843F480332B63D6E7B36E986ACD
:1006F00005F0D0FCE864002896D16FF00B0453E7B6
:100700002B6B43F480136FF001022B63C4F30904D5
:100710000023AA62EC622A646B64B36E9A6AAA64CC
:10072000002C8BD040F2FE339342A98828BF134699
:1007300043EA8123EA6C009243F00053094A3946A8
:100740003046FDF7D7F8041EBFF678AF2CE76FF000
:10075000100429E76FF0140426E76FF01B0423E769
:100760000000104000FC0F700000102000FCFF7F14
:100770002DE9F341144606464A6B0D461BB1012B89
:100780000AD114193AD4736FA34237D3944210D1CB
:10079000204602B0BDE8F081022B08D1D1E90B312F
:1007A000890302D5934238BF1346E418EAE714469A
:1007B000E9E72B6B9B0319D4D6F868800092694651
:1007C0004046FDF7B0FE01A9074640460194FDF7FB
:1007D000AAFE87420AD16B6C019A934206D8A96C93
:1007E0000B449A4202D26C63EA63D1E72946304651
:1007F000FEF738FD0028CCD16C63C9E76FF0150017
:10080000C7E7000070B596B006460D46FEF736F90C
:100810000446002856D12B6A33B92C4B2C4A2D485C
:1008200041F2AB0104F034FEB36E0146DA6A706E39
:1008300005F072F9D6E91A327465DB6ADB00C6E9A5
:100840001742934294BFB365B2650EA93046FEF7D6
:10085000BDF80446002832D11F4B0293B36EDB690A
:100860000393F36E0493336F0593736F0693B36F23
:1008700007931A4BCDE90830194B0A93194B0B9388
:10088000194B0C9302AB0D9308AA03230EA9304613
:10089000FFF70AFD044690B98DF84E000346024664
:1008A0000EA93046FFF700FD044640B90090012331
:1008B0006A460EA930460193FDF7E4FC0446304633
:1008C000FDF75CF8204616B070BD00BFE15A02008B
:1008D000B8660200C8530200010002000000104088
:1008E0000800F00FF75A020018001020FDF746B874
:1008F0002DE9F04F99B00446FEF7C0F805460028F0
:1009000051D101461C2210A805F006F9804BDFF8F2
:100910003CA2DFF83CB293E803000DF1140888E82C
:10092000030001261796374616A8FCF782FD40B350
:1009300004F130063046FCF7C3FD60B9754B0293F5
:10094000A36B0193636B0093236B7349734841F26C
:10095000791205F0ABFF236B03EBD373236396E8A7
:10096000070004F13C0383E80700E26EE36AB3FB8F
:10097000F2F102FB113363650023C4E916332266EA
:1009800011E0414616A8FCF76FFD80B1614B62494A
:10099000634841F2F40205F089FF6FF053092046E5
:1009A000FFF7A4FF4D46284619B0BDE8F08FB742C7
:1009B00005D1169B0593179B06937E000746594B5E
:1009C00008930823099307ABCDE902A3564B07947C
:1009D0004FF0000CCDE9003C16AA544B10A920465C
:1009E000FDF7EAF9B0F1000907F10107D7DB00F0E4
:1009F000848049F3090301337FD0109B2362119B4C
:100A000063620AAB0093494A5B4610A92046FCF793
:100A100071FFB0F10009C2DB0A9A130C022B91B2EC
:100A200001D1012910D93B4903910120022192B241
:100A3000CDE90110009238493D4841F2221205F0FB
:100A400035FF6FF01509AAE781B93249039192B2D7
:100A50000121CDE9013100922F49364841F230128F
:100A600005F024FF236B43F4007323630D9B6BB1EC
:100A7000226F934209D927492F48CDE90021264901
:100A800041F23E1205F012FFDBE723670E9B5BB1DC
:100A9000626F934207D91F492848CDE900211E49BA
:100AA00041F24912EEE763670F9B5BB1A26F93427D
:100AB00007D918492248CDE90021174941F25412BB
:100AC000E0E7A367A16E0C9B0A6A4AB19A4207D07D
:100AD00010491C48CDE900210F494FF48B52D1E752
:100AE000E366CA690B9B934207D00A491648CDE9D1
:100AF0000021094941F26912C4E704F1300210A94A
:100B00002046FCF703FF814600283FF40DAF46E77F
:100B1000C866020038520200C8530200675C020037
:100B2000A8540200F75A02000800F00F00FCFF7FF3
:100B3000005B0200355B0200735B0200A45B0200F5
:100B4000D55B0200065C0200375C0200EDE40000A9
:100B5000180010202DE9F04FAFB0CDE90612054680
:100B6000FFF7B0FB0346002840F00F810DF1280984
:100B700006AA49462846FDF7DFFB061EC0F207819C
:100B800040F2FF38C6F38927474505D16FF01504B9
:100B900020462FB0BDE8F08F0DF1160307AA12A969
:100BA0002846FDF7C9FB041E2ADBC4F3892343450D
:100BB000ECD012A94846FCF746FCAB6A1A93A11C7C
:100BC000804629D1079804F03BFF2B6F984200F232
:100BD000E080BDF81630B8F1000F18D02B6B6FF322
:100BE0009E2343EA872343F09F4343F4E0032B63B0
:100BF0000A9B6B63A21C0B9BAB6347D13A4609E08F
:100C0000A01CC5D1BDF816304345D2D1C0E79F42E4
:100C1000F4D37A1C00233FE0330DB3EB145F4FEAAB
:100C2000145240F0B980BDF81630002840F0B7806B
:100C30009F4201D10024ABE7022A27D15A4A0DF185
:100C4000900A42EA8323CDF800A0584A12A9284608
:100C5000FCF750FE002859DB52461CA92846FDF738
:100C600011FB002852D1219B33F47F034CD1012189
:100C70002846FCF7A9FC002848D11AAB8DF86E0075
:100C8000ADF86C00AB62B8F1000FA7D1BDF816202B
:100C9000474B43EA82233A4624934649BDF816302F
:100CA00003926FF3130641EA83214FEA832B46EA4E
:100CB0008326079B02934FF0000A1846CDE9261AB7
:100CC000CDF894A004F0BCFE029B29934BEA0703E5
:100CD00043F08053064343F48013CDE92A39289624
:100CE000B8F1000F14D1324B039A43EA82232C93BC
:100CF00000232D9324AA052312A92846FFF7D4FA2E
:100D000040B11A9BAB6201E06FF0260004463FE75A
:100D10005346ECE7B8F1000F16D02B6B1A0D12F406
:100D2000E06F11D06FF39E23C5E90C30204BA86310
:100D300043EA8723CDE9083008AA0123494628461B
:100D4000FFF7B2FA0028DCD11A9BAB62A31C3FF478
:100D500071AF240D022C7FF46DAF4FF0FF312846A8
:100D6000FCF732FC044600287FF412AF12AA1CA93B
:100D70002846FDF795FA044600287FF409AF1CAA1F
:100D800012A92846FFF72EFBC0E7044600E73446C9
:100D9000FEE66FF02304FBE66FF01404F8E6022A87
:100DA0003FF44CAF1AE700BF0800002000FC0F70B2
:100DB0000000F04F0000104070B58CB01646039153
:100DC0001D4603AA002304A90446FDF7B5FA00282E
:100DD00023DBC0F3892040F2FF33984206D104F1AF
:100DE000200204A92046FDF74DFAB0B9A36F10996F
:100DF0000C4A0095994228BF194606F5407641EA0B
:100E0000065141EA802304A92046FCF773FD00281F
:100E100005DA831C08BF6FF03C000CB070BDC0F356
:100E20000900FAE700FCFF7F30B4029D846FA54201
:100E300002D830BCFFF756BB6FF01B0030BC7047C8
:100E400010B50446806AFCF755FB30B1054B064AE5
:100E5000064841F2417104F01BFB2046BDE81040FA
:100E6000FFF76CBB9E5C0200ED650200C8530200F8
:100E700008B50346806AFCF73DFB30B9054B064ACE
:100E8000064841F2507104F003FB1846BDE80840E3
:100E9000FFF70FBB9F5C0200DE650200C853020033
:100EA0002DE9F0410446806A0D4616461F46FCF7C0
:100EB00021FB30B90F4B104A41F272710F4804F018
:100EC000E7FA0B6BDA0704D40D4B0E4A40F69C513F
:100ED000F4E79B0307D43B46324629462046BDE84B
:100EE000F041FDF787BB2046FEF7BCF90028F2D0A1
:100EF000BDE8F0819F5C0200D0650200C85302008B
:100F0000D55C0200BF65020010B50446806AFCF79C
:100F1000F1FA30B9054B064A064841F2847104F0F3
:100F2000B7FA2046BDE81040FEF71CBA9F5C0200ED
:100F3000B0650200C853020010B50446806AFCF791
:100F4000D9FA30B9054B064A064841F2967104F0C9
:100F50009FFA2046BDE81040FFF70ABC9F5C0200E4
:100F600090650200C85302002DE9F041054686B0A5
:100F7000806A0C461646FCF7BDFA30B94C4B4D4A18
:100F800041F2A7714C4804F083FA0A6B910704D42C
:100F90004A4B4B4A40F67261F4E7002EC0F284805F
:100FA0009203676BE36A02D5BB4238BF3B469E4261
:100FB0005FD2AA6E936C916A002B3AD040F2FE3257
:100FC0008A424FEAD30328BF0A46934228BF1346FA
:100FD0009E4230D800231A4621462846FFF7C8FB18
:100FE00000285EDB4FF0FF332B60EA683346214672
:100FF0002846FDF7FFFA002853DB236BE06C6FF007
:101000000102C4E90A2643F4A813236300232264DF
:101010006364AB6E9B6AA364E968324604F0A0FF88
:1010200000233A4621462846FFF7A2FB00EAE0707B
:1010300037E0D369C2E721462846FEF713F980BBA3
:1010400005AB029304F138030193731E00930590DE
:10105000D4E90A2304F140012846FDF781FA00BBD8
:10106000A36B6663C4E90A36236B43F4A0232363AE
:10107000D6E7D5D90223002221462846FFF778FB80
:1010800000280EDB4FF00008636B9E42C8D9012395
:1010900005AA214628468DF81480FEF763F900283A
:1010A000F2DA06B0BDE8F0816FF01500F9E700BF95
:1010B0009F5C02007E650200C8530200C95702000F
:1010C0006965020008B5806AFCF714FA30B9084B6C
:1010D000084A094841F2D47104F0DAF9D1E90B0267
:1010E000920303D54B6B984238BF184608BD00BF2A
:1010F0009F5C02005B650200C8530200FDF7A4BCC0
:1011000030B50C4D0A44914200D130BD11F8013B7D
:1011100083EA000404F00F0455F8244084EA101018
:1011200080EA131303F00F0355F8233083EA1010FD
:10113000E9E700BFD0660200032AF8B504460D4671
:10114000134602D84FF0FF30F8BD0A7802714A7892
:1011500042718A788271CA78C2710027042B0773A2
:101160004773077247728772C7721DD00E798681E6
:10117000052B0AD1866007734773AEB9002301229D
:1011800023726272A372E3720EE0002E3CD0721DD5
:1011900093420BD100683246053104F011FE012361
:1011A00027726372A772E7720020CDE7B21D9342E7
:1011B000C8D100683246053104F002FEA3892B44F1
:1011C0005B79A360002BD9D0EEE7B5F8052053BAC0
:1011D0009BB2A360002AE7D100230122237263722D
:1011E000A272D0E702F109018B42ABD12068E91D60
:1011F00004F0E6FDA3892B44DA791B7A43EA022343
:10120000A360002BE8D0CFE7072BDED0062B99D0C8
:10121000B5F8051048BA82B2A081002992D0D11D3C
:101220008B42DFD12068E91D04F0CAFD012326723C
:101230006672A372E672B7E770B50D4604460021E8
:101240002B79A27B03F0EF031ABB23716B796371D7
:10125000AB79A371EB79E371227362730126A673F4
:10126000A389AA8940F23C519818884222DC206860
:101270002968184404F074FEA389AA891344A38141
:101280002B7913F0100317D1A373AB68A36002206E
:1012900070BD22799A420BD162796B799A4207D15B
:1012A000A279AB799A4203D1E279EB799A42D5D00F
:1012B000A173C5E70320EBE73046E9E770B5038982
:1012C00084888A88E41AA4B294420D46016828BF33
:1012D0001446064622461944286804F041FEAC80B4
:1012E0003389E218B38892B29A42328109D2991AAC
:1012F000FF2908DC03F5C2439B1A9BB2EB80002058
:1013000070BDF388FAE746F2FF13F7E72DE9F843DB
:101310000379FF2B0C4613D14379EE2B10D183793F
:10132000FF2B0DD1C379EE2B0AD1FBF7B7FD0023BC
:1013300023716371A3716FF06F03E371BDE8F883EC
:10134000594F397801291CD14279584BCB2A0DD1FC
:1013500000221A70836840F23C52934228BF134621
:1013600083602146BDE8F843FAF732BC1D78012DB1
:1013700003D8C02A01D11970ECE70221DB2A1970C9
:10138000E8D04B4D01462846FFF756FF0128CED046
:10139000022840F08380AA6840F23C539A4228BF5A
:1013A0001A462B79AA6013F07F0009D16979C02908
:1013B00013D1A28021463F48BDE8F843FFF77EBF26
:1013C0003C4B00221A813B78013B062B25D8DFE8F5
:1013D00003F043484D533C595F00364AA42910811D
:1013E000F1D1AA79042AEED1EA791343EBD1DFF8DF
:1013F000C880DFF8C890012618F8012FAB89934206
:101400001FD359F82610286805F012FAC8B9F6B2A9
:10141000062E0AD1F1F72CFE60B900232371637107
:101420006FF07D03A3716A2387E7012E02BF1F4B74
:1014300002221A703B78B34201D000F079F83E7076
:10144000C1E70136082ED7D1E7E71A491848F8F75F
:1014500001FBAB68A380ADE716491548FAF7B8FB66
:10146000F7E714491248F6F7ABF8F2E721461048BF
:10147000BDE8F843F7F764BA21460D48BDE8F843E4
:10148000F1F760BE21460A48BDE8F843F6F7B2BF5F
:1014900021460748BDE8F843F6F70ABE002323714A
:1014A0006371A3716F2348E7FB1E0020BE19002063
:1014B000AA000020A00000201067020018670200A8
:1014C00038B5064D0446024601212846F1F718FCBE
:1014D0002868201A18BF4FF0FF3038BDBC0000202C
:1014E00010B5064C014601222046F1F709FC2068A0
:1014F000013818BF4FF0FF3010BD00BFBC00002006
:1015000008B50020F8F776F90020FAF707FA00206E
:10151000F7F798F90020F3F72BFF0020F1F7BEFD55
:101520000020F6F785FEBDE808400020F9F7C6BBAD
:1015300008B5FAF7D3F9F7F77BF9F1F7A9FDF8F752
:1015400047F9BDE80840F6F725BE30B5044609B3B3
:1015500094F900500078002D0BDB01241C6000245E
:1015600014602CB91B6803448B4284BF01231360B1
:1015700030BD812804D101290CD060780224EDE728
:10158000822807D1022905D9B4F8010040BA80B2F7
:101590000324E3E701240020E2E7000010B5064C35
:1015A000237823B9F1F7DDFB0123237010BDF1F798
:1015B000D5FB0023F9E700BFFC1E002008B5FBF7B0
:1015C0004DF80448FBF7F4FAFBF71EFDBDE80840B0
:1015D000FBF776BC39CB000008B500214FF0FF3097
:1015E00002F0CEFCFBF75AF80020FBF7F3FAFBF70A
:1015F00023FDBDE80840FBF76DBC000008B5F1F71E
:1016000095FB0A4A0346106870B9B3F5FA6F0AD918
:10161000074A1268A3F57A73934204D9054B1878E8
:10162000003818BF012008BD0020FCE7041F00207F
:10163000081F00200D1F0020014B1878704700BFC5
:101640000D1F0020014B1870704700BF0D1F0020B8
:10165000012808B501D1FBF793FA002008BD00006E
:10166000014B1878704700BF0C1F002070B50C4E5E
:10167000336804460D4693B9F1F758FB094B1860DF
:10168000094B1D6044B14FF47A7303FB04003060D2
:10169000BDE87040FFF782BF4FF0FF30F7E770BD45
:1016A000041F0020081F0020001F0020074B10B55A
:1016B00000241C60F1F7D4FC20B1F1F74FFB044B80
:1016C0001C7010BDF1F74DFB0124F8E7041F00204A
:1016D000FC1E00202DE9F047384B0546187810B95C
:1016E000C821FFF7C3FF364CF1F720FB277823789A
:1016F000012B0646FFB221D1DDB1012D1CD0DFF850
:10170000C480B14647F22F5A98F8003013B92378B5
:10171000052B15D1002388F800302378042B01D045
:10172000FFF7C4FF2378042B41D105232370002544
:101730001DE002232370E2E70323FBE70423F9E71C
:101740002378062BE6D02378032B01D1FAF7A6FFE6
:101750002078023818BF0120FBF73CFA0128054623
:101760000BD12378042B05D0FFF7A0FF2570284666
:10177000BDE8F08706232370F9E7F1F7D7FA831B5A
:101780005345054607D92378042B01D0FFF78EFF78
:1017900027700225EBE7A0EB0903632BB4D923786C
:1017A000022B02D00220FBF7EBF9A946ACE7237825
:1017B000062B4FF00103B9D12370EAE70C1F00207C
:1017C000C00000200D1F00202DE9F8430025164E13
:1017D0002F4615F0010F0CBF3221C8210220FFF760
:1017E00045FFF1F7A3FA4FF0000804463378012BC8
:1017F0005FFA83F906D13770FFF758FFF1F796FAD1
:10180000C8460446F1F792FA001BB0F5FA6FEDD323
:10181000B8F1000F05D00135052DDAD10020BDE863
:10182000F8834FF0FF30FAE70D1F002008B5F1F7FD
:101830007DFA0C4B1B689BB1984203D9BDE8084068
:10184000FFF734BF084A1368834209D8074909687B
:10185000C31A8B4204D31060BDE80840FFF79EBE58
:1018600008BD00BF041F0020081F0020001F00202B
:1018700001460148FEF7C6BF10210020014601487D
:10188000FFF736B81021002070B598B01E46164BF1
:1018900000930D4614460123024603A91348FFF79F
:1018A000CFFA002817DB22461048002303A9FFF7D0
:1018B00043FB041E11DB0D4833462A4603A9FFF7FC
:1018C000EFFA041E09DB094803A9FFF7D1FA10EA71
:1018D000200038BF204618B070BD044803A9FFF7A8
:1018E000C7FA2046F7E700BFC400002010210020FF
:1018F000F0B599B01D469DF87830002B174B00933A
:101900000E4640F20253174608BF4FF48173024659
:1019100003A91348FFF794FA041E0EDB10480023B6
:101920003A4603A9FFF708FB041E11DB45B90C4832
:1019300003A9FFF79DFA00EAE074204619B0F0BD54
:1019400007482B46324603A9FFF7DEFA041EEEDAFB
:1019500003A90348FFF78CFAEFE700BFC40000209B
:101960001021002070B598B0154B00930E46154617
:101970004FF48173024603A91248FFF761FA041E6F
:101980000EDB10480223002203A9FFF7D5FA041E3C
:1019900011DB45B90B4803A9FFF76AFA00EAE074C6
:1019A000204618B070BD07482B46324603A9FFF702
:1019B000ABFA041EEEDA03A90248FFF759FAEFE783
:1019C000C40000201021002030B599B00F4B0093C7
:1019D00002460D460E484FF4817303A9FFF730FA13
:1019E000041E0ADB03A90A482A46FFF7BDFA041EB3
:1019F00003A9074804DAFFF73BFA204619B030BDC7
:101A0000FFF736FA00EAE074F7E700BFC4000020F1
:101A10001021002007B5009313460A4601460348EB
:101A2000FFF7CAF903B05DF804FB00BF10210020E6
:101A300007B5009313460A4601460348FFF7F4F939
:101A400003B05DF804FB00BF1021002010B598B072
:101A50000D4B0093024601230C4803A9FFF7F0F950
:101A600000280ADB03A90948FFF72CFB041E03A981
:101A7000064804DAFFF7FCF9204618B010BDFFF75E
:101A8000F7F90028F8DAF8E7C40000201021002058
:101A9000044B9A6ED2E90730584348BF00F2FF303A
:101AA000801270471021002010B5074C2046FFF728
:101AB00025FB002806DBA36EDB69584348BF00F214
:101AC000FF30801210BD00BF102100200A460146E1
:101AD0000148FFF73FB800BF102100202DE9F04179
:101AE0000378052B06460D4620D8032B3C4F00F10A
:101AF0004C0121D922B157F8233002332B70012237
:101B00008623AB543078AB1857F8200058703378E0
:101B1000941C254457F82320284604F021FA3378F2
:101B2000052B20D1284606F0B1FB1CE0063B022B1A
:101B30001FD94FF0FF301AE022B157F8233003339A
:101B40002B7001228623AB54337857F82330A81822
:101B500001334370042383703378D41C281957F859
:101B6000232004F0FDF9337857F823002044BDE822
:101B7000F0811B4F6AB182230B70037857F8233032
:101B80000A331B0A4B70037857F823300A338B70E3
:101B900003228123AB54AB184FF0820883F80180F5
:101BA000317857F821103046090A997010F8081B4F
:101BB000141D57F82110D970291907F017FA31466A
:101BC000042211F80C3B57F823301C442B19A01C9D
:101BD00005F8048028445A7004F0C2F9A01DC6E735
:101BE000506A020010B50A44914201D3002010BD92
:101BF0000B4613F8014BAA2C03D0AB2C13D0114683
:101C0000F2E79A420AD94C78012C01F102031CD167
:101C10009A4203D989780139022919D8194611F84D
:101C2000013BC370E0E79A420AD94C78012C01F1DC
:101C300002030AD19A4203D989780139022907D8C7
:101C4000194611F8013B0371CEE74FF0FF30CEE7A4
:101C50006FF00100CBE700002DE9F04F00F108071D
:101C6000044689B00D4638464FF4A161164607F088
:101C700067F9022363702378052B05D99A1F022A7E
:101C80003FD94FF0FF302DE0DFF8249159F82320A1
:101C9000931CB342F5D82B78062B02D06FF00100CD
:101CA00020E06B789A4205F10208EAD141463846B5
:101CB00004F056F92078394606F0E0FC28B94FF4D4
:101CC000A261204607F03CF9E8E72078394606F0A3
:101CD000E3FF002809DA20464FF4A26107F030F94B
:101CE0006FF0020009B0BDE8F08F237859F8231097
:101CF0004144AA19521A204609B0BDE8F04FFFF737
:101D000071BFDFF8ACA05AF823301B0123814FF0DC
:101D10000123E36004F11003039304F58873049333
:101D200004F50473059304F54473069304F5826384
:101D30000793002EA5D00DF10C0929464FF001089C
:101D40000F4617F8013B4345A8D1791B02AB01AA06
:101D5000711A3846FFF7F9FB019B8346002B90D19F
:101D600023785AF82330834298D3029959F8040B08
:101D70000F44A3EB0B0339465A46184408F10108F7
:101D800004F0EEF8B8F1060F07EB0B010AD1236956
:101D9000064A1BBA934292D9D4F810311BBA934227
:101DA000A7D88CE74B1BB342CAD36AE733F304B519
:101DB000746A02002DE9F04F00F1080A044687B06A
:101DC0000E4650464FF4A161154607F0B9F80223BC
:101DD0009D42637020D933787F2B58D17378482B7C
:101DE00006F1020853D105AB04AAA91E4046FFF72D
:101DF000ACFB049B0290019373B9162847D8059A4F
:101E000008EB0203009303EB000B2378052B0AD9A0
:101E1000063B022B40F28A804FF0FF33019301987A
:101E200007B0BDE8F08F009B5F1CB91BA942F3D23D
:101E300018F80230922B2AD105AB04AA691A384649
:101E4000FFF783FB049B8046002BE5D12278354BBE
:101E500053F8223083421AD3059BF818834519D9C9
:101E60000130811BA942D7D2FB5C992B12D105AB63
:101E700004AA691AFFF769FB049B0746002BCBD124
:101E80002278294B53F822300133834203D26FF07A
:101E90000103C3E700270BF10209A9EB0601A942E0
:101EA000BAD2009B029A9B5C5F2BF0D19BF8013069
:101EB000482BECD105AB04AA691A4846FFF745FB4D
:101EC000049B002BE3D147448742E0D1059B227855
:101ED00009EB0301134B53F8220001EB08039B1B92
:101EE000AB42A0EB080097D84246504404F038F8C3
:101EF0002078514606F0C2FB28B94FF4A261204673
:101F000007F01EF8C3E72078514606F0C5FE00280A
:101F100085DA4FF4A261204607F012F86FF0020351
:101F20007CE700BF746A0200506A0200009B03F164
:101F30000109A9EB0601A942BFF46EAF18F80230FF
:101F4000912BA4D105AB04AA691A4846FFF7FDFA04
:101F5000049B002B7FF460AF042898D1059B09EB0C
:101F600003070137B91BA942BFF456AF19F8033074
:101F7000922B8CD105AB04AA691A3846FFF7E5FA13
:101F8000049B002B7FF448AFDFF80492237859F8C4
:101F9000233083427FF47BAF059B07EB030808F1F6
:101FA0000108A8EB0601A942BFF436AFFB5C932BF6
:101FB0007FF46DAF05AB04AA691A4046FFF7C5FA76
:101FC000049B002B7FF428AF237859F823308342F9
:101FD0007FF45DAF059B08EB03070137B91BA942EE
:101FE000BFF41AAF18F80330942B7FF450AF05AB51
:101FF00004AA691A3846FFF7A8FA049B8146002B09
:102000007FF40AAFDFF888A123785AF8233083429F
:10201000FFF43DAF059B07EB030808F10108A8EBAF
:102020000601A942BFF4F8AEFB5C952B7FF42FAFFD
:1020300005AB04AA691A4046FFF787FA049B0746D6
:10204000002B7FF4E9AE23785AF823308342FFF463
:102050001EAF059B08EB03000130811BA942BFF4B2
:10206000DBAE18F80330962B7FF411AF05AB04AA52
:10207000691AFFF76AFA049B8246002B7FF4CCAE04
:10208000DFF80C81237858F823308342FFF4FFAE49
:102090000BF10203991BA9420393BFF4BDAE009B51
:1020A000029A9B5C5F2B7FF4F2AE9BF80130482BC9
:1020B0007FF4EDAE05AB039804AA691AFFF745FA61
:1020C000049B002B7FF4A8AE237858F8232009EB5B
:1020D000420304333B44534483427FF4D8AE059912
:1020E0000398084403449B1BAB4283463FF694AEDF
:1020F00012010146228104F10C00042203F030FF9A
:1021000020460BF1040B10F8103B594658F82320D9
:1021100003F026FF237858F823209344594604F50A
:10212000887003F01DFF237858F8233004F582608F
:102130009B44A3EB090359464A46184403F010FF99
:10214000237858F82330CB44DB1B04F504703A465F
:102150005946184403F004FF237858F8233004F557
:102160004470A3EB0A03524618440BEB070103F03B
:10217000F7FE2369054A1BBA93427FF6BEAED4F838
:1021800010311BBA93423FF64AAEB6E633F304B5BC
:10219000746A02000A460523FF21FFF73BBC0A468A
:1021A0000523FF21FFF744BC70B504460D46FFF739
:1021B000F1FF002809DB05F1080120464FF4A16377
:1021C000BDE870400022FFF75FBB70BD37B501234B
:1021D00000930C464FF4A163002208310546FFF737
:1021E00087FB002806DB2146284603B0BDE83040C7
:1021F000FFF7D5BF03B030BD10B5012304464370CF
:10220000007805280FD804F1080106F015FD002814
:1022100001DB002010BD4FF4A261204606F090FEC5
:102220004FF0FF30F6E7831F022BF9D8044B53F829
:102230002010C90089B204F1080006F0A3FEE6E709
:10224000506A0200F7B504460078052811D80093BB
:1022500013460A4604F1080106F07EFC002805DB5F
:102260002278084B53F8220003B0F0BD4FF0FF3046
:10227000FAE706380228F9D804F1080006F02CFF26
:10228000ECE700BF2C6A020030B585B0C41C012504
:102290008DF80F300095134620460022FFF728FBEB
:1022A000002803DA4FF0FF3005B030BD2B460DF1AA
:1022B0000F0200212046FFF7BBFB0028F2DB2B4674
:1022C0000DF10F0229462046FFF7B2FBC017EBE7DE
:1022D0002DE9F0431E460378894693424FF00001F2
:1022E00093B00546144681705FD8437893425CD31F
:1022F000C71C01230DF107023846FFF78BFB0028AE
:102300002DDB9DF8073006B133708BB340230022DC
:1023100002A93846FFF7B8FAB0F100081FDB2246E1
:1023200002A9484605F03FFEB4EB080418BF01249B
:10233000844220D09DF80720013AD2B28DF80720C0
:1023400006B1327001230DF1070200213846FFF774
:102350006FFB002808DA402102A806F0F1FD4FF0DB
:10236000FF3013B0BDE8F083402102A806F0E8FD7D
:102370006FF00100F5E70124AC7023460DF1070270
:1023800021463846FFF746FB0028E4DB23460DF1E3
:10239000070200213846FFF74BFB0028DBDB02A8D1
:1023A000402106F0CDFD0020DBE76FF00200D8E70A
:1023B0007FB5134602789A4223D842789A4220D3B6
:1023C0000026C41C01258670324600952046FFF782
:1023D0008FFAB04203DA4FF0FF3004B070BD2B46E5
:1023E0000DF10F0229462046FFF714FB0028F2DB0F
:1023F0002B460DF10F0231462046FFF719FBC0179F
:10240000EBE76FF00200E8E70330FFF71FBB13B5FF
:10241000C41C2046FFF71AFB60B101230DF107022F
:1024200000212046FFF7F6FA0028ACBF9DF8070010
:102430004FF0FF3002B010BD13B5C41C2046FFF7AB
:1024400005FB60B101230DF1070219462046FFF795
:10245000E1FA0028ACBF9DF807004FF0FF3002B052
:1024600010BD30B585B00023C41C012500951A4667
:1024700019462046FFF73CFA002803DA4FF0FF30F8
:1024800005B030BD2B460DF10F0229462046FFF75F
:10249000C1FA0028F2DB2B460DF10F020021204685
:1024A000FFF7C6FAC017EBE783680BB1013B836007
:1024B00070472DE9F041C56815F001050446164640
:1024C000D0E9007003D0BC46BDE8F0416047C31BB3
:1024D000934209DA10B1C4E90055D61A236833448F
:1024E00023604FF0004505E0384603F039FD2368CE
:1024F000334423602846BDE8F081F0B51C4687B020
:1025000013BA21BACDE900131746694606460822D8
:1025100004A89DF8305003F023FD182F74F1000338
:102520000DF117010CD29DF817302B448DF81730A0
:1025300006AA0023521A3046FFF7BBFF07B0F0BDD2
:10254000B7F5807F74F100030FD3B7F5803F74F1C6
:1025500000030CD3002C14BF0323022301229A4052
:10256000891A18352B440B70E2E70023F6E70123A4
:10257000F4E773B51E46FFF797FF009200230A4663
:1025800005460C46FFF7B9FF002808DC0123224668
:102590003146284602B0BDE87040FFF78ABF02B05E
:1025A00070BD7FB51D4603680B6043684B60FFF745
:1025B0007BFF0646531C05F020008B60C8600C466C
:1025C000F16801F001010143561CE1600ED141F0B8
:1025D0001001E1601F35002301220DF10F0120469B
:1025E0008DF80F50FFF765FF04B070BD08B11344BC
:1025F000A360009500232046FFF77FFFF4E701600A
:1026000011440222C0E902234160704707B5194610
:10261000FFF74AFF002300930B46FFF76EFF03B05E
:102620005DF804FB13B5DC171946FFF73DFF04F016
:1026300020030093624084EA0103FFF75EFF02B0CB
:1026400010BDA1F11903062B07B50A4609D9FFF7FA
:102650002BFFE02300930023FFF74FFF03B05DF84B
:1026600004FB4FF48370F9E70B4611464022FFF755
:1026700080BF0B4611466022FFF77BBF8023FFF728
:1026800090BF10B402F100436FF00044A34204D3A2
:102690005DF8044BA023FFF784BF4FF480605DF822
:1026A000044B704713B54B6843600C680460CA68FC
:1026B000D2060AD5FF238DF80730012200230DF141
:1026C0000701FFF7F6FE02B010BD8A68012A06D0A6
:1026D000002A40F2013008BF4FF44070F3E7B3FA2C
:1026E00083F04009C007EEE710B40468406823682F
:1026F0002479E40703D51B685DF8044B1847181AC2
:10270000884234BF002001205DF8044B704730B48C
:102710000346D0E900402579ED0703D5236830BC96
:102720009B6818470844586030BC704700F0DF00D1
:10273000402803D0803818BF012070470020704720
:102740000120704703F00CBC08B504F071F8B0FA32
:1027500080F0400908BDF0B40446D4E9007497F84D
:1027600004C01CF0010F0846154605D038684568BE
:102770002046AC46F0BC604761191A46F0BC03F035
:10278000EFBB70B50D4601210446FFF7ADFF38B130
:10279000294620460123BDE870400022FFF7DBBF39
:1027A00070BD0000F7B5FF238373C37B03F06003A4
:1027B000C3730DF106010446FFF7E3FF002800F0A4
:1027C00090809DF8065005F0E00605F01F051B2DD2
:1027D000A6738DF80650A5811BD91F2D08D040F295
:1027E000031040F20513E02E18BF184603B0F0BDE9
:1027F0003046FFF79BFF28B9E37B43F01003E373F8
:102800000020F3E7E02E40F2051008BF4FF481707E
:10281000ECE7172D18D90127A5F1180107FA01F1E6
:1028200039442046FFF760FF00285AD00023182DB6
:10283000A38114D13B463A460DF107012046FFF72C
:102840008AFF9DF80730A381202E4FEA56131AD134
:10285000E37B43F00403E3730023A373D0E7192D54
:1028600009D102233A4604F10C012046FFF773FF19
:10287000A3895BBAE7E79DF80630E27B03F0030328
:102880001343E373E0E7072BBAD19DF80630143BFE
:102890000B2BB5D8DFE803F0060E0E0E160E0A0A53
:1028A0001E1E1E1E0023A381F523D6E7E37B43F003
:1028B0000203E3730123002204F10E012046FFF717
:1028C0004AFF9DE7A3891F2B9AD8FF23A3734FF4D8
:1028D00083708BE7044B054A05484FF4807102F082
:1028E000D7FD40F2011081E7145502002468020070
:1028F000025D020037B585686B1C044618D10DF1E6
:102900000701FFF73EFF98B19DF80730FF2B0FD16D
:10291000E37B03F06002602A0ED0A27BC02A0BD0BA
:10292000002043F01003A573A060E37303B030BD33
:102930002046FFF737FFF9E74FF48170F6E7836829
:10294000827B591C0BD0C02A07D0013BC27B83601D
:1029500043B1C37B83F04003C373FFF7CBBFC02AEF
:10296000FBD0F6E7FF2122F010028173C2731846F4
:1029700070472DE9FF41C37B13F0140F05460F4646
:10298000164604D140F2071004B0BDE8F0810DF105
:102990000701FFF7F6FE10B940F20110F4E79DF8C9
:1029A0000730FF2BEED0A97B23F01F028A424ED1C5
:1029B00003F01F03172B8DF8073004D83360012470
:1029C0003C600020E0E71B2B44D84FF00108A3F146
:1029D000180408FA04F4444421462846FFF784FE0C
:1029E0000028D9D09DF80730192B15D80BD1022318
:1029F000424602A92846FFF7AEFEBDF808305BBA92
:102A00009BB23360DCE74346424602A92846FFF703
:102A1000A2FE9DF80830F4E71A2B08D104234246A1
:102A200002A92846FFF797FE029B1BBAE9E7082395
:102A300042460DEB03012846FFF78DFEDDE9022338
:102A40001BBA3360002ABBD04FF480609CE74FF480
:102A5000827099E740F2051096E72DE9F3410E46A2
:102A600001A904461746FFF784FF0546F0B9D4E9EB
:102A700000301979019A3F68C90708D51B683146AB
:102A8000D3F80C803B46C04760B105460EE01044C9
:102A9000606039462046FFF727FE58B16268326011
:102AA0003A446260E37B23F00403E373284602B0F8
:102AB000BDE8F08140F20115F8E7000013B5C17BD5
:102AC0008B070BD4837B0633DBB2012B06D90F4B6C
:102AD0000F4A10484FF4A47102F0DAFC11F001041F
:102AE0000AD0694608230122FFF735FE01980099B4
:102AF00000BA09BA02B010BD694604230122FFF7EB
:102B00002AFE0098214600BAF4E700BF425D0200A9
:102B100033680200025D020073B5C47B14F0020446
:102B200005461FD0FFF7CAFF06460C460DF1070108
:102B3000002201232846FFF70EFE9DF8073003F020
:102B40001F03172B88BF01218DF8073086BF183B64
:102B50009940002128460131FFF7D9FD3046214632
:102B600002B070BD8689E1E710B50446FFF7D4FFD7
:102B7000A37B03F0DF03402B13D131B10B4B0C4A85
:102B80004FF49A710B4802F083FCE37BDB0604D51B
:102B9000094B074A40F23511F4E701462046FFF79A
:102BA000B6FD2046BDE81040FFF7C9BEB85D020083
:102BB000FA670200025D0200D15D02002DE9F041DA
:102BC000069D1C4607460E46904618463E4408227F
:102BD000002102F0A1FF266084F804800123C5E9EA
:102BE0000047AB600023EB732846BDE8F041FFF7D8
:102BF000D9BD000008B50346807BFF2806D10C4BE9
:102C00000C4A4FF4EA710C4802F042FCFFF78EFDCB
